:100000000C94F6230C9427240C9427240C94272476
:100010000C9427240C94B0570C9427240C94272478
:100020000C9427240C9427240C9427240C94DBBBD9
:100030000C9427240D947DAF0C9427240C94272432
:100040000C9427240D9420280C9427240C94272406
:100050000C9427240C9427240D94663E0D94ACA791
:100060000C9427240C94E2330C9427240C9427241A
:100070000C9427240C9427240C9427240C942724D4
:100080000C9427240C9427240C9427240C942724C4
:100090000C9427240C9427240C9427240C942724B4
:1000A0000C9427240C9427240C9427240C942724A4
:1000B0000C9427240C9427240C9427240C94272494
:1000C0000C9427240C9427240C9427240C942B3470
:1000D0000C9427240C9427240C9427240C94272474
:1000E0000C942724E5013D017D01DD01C701CB0111
:1000F00055018701AF017901BF01D30133015F01D0
:100100009B019D0149013F0197015D016101BB0117
:100110007301E701B7017F017B015301A301810155
:100120008901950163016F015B01AD01A10193019B
:100130008101B301D501BD014501E30135018B0109
:100140004F015901C501C901750137018F01A9018D
:10015000CD01C1015901B10167015101036EDB36C7
:100160003D9A9999993DABAAAA2A3E000000803F8A
:10017000084AD73B3BCE016E84BCBFFDC12F3D6C0E
:1001800074319ABD56833DDA3D00C77F11BED9E474
:10019000BB4C3E916BAAAABE000000803F072C7AA0
:1001A000A5BA6CC590DA3B9365FC8BBC53F810FD87
:1001B0003C5692834DBD879D3AB63DCBC9BF5BBED1
:1001C00073DA0FC93F05A84CCDB2D44EB93836A961
:1001D000020C50B9918688083CA6AAAA2ABE000043
:1001E00000803F07634236B79BD8A71A3968561874
:1001F000AEBAAB558C1D3CB7CC5763BD6DEDFD75EC
:100200003EF6177231BF000000803F08000000BEBC
:10021000922449123EABAAAA2ABECDCCCC4C3E00B9
:10022000000080BEABAAAAAA3E00000000BF0000EA
:1002300000803F0000000000084178D3BB4387D115
:10024000133D190E3CC3BD4282AD2B3E68EC827655
:10025000BED98FE1A93E4C80EFFFBE01C4FF7F3FB6
:100260000000000000000D94993F0D9498A90D9492
:10027000BBA90D94BD4F0D943A9D0D94F93E0D947C
:1002800058710D94345C0D94F54E0D94A6A90D94FF
:10029000FD8D0D9445710D94515F0D94E26D0D949B
:1002A000A2A90D94DBA90D9401A90D94653F0D94AD
:1002B00077AA0D94E0A90D9439A90D9492710D942B
:1002C000A73F0D9497710D9425A90D943B540D945F
:1002D000D7A90D942E510D94D96D0D94007F0D94D6
:1002E0002FA90D94C3620D94AC710D94B7A90D9410
:1002F000C16F0D946F3F0D94F7A80D94153F0D94A9
:10030000F2A80D9484A90D94C8700D94956E0D9467
:10031000693F0D9415A90D949CA90D94D06D0D9471
:10032000BFA90D941E740D945CA90D941DA90D9484
:100330006D710D948C7C0D94C73F0D9435710D94A7
:1003400080670D9452A90D940BA90D943A620D94F7
:10035000FB4E0D94C5A90D94BC650D9443A90D9455
:100360006B3F0D94D3A90D9466A90D947B960D94C3
:10037000EDA80D94EB6D0D949C710D947AA90D94DC
:10038000713F0D94CDA90D94022B0D94ADA90D9440
:100390003D3F0D94B1A90D944B3F0D94C9A90D9407
:1003A0002E050D9401770D947F3F0D9470A90D9447
:1003B000A54C0D94E64E0D9469800D94233F0D9449
:1003C000504B0D945D4E0D94A9A90D94EB3E0D94E8
:1003D000BC710D94646C0D94568848617264636FAF
:1003E0006465642044656661756C7420536574743B
:1003F000696E6773204C6F616465640053746F723B
:1004000065642073657474696E67732072657472B5
:10041000696576656400202020452F44203D20003A
:100420002020204D393030204B004C696E656172C0
:1004300020616476616E63652073657474696E67AC
:10044000733A0046696C616D656E742073657474EF
:10045000696E67733A2044697361626C6564002059
:1004600020204D32303020440046696C616D656E4D
:10047000742073657474696E67733A002020204D90
:100480003230392053004175746F2D52657472619A
:1004900063743A20533D3020746F20646973616245
:1004A0006C652C203120746F20696E7465727072D7
:1004B000657420657874727564652D6F6E6C792033
:1004C0006D6F7665732061732072657472616374F9
:1004D00073206F72207265636F7665726965730051
:1004E0002046002020204D323038205300526563D2
:1004F0006F7665723A20533D4578747261206C6561
:100500006E67746820286D6D2920463A53706565C2
:100510006420286D6D2F6D2900205A002046002090
:1005200020204D323037205300526574726163745D
:100530003A20533D4C656E67746820286D6D292004
:10054000463A537065656420286D6D2F6D29205AD9
:100550003A205A4C69667420286D6D2900204400A9
:100560002049002020204D33303420500050494491
:1005700020686561746265642073657474696E6770
:10058000733A002044002049002020204D333031B0
:100590002050005049442073657474696E67733A43
:1005A00000205A0020590020204D323036205800BB
:1005B000486F6D65206F666673657420286D6D29C0
:1005C0003A00204500205A002059002058002042BF
:1005D0000020540020204D323035205300416476F5
:1005E000616E636564207661726961626C65733AFD
:1005F00020533D4D696E20666565647261746520A7
:10060000286D6D2F73292C20543D4D696E20747216
:100610006176656C20666565647261746520286D1D
:100620006D2F73292C20423D6D696E696D756D20AB
:100630007365676D656E742074696D6520286D73D0
:10064000292C20583D6D6178696D756D20585920B1
:100650006A65726B20286D6D2F73292C20205A3DFE
:100660006D6178696D756D205A206A65726B2028FE
:100670006D6D2F73292C2020453D6D6178696D7556
:100680006D2045206A65726B20286D6D2F732900DF
:1006900020540020204D32303420530041636365E4
:1006A0006C65726174696F6E3A20533D6163636576
:1006B0006C65726174696F6E2C20543D7265747242
:1006C00061637420616363656C65726174696F6EE8
:1006D00000204500205A0020590020204D323031A2
:1006E0002058004D6178696D756D20416363656CBC
:1006F00065726174696F6E20286D6D2F7332293AAF
:1007000000204500205A0020590020204D3230336F
:100710002058004D6178696D756D2066656564725D
:100720006174657320286D6D2F73293A0020450090
:10073000205A0020590020204D393220580053748F
:100740006570732070657220756E69743A00536528
:100750007474696E67732053746F726564004545E5
:1007600050524F4D204572726F72000020006D652F
:10077000736820626564206C6576656C696E673AA3
:10078000200029002C20002C2000706879736963F8
:10079000616C20636F6F7264696E617465733A2077
:1007A000280029002C20002C2000776F726C642018
:1007B000636F6F7264696E617465733A20280020FC
:1007C00046002045004731205A004D3234004D325A
:1007D000362053256C75004D31303620530047319B
:1007E000204625640047312045312046343830000A
:1007F0004731205A0020463230303000205900471F
:10080000312058004D383300506F736974696F6E32
:1008100020726561642066726F6D20656570726F0D
:100820006D3A004D3233202573002E67636F00460A
:10083000656564726174653A007265636F766572AE
:100840005F6D616368696E655F73746174655F6134
:10085000667465725F706F7765725F70616E6963F1
:100860002C20696E697469616C20007265636F7613
:1008700065725F6D616368696E655F7374617465ED
:100880005F61667465725F706F7765725F70616ECD
:1008900069632C20696E697469616C2000726563FC
:1008A0006F7665725F6D616368696E655F737461B1
:1008B00074655F61667465725F706F7765725F7093
:1008C000616E69632C20696E697469616C200063D4
:1008D000757272656E745F706F736974696F6E5B49
:1008E0005A5F415849535D3A0043757272656E74A0
:1008F00020706F736974696F6E20595F4158495356
:100900003A0043757272656E7420706F7369746912
:100910006F6E20585F415849533A004166746572C2
:100920002077616974696E6720666F722074656DE7
:10093000703A00473120452D312046343830004789
:10094000312045352046313230004D3833004D31AD
:10095000393020532564004D31303920532564004F
:1009600047323820582059004731205A3235204626
:10097000383030004D31343020532564004D313053
:10098000342053256400494E54340055564C4F20B2
:100990002D20656E6400737470730055564C4F00C3
:1009A00020423A0020453A00543A005A206C6976B9
:1009B000652061646A757374206F7574206F66209A
:1009C00072616E67652E2053657474696E6720745A
:1009D0006F20302E20436C69636B20746F20636F2F
:1009E0006E74696E75652E005A206C69766520619B
:1009F000646A757374206F7574206F662072616EFF
:100A000067652E2053657474696E6720746F20309B
:100A10000020573A0020453A00543A004B494C4CCC
:100A20003A20004175746F0020452F443D00416419
:100A300076616E6365204B3D0022283229004431E7
:100A400030303000473238205900473238205800C3
:100A50005400496E76616C6964205420636F64654C
:100A60002E00496E76616C6964204D20636F646569
:100A70002E004D3232302053256900203A200000EC
:100A80004C414E472053454C20464F52434544006D
:100A9000222831290020453A00205A3A0020593AAC
:100AA0000020453A00205A3A0020593A00583A00AE
:100AB00020002E0020423A0020453A00543A0020FF
:100AC000413A0020503A002042403A0020403A008B
:100AD000202F003A00205400202F0020423A00200E
:100AE0002F006F6B20543A002569206D696E2C2011
:100AF00025692073656300496E76616C6964204DD9
:100B000020636F6465004D65736820626564206CC6
:100B10006576656C696E67206E6F742061637469B9
:100B200076652E000A002020000A4D6561737572FB
:100B3000656420706F696E74733A000A5A20736599
:100B400061726368206865696768743A20002C00E8
:100B50004E756D20582C593A2000476F20686F6DF4
:100B6000652066696E6973686564004D6573682009
:100B7000626564206C6576656C696E67206163747C
:100B800069766174656400557073616D706C652081
:100B900066696E697368656400426564206C657699
:100BA000656C696E6720636F7272656374696F6EDE
:100BB0002066696E697368656400206D6963726F91
:100BC0006E7300457863657373697665206265644A
:100BD000206C6576656C696E6720636F7272656301
:100BE00074696F6E3A200042656420636F727265AB
:100BF0006374696F6E2064617461206E6F74207617
:100C0000616C69640A0042656420636F7272656397
:100C100074696F6E20646174612076616C69640A26
:100C2000006261627973746570206170706C6965CF
:100C30006400636C65616E2075702066696E69730F
:100C400068656420004D4553485F484F4D455F5AE5
:100C50005F5345415243483A20004D657368206216
:100C60006564206C6576656C696E67207768696C71
:100C700065206C6F6F702066696E69736865642E9D
:100C80000000206F66667365743A20006D657368B6
:100C900020626564206C6576656C696E673A200039
:100CA0000A00593A200000583A20003A206E6F207E
:100CB000787920636C616D70696E670A003A2078FC
:100CC0007920636C616D7065642E0A00002C2063CE
:100CD000616C6962726174696F6E207A3A200042B9
:100CE0006564206C6576656C696E672C20706F6931
:100CF0006E743A2000005A206A6974746572206428
:100D00006174612066726F6D205A2063616C2E20C1
:100D10006E6F742076616C69642E0A005A206A69CD
:100D20007474657220646174612066726F6D205AFC
:100D30002063616C2E2076616C69642E0A004E6F10
:100D400020636C616D70696E6720666F72206669E2
:100D50007273742063616C6962726174696F6E2072
:100D6000706F696E742E0A00466972737420636135
:100D70006C6962726174696F6E20706F696E742045
:100D8000636C616D7065642E0A00473238205730FD
:100D9000003A200054656D7065726174757265204B
:100DA00063616C6962726174696F6E20646F6E65F5
:100DB0002E20436F6E74696E7565207769746820A4
:100DC0007072657373696E6720746865206B6E6FEF
:100DD000622E0000205A20736869667420286D6DA9
:100DE000293A0050494E44412074656D7065726126
:100DF000747572653A2000002F3600537465703A9E
:100E0000200000205A20736869667420286D6D29BF
:100E10003A0050494E44412074656D7065726174AA
:100E20007572653A20002F362028736B69707065E3
:100E3000642900537465703A2000005A45524F3AB5
:100E400020000073746172742074656D7065726146
:100E5000747572653A200050494E44412070726F9B
:100E600062652063616C6962726174696F6E207380
:100E70007461727400473238205730000A00205ADB
:100E80003A200020593A200020583A2000473238B2
:100E90002C2066696E616C20004732382C20666910
:100EA0006E616C20004732382C2066696E616C20C0
:100EB000004732382C20696E697469616C200047E4
:100EC00032382C20696E697469616C2000443939AC
:100ED00039004D3239002055706C6F616420696EA5
:100EE0002070726F677265737300696E69746961EF
:100EF0006C207A73746570732061667465722072F9
:100F0000657365743A2000696E697469616C207A52
:100F10007374657073206F6E20706F7765722075C3
:100F2000703A2000466163746F72792052455345D0
:100F3000540020202020334420205072696E7465B4
:100F4000727320202020002020204F726967696E74
:100F5000616C205072757361202020004F637420F3
:100F60003234203230313700436F6D70696C656404
:100F70003A2000286E6F6E652C2064656661756C82
:100F80007420636F6E66696729004F637420323482
:100F900020323031372031393A34303A3438007326
:100FA0007461727400202020203344202050726924
:100FB0006E7465727320202020002020204F7269FB
:100FC00067696E616C205072757361202020002566
:100FD000002020202020200020202020202000454C
:100FE000524153494E4720616C6C2064617461002A
:100FF000466163746F727920524553455400FFFF78
:10100000FF0000A0400000A0400000004000007F62
:101010004300005E439AD9514300000000000040A5
:10102000C19A99193E00007F4300005243000052CC
:101030004300000000000040C19A99193E656368B2
:101040006F3A004572726F723A0000002110422020
:1010500063308440A550C660E770088129914AA199
:101060006BB18CC1ADD1CEE1EFF131121002733210
:101070005222B5529442F772D662399318837BB3E9
:101080005AA3BDD39CC3FFF3DEE3622443342004A0
:101090000114E664C774A44485546AA54BB5288539
:1010A0000995EEE5CFF5ACC58DD5533672261116F0
:1010B0003006D776F6669556B4465BB77AA7199789
:1010C0003887DFF7FEE79DD7BCC7C448E558866878
:1010D000A7784008611802282338CCC9EDD98EE9D9
:1010E000AFF9488969990AA92BB9F55AD44AB77A50
:1010F000966A711A500A333A122AFDDBDCCBBFFB29
:101100009EEB799B588B3BBB1AABA66C877CE44C5F
:10111000C55C222C033C600C411CAEED8FFDECCD78
:10112000CDDD2AAD0BBD688D499D977EB66ED55E2F
:10113000F44E133E322E511E700E9FFFBEEFDDDFC8
:10114000FCCF1BBF3AAF599F788F8891A981CAB154
:10115000EBA10CD12DC14EF16FE18010A100C23086
:10116000E3200450254046706760B9839893FBA341
:10117000DAB33DC31CD37FE35EF3B1029012F322D6
:10118000D2323542145277625672EAB5CBA5A89591
:1011900089856EF54FE52CD50DC5E234C324A01426
:1011A00081046674476424540544DBA7FAB7998721
:1011B000B8975FE77EF71DC73CD7D326F236910676
:1011C000B01657667676154634564CD96DC90EF969
:1011D0002FE9C899E9898AB9ABA9445865480678C6
:1011E0002768C018E1088238A3287DCB5CDB3FEB81
:1011F0001EFBF98BD89BBBAB9ABB754A545A376A16
:10120000167AF10AD01AB32A923A2EFD0FED6CDD50
:101210004DCDAABD8BADE89DC98D267C076C645C65
:10122000454CA23C832CE01CC10C1FEF3EFF5DCF60
:101230007CDF9BAFBABFD98FF89F176E367E554EB5
:10124000745E932EB23ED10EF01E7C3C3E5E2B3D72
:101250003F2F5B5D3B2C2A225C004D383420582008
:1012600059205A2045004D3234004D323320257329
:10127000006175746F25692E67000A002F000A004F
:101280002E0044656C6574696F6E206661696C65DB
:10129000642C2046696C653A200046696C652064C0
:1012A000656C657465643A002E002E002E002E00D9
:1012B0004E6F772066726573682066696C653A20A8
:1012C000004E6F7720646F696E672066696C653ABF
:1012D00020002220706F73002220706172656E748E
:1012E0003A2200535542524F5554494E45204341EE
:1012F0004C4C207461726765743A2200747279698B
:101300006E6720746F2063616C6C207375622D674B
:10131000636F64652066696C657320776974682003
:10132000746F6F206D616E79206C6576656C732EBD
:10133000204D4158206C6576656C2069733A002514
:101340006920686F757273202569206D696E7574E8
:1013500065730054494D454F55543A004D31313075
:101360000046756C6C2052582042756666657200A6
:1013700022206661696C65643A2042756666657212
:101380002066756C6C2100456E717565696E67200D
:10139000746F207468652066726F6E743A20220044
:1013A0002200456E717565696E6720746F207468E0
:1013B000652066726F6E743A202200222066616991
:1013C0006C65643A204275666665722066756C6C61
:1013D000210022004D363030005072757361206953
:1013E00033204D4B332072656164792E007A5F6D36
:1013F000696E3A20007A5F6D61783A20005A204F7A
:10140000666673657400795F6D696E3A2000795F76
:101410006D61783A200059657300785F6D696E3AA6
:101420002000785F6D61783A20002057617463680E
:10143000646F6720526573657400496E666F207330
:10144000637265656E0057616974696E6720666FC7
:1014500072206E6F7A7A6C6520616E6420626564BA
:1014600020636F6F6C696E67005761697420666FE7
:101470007220757365722E2E2E005573656420647C
:101480007572696E67207072696E7400556E6C6F4C
:1014900061642066696C616D656E7400556E6C6F79
:1014A0006164696E672066696C616D656E74005574
:1014B0006E6B6E6F776E20636F6D6D616E643A2038
:1014C000220054756E650053442063617264205B92
:1014D000466C73684169725D0053442063617264B5
:1014E000205B6E6F726D616C5D0054656D702E20B7
:1014F00063616C2E205B4F4E5D0054656D702E2035
:1015000063616C2E205B4F46465D0054656D7065CF
:101510007261747572652063616C6962726174696D
:101520006F6E2069732066696E69736865642E202A
:10153000436C69636B20746F20636F6E74696E75A2
:10154000652E0054656D702E2063616C2E20202066
:10155000202020202020200054656D706572617469
:1015600075726500537570706F72740053746F708C
:10157000207072696E740053544F505045442E20B1
:1015800000537465707261746520746F6F206869B0
:1015900067683A2000546F74616C207072696E74D1
:1015A0002074696D65203A00546F74616C2066691F
:1015B0006C616D656E74203A005072696E742074AF
:1015C000696D653A20200046696C616D656E742016
:1015D000757365643A20200053746174697374698B
:1015E00063732020004572726F72202D2073746126
:1015F000746963206D656D6F727920686173206214
:1016000065656E206F7665727772697474656E00B9
:1016100053706565640020536F667477617265204E
:101620005265736574004D6F646520202020205B37
:1016300073696C656E745D004D6F6465205B6869ED
:10164000676820706F7765725D0053686F772065FB
:101650006E642073746F7073005365742074656DCD
:1016600070657261747572653A0053657474696E61
:10167000677300576972696E67206572726F7200D6
:1016800053656C6620746573742073746172742082
:101690002000506C6561736520636865636B203A58
:1016A0000053656C662074657374204F4B004E6F59
:1016B0007420636F6E6E6563746564004D6F746F44
:1016C00072004865617465722F546865726D697344
:1016D000746F720046616E20746573740053656C9C
:1016E0006674657374206661696C65642020004CC3
:1016F00065667420686F74656E642066616E3F0075
:1017000053656C6674657374206572726F72202104
:1017100000456E6473746F70206E6F742068697416
:1017200000456E6473746F707300456E6473746FFC
:10173000700046726F6E74207072696E74206661FC
:101740006E3F00436865636B696E67205A2061785D
:101750006973202000436865636B696E67205920B8
:1017600061786973202000436865636B696E672048
:10177000582061786973202000436865636B696E47
:101780006720686F74656E64202000436865636B32
:10179000696E6720656E6473746F7073004368656B
:1017A000636B696E67206265642020202020004101
:1017B0006C6C20636F72726563742020202020207F
:1017C00000426564202F204865617465720041788D
:1017D0006973206C656E67746800417869730053A3
:1017E000656C6674657374202020202020202020E2
:1017F0000057726974696E6720746F2066696C6542
:101800003A2000766F6C756D652E696E697420667E
:1018100061696C6564002053697A653A2000436110
:1018200072642072656D6F76656400534420707237
:10183000696E74696E67206279746520006F7065E7
:101840006E206661696C65642C2046696C653A207F
:10185000006F70656E526F6F74206661696C6564AD
:10186000004361726420696E73657274656400532D
:101870004420696E6974206661696C0046696C6514
:101880002073656C65637465640046696C65206FE0
:1018900070656E65643A20006572726F72207772AF
:1018A0006974696E6720746F2066696C65005344C3
:1018B0002063617264206F6B0043616E6E6F7420F1
:1018C000656E746572207375626469723A200052A5
:1018D0006573756D696E67207072696E740052650C
:1018E00073756D696E67207072696E7400526573EE
:1018F000756D65207072696E7400526573656E64F3
:101900003A2000426C61636B6F7574206F6363757E
:10191000727265642E205265636F766572207072F4
:10192000696E743F005265636F766572696E6720F9
:101930007072696E742020202000686F77746F2E9B
:10194000707275736133642E636F6D00666F7275AC
:101950006D2E707275736133642E636F6D007072DB
:1019600075736133642E636F6D005072696E7420FD
:10197000706175736564005072696E742061626F86
:1019800072746564005072696E7465722064697364
:10199000636F6E6E656374656400616E642070725F
:1019A00065737320746865206B6E6F62005072659A
:1019B0006865617420746865206E6F7A7A6C652141
:1019C000005072656865617400506F77657255707C
:1019D00000506C6561736520776169740020205048
:1019E0006C616E6E65724275666665724279746589
:1019F000733A200050494E44412048656174696E35
:101A000067005049442063616C2E20202020202054
:101A10002020202020005049442063616C2E206645
:101A2000696E6973686564005049442063616C693C
:101A300062726174696F6E005061757365207072B7
:101A4000696E7400506C6163652061207368656520
:101A500074206F6620706170657220756E646572A7
:101A600020746865206E6F7A7A6C6520647572697F
:101A70006E67207468652063616C69627261746965
:101A80006F6E206F66206669727374203420706FE9
:101A9000696E74732E20496620746865206E6F7AB3
:101AA0007A6C65206361746368657320746865206F
:101AB00070617065722C20706F776572206F66663A
:101AC00020746865207072696E74657220696D6D2E
:101AD0006564696174656C792E006F6B004F666692
:101AE000004E6F206D6F76652E004E6F20534420A0
:101AF00063617264004E6F7A7A6C650046696C614E
:101B00006D656E74206E6F74206C6F616465640027
:101B1000436F6C6F72206E6F7420636C656172002E
:101B20004E6F00506C6561736520757067726164FB
:101B3000652E004E6577206669726D77617265204B
:101B400076657273696F6E20617661696C61626C33
:101B5000653A004D6F7665205A004D6F76652059C5
:101B6000004D6F7665205800457874727564657213
:101B7000004D6F76652061786973004D657368204C
:101B8000426564204C6576656C696E670043616CE4
:101B90006962726174696F6E00206F662039004D52
:101BA0006561737572696E67207265666572656ED0
:101BB000636520686569676874206F662063616C7F
:101BC0006962726174696F6E20706F696E74004D26
:101BD00061696E004D32323120496E76616C696404
:101BE00020657874727564657220004D323138203A
:101BF000496E76616C69642065787472756465728B
:101C000020004D32303020496E76616C6964206569
:101C10007874727564657220005265706F727469B1
:101C20006E6720656E6473746F7020737461747571
:101C300073004649524D574152455F4E414D453A1A
:101C40004D61726C696E2056312E302E323B20531E
:101C50007072696E7465722F6772626C206D617349
:101C600068757020666F722067656E36204649522F
:101C70004D574152455F55524C3A68747470733AEF
:101C80002F2F6769746875622E636F6D2F70727580
:101C9000736133642F50727573612D69332D506CED
:101CA00075732F2050524F544F434F4C5F5645523F
:101CB00053494F4E3A312E30204D414348494E450D
:101CC0005F545950453A5072757361206933204D05
:101CD0004B332045585452554445525F434F554E5F
:101CE000543A3120555549443A3030303030303054
:101CF000302D303030302D303030302D30303030ED
:101D00002D3030303030303030303030300A004D0F
:101D100031303920496E76616C696420657874725F
:101D20007564657220004D31303520496E76616CE6
:101D3000696420657874727564657220004D313075
:101D40003420496E76616C696420657874727564BC
:101D5000657220004C6F6F73652070756C6C6579CF
:101D6000004C6F61642066696C616D656E74004C37
:101D70006F6164696E672066696C616D656E740081
:101D80004C6F6164696E6720636F6C6F720053659E
:101D90006C656374206C616E6775616765004B49A3
:101DA0004C4C45442E2000496E76616C6964206578
:101DB0007874727564657200496E7365727420661A
:101DC000696C616D656E74005072696E7420464175
:101DD0004E3A20004E6F7A7A6C652046414E3A00AA
:101DE000457874727564657220696E666F00206F45
:101DF00066203900496D70726F76696E6720626582
:101E0000642063616C6962726174696F6E20706FC7
:101E1000696E740043616C6962726174696E6720F7
:101E20005A0043616C6962726174696F6E20646FFD
:101E30006E650043616C696272617465205A004886
:101E4000656174696E6720646F6E652E0048656118
:101E500074696E670046696C2E2073656E736F72CD
:101E600020205B6F6E5D0046696C2E2073656E737B
:101E70006F72205B6F66665D002046726565204D5F
:101E8000656D6F72793A2000466C6F770046696E17
:101E9000697368696E67206D6F76656D656E7473C2
:101EA00000206F66203400536561726368696E6755
:101EB000206265642063616C6962726174696F6E2F
:101EC00020706F696E7400497465726174696F6E19
:101ED0002000446F6E6520736176696E67206669C5
:101EE0006C652E00446F6E65207072696E74696E49
:101EF000672066696C6500497320636F6C6F7220A0
:101F0000636C6561723F004368616E676520666956
:101F10006C616D656E740046616E207370656564FA
:101F200000656E717565696E672022004578747270
:101F300075646572002045787465726E616C20521C
:101F400065736574005072696E7465722073746F86
:101F5000707065642064756520746F206572726F9F
:101F600072732E2046697820746865206572726FDE
:101F70007220616E6420757365204D393939207483
:101F80006F20726573746172742E202854656D70B1
:101F9000657261747572652069732072657365740A
:101FA0002E205365742069742061667465722072F6
:101FB000657374617274696E6729004E6F204C6995
:101FC0006E65204E756D6265722077697468206356
:101FD0006865636B73756D2C204C617374204C695C
:101FE0006E653A20004E6F20436865636B73756DB4
:101FF0002077697468206C696E65206E756D626506
:10200000722C204C617374204C696E653A2000205C
:10201000746F6F206C6F6E6720657874727573696A
:102020006F6E2070726576656E746564004C696EC3
:1020300065204E756D626572206973206E6F742025
:102040004C617374204C696E65204E756D626572CB
:102050002B312C204C617374204C696E653A200042
:102060005072696E7465722068616C7465642E20AC
:102070006B696C6C28292063616C6C65642100209D
:10208000636F6C6420657874727573696F6E20700D
:10209000726576656E74656400636865636B7375FD
:1020A0006D206D69736D617463682C204C6173746D
:1020B000204C696E653A20004552524F523A004515
:1020C0006E642066696C65206C697374006F70655E
:1020D0006E0054524947474552454400656E64734B
:1020E000746F7073206869743A2000536C65657072
:1020F0002E2E2E0044697361626C652073746570C6
:10210000706572730043757272656E74004372611C
:102110007368206465742E2020205B6F6E5D004321
:1021200072617368206465742E20205B6F66665D43
:102130000020436F756E7420583A20004368616E2A
:1021400067656420636F72726563746C793F0043E6
:102150006F6F6C646F776E00204C617374205570E4
:1021600064617465643A200043686F6F736520652D
:10217000787472756465723A004368616E676520B1
:102180007375636365737321005072696E742066A2
:10219000726F6D2053440054656D702E2063616C26
:1021A0006962726174696F6E0043616C6962726129
:1021B00074696E67205A2E2E2E0043616C6962721C
:1021C0006174650052657365742058595A206361C3
:1021D0006C6962722E0043616C6962726174652081
:1021E00058595A002042726F776E206F75742052D2
:1021F0006573657400426567696E2066696C652069
:102200006C6973740058595A2063616C6962726119
:1022100074696F6E20636F6D70726F6D6973656442
:102220002E204C6566742066726F6E742063616C3C
:102230006962726174696F6E20706F696E74206E6E
:102240006F7420726561636861626C652E00585915
:102250005A2063616C6962726174696F6E20636F8A
:102260006D70726F6D697365642E2046726F6E7447
:102270002063616C6962726174696F6E20706F694E
:102280006E7473206E6F7420726561636861626C36
:10229000652E0058595A2063616C696272617469D5
:1022A0006F6E20616C6C2072696768742E20582FE5
:1022B0005920617865732061726520736C69676865
:1022C000746C7920736B657765642E20476F6F643B
:1022D000206A6F62210058595A2063616C696272EA
:1022E0006174696F6E20616C6C2072696768742E0E
:1022F00020536B65772077696C6C20626520636F73
:1023000072726563746564206175746F6D61746960
:1023100063616C6C792E0058595A2063616C696254
:10232000726174696F6E206661696C65642E20420B
:1023300065642063616C6962726174696F6E20709C
:102340006F696E7420776173206E6F7420666F758D
:102350006E642E0058595A2063616C696272617410
:10236000696F6E206F6B2E20582F5920617865732E
:10237000206172652070657270656E646963756C4A
:1023800061722E20436F6E67726174756C6174693F
:102390006F6E73210058595A2063616C69627261D3
:1023A00074696F6E206661696C65642E20506C657F
:1023B00061736520636F6E73756C7420746865203B
:1023C0006D616E75616C2E0058595A2063616C699D
:1023D00062726174696F6E206661696C65642E203B
:1023E0004C6566742066726F6E742063616C6962FE
:1023F000726174696F6E20706F696E74206E6F7495
:1024000020726561636861626C652E0058595A20BC
:1024100063616C6962726174696F6E206661696C78
:1024200065642E2046726F6E742063616C696272FF
:102430006174696F6E20706F696E7473206E6F7453
:1024400020726561636861626C652E00426564207C
:102450006C6576656C696E67206661696C65642E73
:102460002053656E736F7220646973636F6E6E655F
:1024700063746564206F72206361626C65206272B0
:102480006F6B656E2E2057616974696E6720666F89
:10249000722072657365742E00426564206C6576E7
:1024A000656C696E67206661696C65642E20536592
:1024B0006E736F72206469646E74207472696767EA
:1024C00065722E20446562726973206F6E206E6F94
:1024D0007A7A6C653F2057616974696E6720666F10
:1024E000722072657365742E00426564206C657697
:1024F000656C696E67206661696C65642E20536542
:102500006E736F7220747269676765726564207498
:102510006F6F20686967682E2057616974696E67FC
:1025200020666F722072657365742E0042656420A8
:1025300048656174696E670042656420646F6E650A
:1025400000526967687420736964655B756D5D002E
:102550005265736574005265617220736964652009
:102560005B756D5D00426564206C6576656C20630B
:102570006F7272656374004C65667420736964657C
:10258000205B756D5D0046726F6E742073696465C3
:102590005B756D5D004265640044697374616E63D0
:1025A00065206265747765656E20746970206F665A
:1025B00020746865206E6F7A7A6C6520616E642085
:1025C0007468652062656420737572666163652056
:1025D000686173206E6F74206265656E2073657428
:1025E000207965742E20506C6561736520666F6C70
:1025F0006C6F7720746865206D616E75616C2C203E
:1026000063686170746572204669727374207374B4
:102610006570732C2073656374696F6E20466972F0
:102620007374206C617965722063616C6962726198
:1026300074696F6E2E004C6976652061646A7573EB
:1026400074205A0041646A757374696E67205A0079
:102650004175746F20686F6D6500207C2041757432
:10266000686F723A2000416C6C0041637469766552
:102670002045787472756465723A2000D913ED13A1
:10268000F513FD1306140E1416141A1422142A142A
:102690003A14461469147A148C149C14AF14C2149E
:1026A000C714D914EA14FA140B15431558156415F8
:1026B0006C15771581159515A815B915C715D81579
:1026C000E51510161616261638164A1659166A16E5
:1026D000731680169216A116AE16BC16C216D41624
:1026E000DD16EF160017111721172A173217431797
:1026F0005517671779178B179D17AF17C117CE1787
:10270000DA17DF17F117031816181E182B183D18C3
:10271000511861186F187C188A189818AE18B918D3
:10272000CF18DE18ED18FA18031925193A194C19A3
:102730005E196A19771985199A19AD19C119C9193C
:10274000D119DD19F419021A161A281A381A441A5E
:10275000DA1ADD1AE11AEA1AF51AFC1A101B201B04
:10276000231B331B531B5A1B611B681B711B7B1BD9
:102770008D1B991B9F1BCF1BD41BEB1B021C191C11
:10278000321C0F1D261D3D1D541D611D6F1D801D1A
:102790008E1D9E1DA71DB81DC81DD41DE01DEE1D5C
:1027A000F41D141E221E331E3F1E4D1E551E671E95
:1027B000791E881E8D1EA11EA71EC71ED21EE41ED6
:1027C000F71E071F171F211F2C1F351F451FBB1F7B
:1027D000E51F0F202D2060207F209920B820BF20EA
:1027E000CD20D220DC20EB20F42005210D211F215B
:1027F00031213C214F2158216821792189219721BC
:10280000A921BA21C421D621E421F52105224E2295
:102810009322D622172354239523C8230C244C2417
:102820009924E9242C253825412550255625652550
:1028300077258625952599253626442650265A261D
:1028400066266A26457872656D65207370616E2014
:102850006F6620746865205A2076616C75657321F7
:1028600000626F74746F6D00746F700000506F6958
:102870006E742068656967687420746F6F20736D6B
:10288000616C6C3A20007269676874006C656674EC
:102890000000506F696E7420776964746820746FEB
:1028A0006F20736D616C6C3A2000002C20003A2080
:1028B0000046696E616C2063616C63756C61746560
:1028C000642062656420706F696E74200000793A3C
:1028D000000044697374616E63652066726F6D20D9
:1028E0006D696E3A000043616C63756C6174696F69
:1028F0006E206F6620746865206D616368696E651F
:1029000020736B657720616E64206F6666736574F3
:10291000206661696C65642E00002C20003A20005E
:1029200046696E616C206D656173757265642062C5
:10293000656420706F696E74200000206661696CA8
:1029400065642E204C6F776572696E67207A2074FB
:102950006F20002C20697465726174696F6E2000AD
:10296000496D70726F76696E672062656420706F62
:10297000696E742000002C207A002C206974657226
:102980006174696F6E2000496D70726F76696E6751
:102990002062656420706F696E742000006C6F7730
:1029A0006572207468616E20596D696E2E20592001
:1029B000636F6F7264696E61746520636C616D70C2
:1029C000696E672077617320757365642E004361BB
:1029D0006C6962726174696F6E20706F696E7420C9
:1029E00000417420595F4D494E5F504F5300417470
:1029F00020593000496D70726F76696E672062658C
:102A000064206F666673657420616E6420736B6505
:102A10007700002C20002C200020004D656173758C
:102A20007265642000002C200041646A757374652F
:102A30006420706F736974696F6E3A2000002C20F7
:102A4000683A002C20646D61783A005061727469B4
:102A5000616C20706F696E7420657374696D617448
:102A600065642072616469757320746F6F20736D83
:102A7000616C6C3A2000005061727469616C207066
:102A80006F696E74206469616D6574657220746F1E
:102A90006F20736D616C6C3A2000746F7000726906
:102AA000676874006C656674007269676874006CAE
:102AB00065667400746F70006661696C6564202DD2
:102AC000206E6F7420666F756E640A0072696768A5
:102AD00074006C65667400002C2000496E6974698E
:102AE000616C20706F736974696F6E3A200066695B
:102AF0006E642062656420696E64756374696F6ECC
:102B00002073656E736F7220706F696E74207A0027
:102B10005920736561726368696E672072616469C8
:102B2000757320686967686572207468616E2058E3
:102B30005F4D41582E20436C616D70696E67207740
:102B4000617320646F6E652E005920736561726336
:102B500068696E6720726164697573206C6F776550
:102B600072207468616E20595F4D494E2E20436C6F
:102B7000616D70696E672077617320646F6E652E7A
:102B8000005820736561726368696E6720726164C2
:102B900069757320686967686572207468616E2062
:102BA000585F4D41582E20436C616D70696E6720EF
:102BB00077617320646F6E652E00582073656172B3
:102BC0006368696E6720726164697573206C6F77E2
:102BD0006572207468616E20585F4D494E2E204307
:102BE0006C616D70696E672077617320646F6E65CC
:102BF0002E00536176696E67206265642063616CA4
:102C00006962726174696F6E20766563746F727346
:102C100020746F20454550524F4D005065727065CD
:102C20006E646963756C6172697479005A65726F5C
:102C300020706F696E7420636F7272656374696F60
:102C40006E3A005920766563746F72206C656E670A
:102C500074683A005820766563746F72206C656EF4
:102C60006774683A00203C20005741524E494E4755
:102C70003A2046726F6E7420706F696E74206E6FAA
:102C80007420726561636861626C652E20592063EF
:102C90006F6F7264696E6174653A000070745B31C5
:102CA0005D3A0070745B305D3A00004D656173758C
:102CB0007265643A000063757272656E745F706F5E
:102CC000736974696F6E5B5A5F415849535D3A008E
:102CD0000063757272656E745F706F736974696F8B
:102CE0006E5B595F415849535D3A000063757272DB
:102CF000656E745F706F736974696F6E5B585F4166
:102D00005849535D3A00417420592D3400417420D4
:102D100059300000636E74725B315D3A0000636E7F
:102D200074725B305D3A00007665635F795B315D9C
:102D30003A00007665635F795B305D3A0000766546
:102D4000635F785B315D3A00007665635F785B3086
:102D50005D3A00566563746F72733A20004974657A
:102D6000726174696F6E3A2000496E76616C6964B5
:102D70002062656420636F7272656374696F6E2090
:102D80006D61747269782E20526573657474696E12
:102D90006720746F206964656E746974792E0049C8
:102DA0006E76616C69642062656420636F7272651F
:102DB0006374696F6E206D61747269782E20582F6C
:102DC00059206178657320617265206661722066A2
:102DD000726F6D206265696E672070657270656ED6
:102DE000646963756C61722E00496E76616C69640A
:102DF0002062656420636F7272656374696F6E2010
:102E00006D61747269782E205368696674206F75DD
:102E100074206F662072616E67652E005A65726F4E
:102E200020706F696E7420636F7272656374696F6E
:102E30006E3A00496E76616C696420626564206355
:102E40006F7272656374696F6E206D6174726978F8
:102E50002E204C656E677468206F6620746865204C
:102E60005920766563746F72206F7574206F6620C9
:102E700072616E67652E005920766563746F7220EB
:102E80006C656E6774683A00496E76616C6964209F
:102E900062656420636F7272656374696F6E206D22
:102EA00061747269782E204C656E677468206F6655
:102EB00020746865205820766563746F72206F7582
:102EC00074206F662072616E67652E0058207665EB
:102ED00063746F72206C656E6774683A00556E6437
:102EE0006566696E65642062656420636F727265F1
:102EF0006374696F6E206D61747269782E000000D2
:102F000043616C63756C617465206F66667365748C
:102F100020616E6420736B65772072657475726EC4
:102F2000696E6720726573756C743A000000292C15
:102F3000206572726F723A20002C2000293B2074A9
:102F400061726765743A2028002C2000293B206DAF
:102F5000656173757265642D636F72726563746504
:102F6000643A2028002C20006D65617375726564D9
:102F70003A202800706F696E7420230044696666E9
:102F80006572656E636520616674657220636F7239
:102F900072656374696F6E3A2000002C20006365CF
:102FA0006E7465722C2061646A75737465643A206E
:102FB00000002C20005920766563746F722C20610C
:102FC000646A75737465643A2000002C20005820F0
:102FD000766563746F722C2061646A7573746564BE
:102FE0003A200000636E74725B315D3A0000636EDC
:102FF00074725B305D3A0046696E616C20636E747A
:10300000722076616C7565733A0000000077793A3A
:103010000000636E74725B315D3A0000576569674A
:1030200068745F793A000077783A0000636E7472D2
:103030005B305D3A00005765696768745F783A00F5
:103040000056657279206C6974746C6520736B65C9
:10305000772064657465637465642E204F727468AC
:103060006F676F6E616C697A696E6720746865203E
:10307000617865732E00004D61782E206572726F45
:1030800072206575636C696469616E3A004D6178A0
:103090002E206572726F7220593A004D61782E2091
:1030A0006572726F7220583A004D61782E206572F9
:1030B000726F72733A0000002C206572726F72207A
:1030C000593A20002C206572726F7220583A200005
:1030D0006572726F723A200029002C2000293B2073
:1030E0007461726765743A2028002C2000293B2007
:1030F000636F727265637465643A2028002C200047
:103100006D656173757265643A202800002C206536
:1031100072726F72203E206D61782E206572726F20
:1031200072206575636C696469616E00506F696EC9
:1031300074206E6F74206F6E2066697273742072D3
:103140006F77002C206572726F722059203E206DBF
:1031500061782E206572726F722059002C20657282
:10316000726F722058203E206D61782E2065727239
:103170006F722058002C2077656967746820593A6F
:103180002000506F696E74206F6E206669727374D0
:1031900020726F77003A00706F696E7420230045CB
:1031A00072726F7220616674657220636F727265ED
:1031B0006374696F6E3A2000002C200063656E74A2
:1031C0006572206E65772C20696E76657274656411
:1031D0003A2000002C20005920766563746F72201D
:1031E0006E65772C20696E7665727465643A20008E
:1031F000002C20005820766563746F72206E65770E
:103200002C20696E7665727465643A2000002C206B
:1032100000636F7272656374696F6E20616E676CB4
:1032200065733A2000002C2000636F72726563742E
:10323000656420616E676C65733A2000002C200085
:10324000636F7272656374656420782F793A200029
:10325000002C20002C20002C20003B20636F727279
:10326000656374696F6E20766563746F723A2000CF
:10327000697465726174696F6E3A200000292C20B0
:103280006572726F723A20002C2000293B20746115
:10329000726765743A2028002C2000206D656173E8
:1032A000757265643A202800706F696E742023007F
:1032B000002C200063656E7465722C20696E697441
:1032C00069616C3A2000002C2000592076656374F7
:1032D0006F722C20696E697469616C3A2000002C51
:1032E00020005820766563746F722C20696E6974B3
:1032F00069616C3A200063616C63756C6174652070
:103300006D616368696E6520736B657720616E64BB
:10331000206F6666736574204C53000000E4420021
:10332000000000000057430000C0420000E44200DB
:10333000004043000040410000C042000040410006
:103340000000000000E442000000000000574300BD
:10335000000000000057430000C0420000E44200AB
:1033600000C042000040410000C042000040410057
:103370000040430000E44200004043000057430087
:103380000040435A00205A3A00590020593A005848
:103390000020583A0024F4D43050C38E20C2A240FA
:1033A00017828B7011127A910D816CD90AA861E194
:1033B00008C7586607615143061E4B5D05C145A706
:1033C000041A411104093D9803713931034036DB79
:1033D0000265339102D4305402802E1D02632CEE1C
:1033E00001752AC501B028A001102781018F25642D
:1033F000012B244B01E0223401AC211F018D200D53
:1034000001801FFC00841EED00971DDF00B81CD258
:1034100000E61BC600201BBC00641AB200B219A84B
:10342000000A19A0006A189900D117910040178B63
:1034300000B516840031167E00B31579003A157375
:1034400000C7146F0058146A00EE136600881363F7
:103450000025135E00C7125B006C12570015125452
:1034600000C111510070114F0021114B00D61049BD
:10347000008D1047004610440002104200C00F406B
:1034800000800F3E00420F3C00060F3B00CB0E3881
:1034900000930E37005C0E3500270E3400F30D321A
:1034A00000C10D3100900D3000600D2E00320D2D49
:1034B00000050D2C00D90C2B00AE0C2900850C2921
:1034C000005C0C2700350C27000E0C2600E80B24AE
:1034D00000C40B2400A00B23007D0B23005A0B21FA
:1034E00000390B2100180B2000F80A1F00D90A1E12
:1034F00000BB0A1E009D0A1D00800A1D00630A1CF5
:1035000000470A1B002C0A1B00110A1A00F7091AAF
:1035100000DD091900C4091900AB09190092091747
:10352000007B091800630917004C091600360916BC
:1035300000200916000A091500F5081500E0081416
:1035400000CC081400B8081400A408140090081354
:10355000007D0812006B081300580812004608127C
:10356000003408110023081100120811000108118D
:1035700000F0071000E0071000D0071000C007108F
:1035800000B0070F00A107100091070E0083070F7E
:103590000074070F0065070E0057070E0049070E5D
:1035A000003B070D002E070E0020070D0013070D2E
:1035B0000006070D00F9060C00ED060D00E0060CF4
:1035C00000D4060C00C8060C00BC060C00B0060CAB
:1035D00000A4060B0099060C008D060B0082060B5A
:1035E0000077060B006C060B0061060A0057060BFD
:1035F000004C060A0042060A0038060A002E060A97
:103600000024060A001A060A001006090007060A26
:1036100000FD050900F4050900EB050900E20509B4
:1036200000D9050900D0050900C7050900BE050934
:1036300000B5050800AD050800A50509009C0508B2
:1036400000940508008C050800840508007C050826
:1036500000740508006C050700650508005D050796
:1036600000560508004E05070047050700400508FD
:103670000038050700310507002A05070023050764
:10368000001C050600160507000F050700080506C3
:103690000002050700FB040600F5040700EE04061F
:1036A00000E8040600E2040700DB040600D5040677
:1036B00000CF040600C9040600C3040600BD0406CA
:1036C00000B7040600B1040500AC040600A6040619
:1036D00000A00405009B0406009504050090040664
:1036E000008A04050085040500800406007A0405AC
:1036F0000075040500700405006B040500660405F0
:1037000000610405005C040500570405005204052F
:10371000004D04050048040500430405003E040470
:10372000003A04050035040500300404002C0405AB
:103730000027040400230405001E0404001A0404E6
:103740000016040500110404000D0404000904051A
:10375000000404040000040400FC030400F8030453
:1037600000F4030400F0030400EC030400E8030485
:1037700000E4030400E0030400DC030400D80304B5
:1037800000D4030400D0030400CC030400C80303E6
:1037900000C503030024F404D9201BC40C5C0E985C
:1037A00004C4095F0265077101F405F900FB04B365
:1037B0000048048700C1036900580355000303450E
:1037C00000BE023A008402310053022A0029022579
:1037D0000004022000E4011C00C8011900AF011719
:1037E00000980114008401130071011000610110A0
:1037F0000051010E0043010D0036010B002B010B9F
:103800000020010B00150109000C0109000301084B
:1038100000FB000800F3000800EB000700E40006CE
:1038200000DE000600D8000600D2000600CC00052D
:1038300000C7000500C2000500BD000400B9000477
:1038400000B5000400B1000400AD000400A90004AC
:1038500000A5000300A20003009F0004009B0003DA
:1038600000980003009500020093000300900003FD
:10387000008D0002008B0003008800020086000219
:103880000084000300810002007F0002007D00022E
:10389000007B000200790002007700010076000240
:1038A000007400020072000100710002006F00024B
:1038B000006D0001006C0002006A00010069000256
:1038C000006700010066000100650001006400025D
:1038D000006200010061000100600001005F000261
:1038E000005D0001005C0001005B0001005A000166
:1038F0000059000100580001005700010056000166
:103900000055000100540001005300000053000165
:10391000005200010051000100500001004F000161
:10392000004E0000004E0001004D0001004C00015F
:10393000004B0000004B0001004A0001004900015B
:103940000048000000480001004700010046000058
:103950000046000100450000004500010044000150
:10396000004300000043000100420000004200014B
:10397000004100000041000100400001003F000044
:10398000003F0001003E0000003E0001003D00003D
:10399000003D0001003C0000003C0000003C000134
:1039A000003B0000003B0001003A0000003A00012B
:1039B0000039000000390001003800000038000024
:1039C0000038000100370000003700010036000019
:1039D0000036000000360001003500000035000010
:1039E0000035000100340000003400000034000104
:1039F00000330000003300000033000100320000FB
:103A000000320000003200010031000000310000EF
:103A100000310001003000000030000000300001E3
:103A2000002F0000002F0000002F0000002F0001D9
:103A3000002E0000002E0000002E0001002D0000CE
:103A4000002D0000002D0000002D0001002C0000C2
:103A5000002C0000002C0000002C0001002B0000B6
:103A6000002B0000002B0000002B0001002A0000AA
:103A7000002A0000002A0000002A0001002900009E
:103A80000029000000290000002900000029000191
:103A90000028000000280000002800000028000086
:103AA0000028000100270000002700000027000078
:103AB000002700000027000100260000002600006B
:103AC000002600000026000000260001002500005E
:103AD0000025000000250000002500000025000052
:103AE0000025000100240000002400000024000044
:103AF0000024000000240001002300000023000037
:103B00000023000000230000002300000023000029
:103B1000002300010022000000220000002200001B
:103B2000002200000022000000220001002100000D
:103B30000021000000210000002100000021000001
:103B400000210000002100010020000000200000F2
:103B500000200000002000000020000000200000E5
:103B60000020000000200001001F0000001F0000D6
:103B7000001F0000001F0000001F0000001F0000C9
:103B8000001F0001001E0000001E0000001E0000BB
:103B9000001E0000004572723A204D494E54454DBA
:103BA00050204245440054656D70657261747572B1
:103BB0006520686561746564206265642073776957
:103BC0007463686564206F66662E204D494E5445C7
:103BD0004D502074726967676572656420210045E5
:103BE00072723A204D415854454D50204245440090
:103BF00054656D7065726174757265206865617475
:103C00006564206265642073776974636865642005
:103C10006F66662E204D415854454D502074726990
:103C20006767657265642021004572723A204D49CC
:103C30004E54454D50003A20457874727564657253
:103C4000207377697463686564206F66662E204D03
:103C5000494E54454D5020747269676765726564BA
:103C60002021004572723A204D415854454D500074
:103C70003A2045787472756465722073776974634D
:103C8000686564206F66662E204D415854454D503E
:103C90002074726967676572656420210020484F4F
:103CA00054454E4420544845524D414C2052554EA7
:103CB0004157415900204845415442454420544809
:103CC00045524D414C2052554E41574159005448A0
:103CD00045524D414C2052554E41574159004245A5
:103CE0004420544845524D414C2052554E41574175
:103CF000590020544845524D414C2052554E415791
:103D000041592028205052454845415420484F549D
:103D1000454E44290020544845524D414C205255AF
:103D20004E41574159202820505245484541542082
:103D30004845415442454429005052454845415464
:103D4000204552524F52004245442050524548456A
:103D50004154204552524F52004572723A205052FF
:103D6000494E542046414E204552524F5200455232
:103D7000524F523A205072696E742066616E207301
:103D800070656564206973206C6F77657220746854
:103D9000656E206578706563746564004572723A7B
:103DA00020455854522E2046414E204552524F52E3
:103DB000004552524F523A204578747275646572CC
:103DC0002066616E207370656564206973206C6F76
:103DD000776572207468656E2065787065637465B8
:103DE0006400202D20496E76616C696420657874CA
:103DF0007275646572206E756D6265722021005067
:103E00004944204175746F74756E652066696E69EA
:103E100073686564212050757420746865206C6136
:103E20007374204B702C204B6920616E64204B64AE
:103E300020636F6E7374616E74732066726F6D2091
:103E400061626F766520696E746F20436F6E66697C
:103E50006775726174696F6E2E6800504944204125
:103E600075746F74756E65206661696C6564212078
:103E700074696D656F75740020403A006F6B205453
:103E80003A006F6B20423A00504944204175746FEC
:103E900074756E65206661696C6564212054656D7A
:103EA000706572617475726520746F6F20686967E0
:103EB0006800204B643A2000204B693A2000204BD8
:103EC000703A200020436C61737369632050494449
:103ED00020002054753A2000204B753A2000206DB8
:103EE00061783A2000206D696E3A200020643A2003
:103EF0000020626961733A200010137D002015785C
:103F00000060177300C0196E00401C6900E01E6459
:103F10000080215F0040245A00F02655009029506F
:103F200000202C4B00802E4600C0304100D0323C97
:103F300000B034370050363200C0372D0000392829
:103F400000103A2300F03A1E00B03B1900503C1418
:103F500000D03C0F00303D0A00803D0500C03D0010
:103F600000F03DFBFF103EF6FF303EF1FF403EEC1F
:103F7000FF503EE7FF603EE2FF703EDDFF703ED83F
:103F8000FF1000C90210012C01400122017001182C
:103F900001B0010E01F00104015002FA00B002F07C
:103FA000003003E600D003DC009004D2007005C8A6
:103FB00000A006BE000008B400B009AA00D00BA003
:103FC00000600E960060118C0000158200201978A8
:103FD00000C01D6E00A0226400B0275A00902C5033
:103FE0000000314600E0343C0010383200903A289E
:103FF00000603C1E00A03D1400803E0A00203F00EF
:104000000070012C0190012701B0012201C0011DA7
:1040100001F00118011002130130020E01600209C3
:104020000190020401C002FF000003FA004003F502
:10403000008003F000D003EB002004E6007004E1F0
:1040400000E004DC004005D700C005D2004006CDEA
:1040500000D006C8008007C3003008BE00F008B9D1
:1040600000C009B400B00AAF00B00BAA00D00CA584
:1040700000000EA000500F9B00C01096005012913F
:104080000000148C00C0158700B0178200B0197DA5
:1040900000D01B7800001E730040206E0090226943
:1040A00000F024640040275F0090295A00E02B555F
:1040B00000102E500020304B0010324600E03341FB
:1040C0000090353C001037370070383200A0392D91
:1040D00000B03A2800A03B2300603C1E00103D19B0
:1040E00000903D1400103E0F00703E0A00C03E05D7
:1040F00000003F0000544D43204452495645522091
:104100004F56455254454D502000436F6E74696EB2
:104110007565207769746820616E6F7468657220B8
:10412000626F7764656E3F00473736004D34352047
:104130005A004D3435004738300020003E003E0024
:1041400020003E003E000053657665726520736B6B
:1041500065773A0000536C6967687420736B657704
:104160003A002D2D2D2D2D2D2D2D2D2D2D2D2D2D9F
:104170002D2D2D2D2D2D004E2F41004D6561737578
:1041800072656420736B65773A20004E2F41006D95
:104190006D000052696768743A0043656E74657219
:1041A0003A004C6566743A00592064697374616E14
:1041B00063652066726F6D206D696E3A004D373011
:1041C00031004D373032004D353030004731205A04
:1041D0003135204631353030004739310047312004
:1041E000583530205931393020453020463730306D
:1041F0003000473930004D373032004D37303220F3
:1042000043004D3730322055004D373032004731B2
:10421000205A31352046313530300047393100479A
:10422000312058353020593139302045302046373B
:10423000303030004D383300473930004D383400CD
:104240004D3130342053300047393000473120455C
:1042500031004D3832004D3833004D313036205367
:104260002564004D32323020532564003A2000206E
:10427000202020202020202020202020202020203E
:10428000202000203A200020202020202020202054
:10429000202020202020202020202000202020203E
:1042A0002020202020202020200025730020200016
:1042B0002D2D3A2D2D002000200020004C00202024
:1042C000002046002D2D2D003E5553420053440042
:1042D0002D2D00252020202020002020002020003F
:1042E0000120002020202D2D2D200020205A0020EC
:1042F00020000120004D36303000464C4558202D1E
:1043000020203233302F35300050502020202D20F7
:10431000203235342F3130300048495053202D2081
:10432000203232302F3130300050455420202D20A3
:10433000203234302F393000504C4120202D2020A5
:104340003231352F35350041425320202D20203287
:1043500035352F313030004D3234004D3233202589
:104360007300052E2E00580059005A0045787472CB
:1043700075646572004739390044697361626C6520
:10438000206661726D206D6F64653F0044697361E2
:10439000626C65206661726D206D6F6465004661B8
:1043A000726D206E756D626572004D38340050720A
:1043B000696E742066616E3A004578747275646542
:1043C000722066616E3A0041786973206C656E6791
:1043D000746820646966666572656E63653A004D4F
:1043E000656173757265642061786973206C656EB0
:1043F0006774683A004D3834004732382057005A05
:1044000030005A31005930005931005830005831CD
:1044100000456E642073746F707320646961670077
:104420004D3434004732382057004175746F207284
:1044300065636F76657220637261736800436865B7
:10444000636B2066616E73205B4449535D00436873
:1044500065636B2066616E73205B454E5D0054653D
:104460006D7065726174757265730058595A206376
:10447000616C2E2064657461696C73002D2D2D2D87
:104480002D2D2D2D2D2D2D2D00466C61736841692C
:104490007220495020416464723A002D2D2D2D2D3B
:1044A0002D2D2D2D2D2D2D004F63742032342032D3
:1044B00030313700446174653A20002D2D2D2D2DAB
:1044C0002D2D2D2D2D2D2D00453344763666756C02
:1044D0006C0045494E595F30346100315F37356DAE
:1044E0006D5F4D4B33002D2D2D2D2D2D2D2D2D2D73
:1044F0002D2D0020332E302E31322D5243322062AA
:10450000313033004669726D776172653A00256417
:104510002E25642E25642E2564004661696C207367
:1045200074617473004661726D206E756D626572A0
:1045300000007263006265746100616C7068610004
:104540006465760050525553413344465700332E2C
:10455000302E31322D5243320000000A0B02090C7A
:104560000D0E080703040100000000000000000019
:10457000000000000000000000000000000000003B
:1045800000000000001211100000000000000000F8
:10459000000000000000000000000000000000001B
:1045A000000000000000000000000000000000010A
:1045B0000210202008081020401020408002010234
:1045C00001080402010102040810204080804020FC
:1045D0001008040201800402018040201008040237
:1045E00001080402010102040810204080010204B5
:1045F00008102040801008040880102040044080EB
:104600001020400480050505050705080808080274
:104610000202020A0A08080404040401010101015B
:104620000101010303030303030303040707070C4A
:104630000C0C0C0C0C0C0C02020202060606060600
:104640000606060B0B0B0B0B0B0B0B07070A0A0AD4
:104650000A0A0A05050504040408080000200023CE
:1046600000260029002C002F00320000010000036A
:10467000010601090100002200250028002B002E60
:10468000003100340002010000050108010B0100A7
:10469000002100240027002A002D003000330001F3
:1046A000010000040107010A01024E414E494E4932
:1046B0005459494E46CDCCCC3D0AD7233C17B7D1EF
:1046C0003877CC2B329595E6241FB14F0A00002095
:1046D000410000C84200401C4620BCBE4CCA1B0E14
:1046E0005AAEC59D7400407A10F35A00A0724E185D
:1046F000090010A5D4E80000E87648170000E40B94
:1047000054020000CA9A3B000000E1F50500008059
:10471000969800000040420F000000A086010000B3
:1047200000102700000000E8030000000064000003
:104730000000000A00000000000100000000002C42
:1047400076D888DC674F0823DFC1DFAE59E1B1B707
:1047500096E5E3E453C63AE651997696E8E6C284D4
:1047600026EB898C9B62ED407C6FFCEFBC9C9F40EC
:10477000F2BAA56FA5F490055A2AF75C936B6CF911
:10478000676DC11BFCE0E40D47FEF520E6B500D0E7
:10479000ED902E0300943577050080841E080000FC
:1047A000204E0A000000C80C333333330F986E12CA
:1047B000831141EF8D2114893BE65516CFFEE6DBD0
:1047C00018D1844B381BF77C1D901DA4BBE424201A
:1047D0003284725E228100C9F124ECA1E53D2700FC
:1047E000A89431BBCF01C301E901CF9411241FBEAE
:1047F000CFEFD1E2DEBFCDBF00E00CBF1AE0A0E0FA
:10480000B2E0E0E7FFE703E00BBF02C007900D92C4
:10481000AE33B107D9F72CE1AEE3BAE001C01D9287
:10482000AF37B207E1F717E4CAEED7E400E006C0FD
:1048300022970109FE010BBF0F9428B6C03ED10795
:1048400080E00807A9F70F94DDAF0D94A6BF0C9484
:104850000000CF92DF92EF92FF920F931F93CF93BE
:10486000DF938C01D42EC62FD72FD60EDC1671F114
:10487000F801E080F180C990C7010F946ABCC816A6
:10488000F1F06C2DC7010F949ABCC7010F946ABC5C
:104890008C15A9F0EEE5F7E08491882341F0909122
:1048A000C00095FFFCCF8093C6003196F5CF809174
:1048B000C00085FFFCCF8AE08093C60007C0F801E6
:1048C00080819181019691838083D0CFDF91CF91B8
:1048D0001F910F91FF90EF90DF90CF900895EF928E
:1048E000FF920F931F93CF93DF931F92CDB7DEB745
:1048F0008C017B01460FF8018081918149830F94DF
:104900006ABCF70181937F01F80180819181019652
:104910009183808349814E11EECF0F90DF91CF912B
:104920001F910F91FF90EF900895FF920F931F93A7
:10493000CF93DF93CDB7DEB72C970FB6F894DEBFD9
:104940000FBECDBF8C01F62E80E390E3A0E3B0E074
:104950008D839E83AF83B8871C870B8744E0BE019D
:104960006B5F7F4FCE010B9674DF40E169ED79E11B
:10497000CE010B966EDF40E169EE79E1CE010B9638
:1049800068DF40E169EC79E1CE010B9662DF44E03B
:1049900061EC79E1CE010B965CDF44E06DEB79E1EF
:1049A000CE010B9656DF44E065EC79E1CE010B9623
:1049B00050DF44E069EA79E1CE010B964ADF44E03A
:1049C00069EF79E1CE010B9644DF44E06DEA79E1CD
:1049D000CE010B963EDF44E061EB79E1CE010B9610
:1049E00038DF44E065EB79E1CE010B9632DF44E03D
:1049F00069EB79E1CE010B962CDF4CE069E77BE0B7
:104A0000CE010B9626DF44E062E77BE0CE010B96F9
:104A100020DF44E06EE972E0CE010B961ADF44E03D
:104A20006AE972E0CE010B9614DF44E066E972E0B9
:104A3000CE010B960EDF44E06EE872E0CE010B96DD
:104A400008DF44E06AE872E0CE010B9602DF44E042
:104A500066E872E0CE010B96FCDE80E290E09A8779
:104A6000898742E0BE01675F7F4FCE010B96F1DE82
:104A700041E06EE67BE0CE010B96EBDE44E06DE1BB
:104A800072E0CE010B96E5DE44E065E172E0CE0116
:104A90000B96DFDE44E069E67BE0CE010B96D9DEC3
:104AA00044E065E67BE0CE010B96D3DE44E061E1B5
:104AB00072E0CE010B96CDDE41E065E97BE0CE01F0
:104AC0000B96C7DE44E06DE372E0CE010B96C1DECB
:104AD00089E08F1560F444E068EF73E1CE010B9636
:104AE000B8DE44E064EF73E1CE010B96B2DE46E53A
:104AF00051E360E070E049835A836B837C831C87B9
:104B00000B8744E0BE016F5F7F4FCE010B96A1DEA5
:104B1000EDE3F0E18491882341F09091C00095FF8E
:104B2000FCCF8093C6003196F5CFEEE4F7E0849198
:104B3000882341F09091C00095FFFCCF8093C60080
:104B40003196F5CF8091C00085FFFCCF8AE080933D
:104B5000C6002C960FB6F894DEBF0FBECDBFDF9116
:104B6000CF911F910F91FF9008951F93CF93DF93E3
:104B7000182FCDE3D0E1FE018491882341F090917C
:104B8000C00095FFFCCF8093C6003196F5CFEEE3D1
:104B9000F7E08491882341F09091C00095FFFCCF0D
:104BA0008093C6003196F5CF8091C00085FFFCCF81
:104BB0008AE08093C600FE018491EDE3F0E1882352
:104BC00049F09091C00095FFFCCF8093C6003196CC
:104BD0008491F5CF4091D9195091DA196091DB1980
:104BE0007091DC1986E397E00E94DE3B4091DD196D
:104BF0005091DE196091DF197091E01983E397E01D
:104C00000E94DE3B4091E1195091E2196091E31955
:104C10007091E41980E397E00E94DE3B4091E51932
:104C20005091E6196091E7197091E8198DE297E0CB
:104C30000E94DE3B8091C00085FFFCCF8AE080931C
:104C4000C600FE018491EDE3F0E1882349F09091E4
:104C5000C00095FFFCCF8093C60031968491F5CFBC
:104C6000E3E1F7E08491882341F09091C00095FF43
:104C7000FCCF8093C6003196F5CF8091C00085FFB0
:104C8000FCCF8AE08093C600FE018491EDE3F0E161
:104C9000882349F09091C00095FFFCCF8093C60017
:104CA00031968491F5CF4091E9195091EA196091BC
:104CB000EB197091EC198AE097E00E94DE3B40917D
:104CC000ED195091EE196091EF197091F01987E08C
:104CD00097E00E94DE3B4091F1195091F2196091EA
:104CE000F3197091F41984E097E00E94DE3B409143
:104CF000F5195091F6196091F7197091F81981E042
:104D000097E00E94DE3B8091C00085FFFCCF8AE0E7
:104D10008093C600FE018491EDE3F0E1882349F021
:104D20009091C00095FFFCCF8093C600319684918E
:104D3000F5CFE3EEF6E08491882341F09091C00036
:104D400095FFFCCF8093C6003196F5CF8091C000CF
:104D500085FFFCCF8AE08093C600FE018491EDE3DD
:104D6000F0E1882349F09091C00095FFFCCF80933B
:104D7000C60031968491F5CF4091C9195091CA1956
:104D80006091CB197091CC198AED96E00E94EF3BAF
:104D90004091CD195091CE196091CF197091D019D1
:104DA00087ED96E00E94EF3B4091D1195091D219C6
:104DB0006091D3197091D41984ED96E00E94EF3B75
:104DC0004091D5195091D6196091D7197091D81981
:104DD00081ED96E00E94EF3B8091C00085FFFCCF03
:104DE0008AE08093C600FE018491EDE3F0E1882320
:104DF00049F09091C00095FFFCCF8093C60031969A
:104E00008491F5CFECE9F6E08491882341F090910C
:104E1000C00095FFFCCF8093C6003196F5CF8091FE
:104E2000C00085FFFCCF8AE08093C600FE0184911C
:104E3000EDE3F0E1882349F09091C00095FFFCCFAD
:104E40008093C60031968491F5CF4091C11950915D
:104E5000C2196091C3197091C41983E996E00E9448
:104E6000DE3B4091BD195091BE196091BF19709100
:104E7000C01980E996E00E94DE3B8091C00085FF6A
:104E8000FCCF8AE08093C600FE018491EDE3F0E15F
:104E9000882349F09091C00095FFFCCF8093C60015
:104EA00031968491F5CFEDEDF5E08491882341F0C2
:104EB0009091C00095FFFCCF8093C6003196F5CF4E
:104EC0008091C00085FFFCCF8AE08093C600FE0180
:104ED0008491EDE3F0E1882349F09091C00095FFC3
:104EE000FCCF8093C60031968491F5CF4091C519CF
:104EF0005091C6196091C7197091C81984ED95E059
:104F00000E94DE3B4091A9195091AA196091AB19FA
:104F10007091AC1981ED95E00E94DE3B4091F9194A
:104F20005091FA196091FB197091FC198EEC95E083
:104F30000E94EF3B4091AD195091AE196091AF19AD
:104F40007091B0198BEC95E00E94DE3B4091B11955
:104F50005091B2196091B3197091B41988EC95E031
:104F60000E94DE3B4091B5195091B6196091B71976
:104F70007091B81985EC95E00E94DE3B4091B9191B
:104F80005091BA196091BB197091BC1982EC95E0EF
:104F90000E94DE3B8091C00085FFFCCF8AE08093B9
:104FA000C600FE018491EDE3F0E1882349F0909181
:104FB000C00095FFFCCF8093C60031968491F5CF59
:104FC000E0EBF5E08491882341F09091C00095FFDB
:104FD000FCCF8093C6003196F5CF8091C00085FF4D
:104FE000FCCF8AE08093C600FE018491EDE3F0E1FE
:104FF000882349F09091C00095FFFCCF8093C600B4
:1050000031968491F5CF4091790B50917A0B609154
:105010007B0B70917C0B87EA95E00E94DE3B409110
:105020007D0B50917E0B60917F0B7091800B84EA19
:1050300095E00E94DE3B4091810B5091820B609184
:10504000830B7091840B81EA95E00E94DE3B809196
:10505000C00085FFFCCF8AE08093C600FE018491EA
:10506000EDE3F0E1882349F09091C00095FFFCCF7B
:105070008093C60031968491F5CFE3E9F5E0849101
:10508000882341F09091C00095FFFCCF8093C6002B
:105090003196F5CF8091C00085FFFCCF8AE08093E8
:1050A000C600FE018491EDE3F0E1882349F0909180
:1050B000C00095FFFCCF8093C60031968491F5CF58
:1050C00040919E0250919F026091A0027091A102B6
:1050D00089E895E00E94DE3B60919A0270919B0204
:1050E00080919C0290919D020F949F40AB01BC0166
:1050F00086E895E00E94DE3B6091960270919702EF
:1051000080919802909199020F94AB40AB01BC0141
:1051100083E895E00E94DE3B8091C00085FFFCCFD4
:105120008AE08093C600FE018491EDE3F0E18823DC
:1051300049F09091C00095FFFCCF8093C600319656
:105140008491F5CFEDE6F5E08491882341F09091CC
:10515000C00095FFFCCF8093C6003196F5CF8091BB
:10516000C00085FFFCCF8AE08093C600FE018491D9
:10517000EDE3F0E1882349F09091C00095FFFCCF6A
:105180008093C60031968491F5CF40918E02509164
:105190008F02609190027091910283E695E00E94E7
:1051A000DE3B60918A0270918B0280918C0290911B
:1051B0008D020F949F40AB01BC0180E695E00E94F8
:1051C000DE3B609186027091870280918802909107
:1051D00089020F94AB40AB01BC018DE595E00E94C4
:1051E000DE3B8091C00085FFFCCF8AE08093C60043
:1051F000FE018491EDE3F0E1882349F09091C00035
:1052000095FFFCCF8093C60031968491F5CFE9E2FB
:10521000F5E08491882341F09091C00095FFFCCF88
:105220008093C6003196F5CF8091C00085FFFCCFFA
:105230008AE08093C600FE018491EDE3F0E18823CB
:1052400049F09091C00095FFFCCF8093C600319645
:105250008491F5CF40911D0250911E0260911F0272
:10526000709120028FE195E00E94DE3B20E030E06B
:1052700040E752E460911502709116028091170286
:10528000909118020F94DDB3AB01BC018CE195E065
:105290000E94DE3B4091690B50916A0B60916B0B51
:1052A00070916C0B89E195E00E94DE3B8091C0001B
:1052B00085FFFCCF8AE08093C600FE018491EDE378
:1052C000F0E1882349F09091C00095FFFCCF8093D6
:1052D000C60031968491F5CFEDEEF4E084918823F9
:1052E00041F09091C00095FFFCCF8093C6003196AD
:1052F000F5CF8091C00085FFFCCF8AE08093C60087
:10530000FE018491EDE3F0E1882349F09091C00023
:1053100095FFFCCF8093C60031968491F5CF4091E4
:10532000650B5091660B6091670B7091680B83EE73
:1053300094E00E94DE3B20E030E040E752E46091E0
:1053400011027091120280911302909114020F9435
:10535000DDB3AB01BC0180EE94E00E94DE3B8091A6
:10536000C00085FFFCCF8AE08093C600FE018491D7
:10537000EDE3F0E1882349F09091C00095FFFCCF68
:105380008093C60031968491F5CFE6E8F4E08491ED
:10539000882341F09091C00095FFFCCF8093C60018
:1053A0003196F5CF8091C00085FFFCCF8AE08093D5
:1053B000C600FE018491EDE3F0E1882349F090916D
:1053C000C00095FFFCCF8093C60031968491F5CF45
:1053D00040916E0B50E060E070E08CE794E00E943A
:1053E000EF3B8091C00085FFFCCF8AE08093C60030
:1053F000FE018491EDE3F0E1882349F09091C00033
:1054000095FFFCCF8093C60031968491F5CF8091B3
:10541000950B8823A1F1E9E6F4E08491882341F01B
:105420009091C00095FFFCCF8093C6003196F5CFD8
:105430008091C00085FFFCCF8AE08093C600FE010A
:105440008491EDE3F0E1882349F09091C00095FF4D
:10545000FCCF8093C60031968491F5CF40913D02F8
:1054600050913E0260913F02709140028FE594E0BE
:105470000E94DE3B8091C00085FFFCCF11C0E3E4B9
:10548000F4E08491882341F09091C00095FFFCCF17
:105490008093C6003196F5CF8091C00085FFFCCF88
:1054A0008AE08093C6001A3008F43EC0FE01C49121
:1054B000EDE3F0E1CC2349F08091C00085FFFCCF03
:1054C000C093C6003196C491F5CFEAE2F4E084912E
:1054D000882341F09091C00095FFFCCF8093C600D7
:1054E0003196F5CF8091C00085FFFCCF8AE0809394
:1054F000C6004091F8135091F9136091FA1370911E
:10550000FB1380E294E00E94DE3B4091F413509143
:10551000F5136091F6137091F71386E194E0DF9133
:10552000CF911F910C94DE3BDF91CF911F91089595
:10553000AF92BF92CF92DF92EF92FF920F931F93A1
:10554000CF93DF93CDB7DEB7E0970FB6F894DEBF09
:105550000FBECDBF80E1E3EDF2E0DE019196019058
:105560000D928A95E1F780E1E3EEF2E0DE015196DB
:1055700001900D928A95E1F780E1E3EFF2E0DE0120
:10558000119601900D928A95E1F76E0181E2C80EA5
:10559000D11C89EDE82E89E1F82E8E010F5E1F4F98
:1055A00069EE79E1AE014F5F5F4F99ECA92E99E169
:1055B000B92E20E030E0F60181919191A191B19155
:1055C0006F01F70181939193A193B1937F01F8014A
:1055D00081919191A191B1918F01FB01819391935F
:1055E000A193B193BF01FA0181919191A191B191E0
:1055F000AF01F50181939193A193B1935F012F5F67
:105600003F4F24303105B9F60F94241D80E090E41B
:10561000ACE9B4E48093C1199093C219A093C31963
:10562000B093C4198093BD199093BE19A093BF196C
:10563000B093C0191092C5191092C6191092C719CB
:105640001092C81980E29EE4A0E0B0E08093F919BE
:105650009093FA19A093FB19B093FC191092A91911
:105660001092AA191092AB191092AC1980E090E038
:10567000A0E7B1E48093AD199093AE19A093AF1950
:10568000B093B0198093B1199093B219A093B31944
:10569000B093B4198DEC9CECACECBEE38093B519DF
:1056A0009093B619A093B719B093B81980E090E021
:1056B000A0E2B0E48093B9199093BA19A093BB19F2
:1056C000B093BC191092810B1092820B1092830B35
:1056D0001092840B10927D0B10927E0B10927F0B18
:1056E0001092800B1092790B10927A0B10927B0B18
:1056F00010927C0B8DE39AE0A1E8B1E480939E02C6
:1057000090939F02A093A002B093A1026DEC7CEC59
:1057100084E99FE30F94994060939A0270939B02EF
:1057200080939C0290939D0265E87BEE80E692E474
:105730000F94A5406093960270939702809398020D
:10574000909399020F94CA2F80E090E0A0E8BFE305
:105750008093920290939302A0939402B093950247
:1057600010926E0B80E090E0A0E4B0E480931D0204
:1057700090931E02A0931F02B093200240E050E0DD
:1057800064E372E44093150250931602609317028B
:10579000709318021092690B10926A0B10926B0BA7
:1057A00010926C0B1092650B1092660B1092670BA7
:1057B0001092680B40E050E060E071E44093110209
:1057C0005093120260931302709314021092950B7F
:1057D00080933D0290933E02A0933F02B09340021B
:1057E0000E94394EEDE3F0E18491882341F09091DD
:1057F000C00095FFFCCF8093C6003196F5CFEAED4F
:10580000F3E08491882341F09091C00095FFFCCF94
:105810008093C6003196F5CF8091C00085FFFCCF04
:105820008AE08093C600E0960FB6F894DEBF0FBE04
:10583000CDBFDF91CF911F910F91FF90EF90DF903F
:10584000CF90BF90AF9008951F93CF93DF93CDB7C4
:10585000DEB72C970FB6F894DEBF0FBECDBF162F64
:105860009C878B8786E591E3A0E0B0E089839A83EB
:10587000AB83BC8344E0BE016B5F7F4FCE010B96D0
:105880002ED843E050E0BE016B5F7F4FCE01019602
:105890000F94D9B9892B09F0FFC040E169ED79E196
:1058A000CE010B961CD840E169EE79E1CE010B9652
:1058B00016D840E169EC79E1CE010B9610D80F942F
:1058C000241D44E061EC79E1CE010B9608D844E058
:1058D0006DEB79E1CE010B9602D844E065EC79E1FD
:1058E000CE010B960E946F2444E069EA79E1CE0173
:1058F0000B960E946F2444E069EF79E1CE010B968C
:105900000E946F2444E06DEA79E1CE010B960E947B
:105910006F2444E061EB79E1CE010B960E946F2485
:1059200044E065EB79E1CE010B960E946F2444E0E0
:1059300069EB79E1CE010B960E946F244CE069E798
:105940007BE0CE010B960E946F2444E062E77BE08F
:10595000CE010B960E946F2444E06EE972E0CE0106
:105960000B960E946F2444E06AE972E0CE010B9628
:105970000E946F2444E066E972E0CE010B960E941B
:105980006F2444E06EE872E0CE010B960E946F2413
:1059900044E06AE872E0CE010B960E946F2444E076
:1059A00066E872E0CE010B960E946F2442E0BE01D1
:1059B000675F7F4FCE010B960E946F2441E06EE639
:1059C0007BE0CE010B960E946F2444E06DE172E013
:1059D000CE010B960E946F2444E065E172E0CE0197
:1059E0000B960E946F2444E069E67BE0CE010B96A3
:1059F0000E946F2444E065E67BE0CE010B960E9496
:105A00006F2444E061E172E0CE010B960E946F24A6
:105A100041E065E97BE0CE010B960E946F2444E0F3
:105A20006DE372E0CE010B960E946F241A3070F085
:105A300044E068EF73E1CE010B960E946F2444E0CE
:105A400064EF73E1CE010B960E946F240E94394EE1
:105A50000F94CA2FEDE3F0E18491882341F09091F7
:105A6000C00095FFFCCF8093C6003196F5CFECEFD8
:105A7000F3E08491882341F09091C00095FFFCCF22
:105A80008093C6003196F5CF8091C00085FFFCCF92
:105A90008AE08093C60001C04BDD2C960FB6F894C7
:105AA000DEBF0FBECDBFDF91CF911F910895682F4C
:105AB000772767FD70958091DD109091DE108E51F3
:105AC0009F4E0F94BEB99093D4108093D31021E0D1
:105AD000892B09F420E0822F08958091D3109091B2
:105AE000D41060E070E001960D9467B68A3010F033
:105AF000895A01C0805D9091C00095FFFCCF8093D2
:105B0000C6000895CF93C82F82958F70EFDF8C2F3A
:105B10008F70CF91EBCFCF93C82F892FF3DF8C2FCE
:105B2000CF91F0CFCF93DF93FB0120E030E0DC0199
:105B3000ED018D918823A1F14115510519F024172C
:105B4000350774F58032A1F38A3051F190ED980F4A
:105B50009A3020F4682F6295607F08C09FE9980F03
:105B60009630A8F4682F6295607F6057CE01029648
:105B70007981A0EDA70FAA3018F4762F7A2B0CC0EC
:105B8000AFE9A70FA63018F47755762B05C0882704
:105B90009927821B930B05C071932F5F3F4FC7CF8F
:105BA000C901DF91CF910895E091D310F091D41005
:105BB0008181882371F06BE573E08EE39AE0F6D77C
:105BC00082E475DF882319F00C9400F008950C949A
:105BD00000000895CF93DF9366E673E08EE39AE0CA
:105BE000E5D7F894C0E0D0E060E0CE010F949ABC15
:105BF0002196C11580E1D807B9F77894DF91CF914C
:105C00000895AF92BF92CF92DF92EF92FF920F93DF
:105C10001F93CF93DF93CDB7DEB760970FB6F8949D
:105C2000DEBF0FBECDBF68E773E08EE39AE0BED75C
:105C300081E43DDF8823A9F08091D3109091D410A6
:105C4000FC012181283741F440E150E060E070E040
:105C500002960F94CFB703C040DF0F944BB17B0186
:105C600002C0E12CF12C83E422DF882331F035DF00
:105C70000F944BB1262F872F02C020E080E2FFE176
:105C8000FF22022F182F013020E2120710F000E04F
:105C900010E2C8018E0D9F1D8130904220F000E07F
:105CA00010E20E191F0988E502DF882371F1809147
:105CB000D3109091D41040E150E0BE016F5F7F4F50
:105CC000019630DF8C01009701F1FE013196CF0182
:105CD000800F911FD701E817F90719F021912D9333
:105CE000FACF4AE050E0B8018EE39AE0C4D76CE8FE
:105CF00073E08EE39AE05AD7C7010DDF8091C000B0
:105D000085FFFCCF8AE08093C60080E2B82E9AE03F
:105D1000A92E0115110529F1C701FDDE8091C000F2
:105D200085FFFCCFB092C6006701F0E1CF0ED11C19
:105D3000F7012FEFE21AF20A80819091C00095FFDF
:105D4000FCCFB092C600DEDE0150110919F0EC1450
:105D5000FD0471F78091C00085FFFCCFA092C600C2
:105D6000D8CF60960FB6F894DEBF0FBECDBFDF91DF
:105D7000CF911F910F91FF90EF90DF90CF90BF9048
:105D8000AF900895AF92BF92CF92DF92EF92FF92C1
:105D90000F931F93CF93DF93CDB7DEB760970FB606
:105DA000F894DEBF0FBECDBF6DEA73E08EE39AE0DC
:105DB000FDD681E47CDE8823A9F08091D3109091F8
:105DC000D410FC012181283741F440E150E060E02B
:105DD00070E002960F94CFB703C07FDE0F944BB1F3
:105DE0007B0102C0E12CF12C83E461DE882331F0D9
:105DF00074DE0F944BB1262F872F02C020E080E283
:105E0000FFE1FF22022F182F013020E2120710F0CD
:105E100000E010E2C8018E0D9F1D8130904220F0FD
:105E200000E010E20E191F0988E541DE8823B1F178
:105E30008091D3109091D41040E150E0BE016F5F8B
:105E40007F4F01966FDE8C01009741F1CE010196E4
:105E50005C01C12CD12CC016D10661F0F501619115
:105E60005F01C6018E0D9F1D0F949ABCFFEFCF1AE4
:105E7000DF0AF1CF4AE050E0B8018EE39AE0FBD6AA
:105E800064EC73E08EE39AE091D6C70144DE809122
:105E9000C00085FFFCCF8AE08093C60020E2B22ECE
:105EA0003AE0A32E0115110531F1C70134DE8091CE
:105EB000C00085FFFCCFB092C600670120E1C20E92
:105EC000D11CC701EFEFEE1AFE0A0F946ABC909145
:105ED000C00095FFFCCFB092C60014DE015011093E
:105EE00019F0EC14FD0469F78091C00085FFFCCF28
:105EF000A092C600D7CF60960FB6F894DEBF0FBE53
:105F0000CDBFDF91CF911F910F91FF90EF90DF9068
:105F1000CF90BF90AF900895CF92DF92EF92FF9213
:105F2000CF93DF9368EE73E08EE39AE03FD680E58F
:105F3000BEDD882309F46BC0D0DD0F944BB16B013B
:105F40007C018FEFC816D10411F008F060C086E420
:105F5000AEDD882379F0C1DD0F944BB16115710579
:105F600011F460E004C06130710521F461E08C2D12
:105F70000F94E1A986E59BDD8823B1F0AEDD0F9497
:105F80004BB16115710511F460E005C06130710518
:105F900009F03DC061E08C2DDF91CF91FF90EF9033
:105FA000DF90CF900D941AAA8C2D0F944FAAC1E0C8
:105FB000D0E0892B11F4C0E0D0E0E8EFF3E081916C
:105FC000882339F09091C00095FFFCCF8093C600E4
:105FD000F6CF4AE050E0B6018EE39AE0F4D5E4E46F
:105FE000F4E08191882339F09091C00095FFFCCFB7
:105FF0008093C600F6CF4AE050E0BE018EE39AE0FF
:10600000DF91CF91FF90EF90DF90CF90E3C5DF91CC
:10601000CF91FF90EF90DF90CF900895CF936CEFEA
:1060200073E08EE39AE0C2D5E091D310F091D410E2
:1060300085818F3311F0811170C0ECE0F4E0819123
:10604000882339F09091C00095FFFCCF8093C60063
:10605000F6CF4AE050E06091DC138EE39AE0F8D589
:10606000E3E1F4E08191882339F09091C00095FF3D
:10607000FCCF8093C600F6CF4AE050E06091DB137E
:106080008EE39AE0E5D5EBE1F4E08191882339F0E5
:106090009091C00095FFFCCF8093C600F6CF609131
:1060A000D9137091DA134AE050E08EE39AE08BD571
:1060B000EFE1F4E08191882339F09091C00095FFE1
:1060C000FCCF8093C600F6CF6091D7137091D813A0
:1060D0004AE050E08EE39AE076D5E3E2F4E0819185
:1060E000882339F09091C00095FFFCCF8093C600C3
:1060F000F6CF4AE050E06091D6138EE39AE0A8D53F
:10610000E7E2F4E08191882309F455C09091C00042
:1061100095FFFCCF8093C600F5CF813209F053C0C4
:106120000F94C408ECE1F4E08191882339F0909158
:10613000C00095FFFCCF8093C600F6CF6091D913C5
:106140007091DA134AE050E08EE39AE03CD5EFE13B
:10615000F4E08191882339F09091C00095FFFCCF45
:106160008093C600F6CF6091D7137091D8134AE0A0
:1061700050E08EE39AE027D5E3E2F4E081918823B2
:1061800039F09091C00095FFFCCF8093C600F6CF08
:106190004AE050E06091D6138EE39AE059D5E7E2E9
:1061A000F4E08191882339F09091C00095FFFCCFF5
:1061B0008093C600F6CF4AE050E06091D5138EE39D
:1061C0009AE0CF914BC582E572DC882361F185DCD2
:1061D0000F944BB1C62FEBE2F4E08191882339F0A4
:1061E0009091C00095FFFCCF8093C600F6CF4AE0A7
:1061F00050E06C2F8EE39AE02BD5E3E4F4E081913C
:10620000882339F09091C00095FFFCCF8093C600A1
:10621000F6CF6C2F8C2F0F9450094AE050E0BC0150
:106220008EE39AE0D7D488E542DC8823E1F055DCA0
:106230000F944BB17093DA136093D913E6E4F4E052
:106240008191882339F09091C00095FFFCCF809315
:10625000C600F6CF6091D9137091DA134AE050E08E
:106260008EE39AE0B0D489E522DC8823E9F035DCBE
:106270000F944BB17093D8136093D713E1E5F4E01A
:106280008191882339F09091C00095FFFCCF8093D5
:10629000C600F6CF6091D7137091D8134AE050E052
:1062A0008EE39AE0CF918FC4CF910895CF93DF937F
:1062B000EC0160E08E810F941AAA81E090E00F94C7
:1062C0005CA861E08E810F941AAA81E090E00F949F
:1062D0005CA860E08E810F941AAA84E690E0DF91BA
:1062E000CF910D945CA8CF92DF92EF92FF920F9323
:1062F0001F93CF93DF937C01C0E0D0E0C62ED12C5A
:1063000087010C0F1D1F61E0F80187810F94E1A93F
:10631000B6010C2E02C0759567950A94E2F761707C
:10632000F80187810F941AAA2196C430D10541F74C
:10633000C701DF91CF911F910F91FF90EF90DF90F8
:10634000CF90B4CFCF92DF92EF92FF920F931F9333
:10635000CF93DF937C01C0E0D0E0C62ED12C870123
:106360000C0F1D1F61E0F80187810F94E1A9B601B0
:106370000C2E02C0759567950A94E2F76170F801DA
:1063800087810F941AAA2196C830D10541F7C70119
:10639000DF91CF911F910F91FF90EF90DF90CF9001
:1063A00085CF1F93CF93DF93EC01162F642F8C8141
:1063B0000F941AAA8D818F3F19F060E00F941AAAEA
:1063C0008F85612F84FF05C0CE01DF91CF911F9192
:1063D000B9CF70E084E0759567958A95E1F7CE01B5
:1063E00082DF612FCE01DF91CF911F917CCF40E002
:1063F000D8CF61E0FCDF80E496E00D945CA862E019
:10640000F6DF80E496E00D945CA8CF93DF93CDB7E0
:10641000DEB728970FB6F894DEBF0FBECDBF28E0D9
:10642000E3E0F3E0DE01119601900D922A95E1F789
:10643000FC012389421710F04FEF420FFE01319605
:10644000E40FF11DE40FF11D2081260F2068622F5B
:1064500028960FB6F894DEBF0FBECDBFDF91CF9167
:10646000C6CFFC016089262F2460208B6C60BFCFD3
:10647000CF93DF93EC01423018F08F8588608F87CF
:106480004B8B1C8A222329F0413019F48F858460BC
:106490008F8780E593EC0F945CA860E08C810F946B
:1064A0001AAA60E08E810F941AAA8D818F3F19F08D
:1064B00060E00F941AAA6F8564FD19C063E0CE01F5
:1064C00012DF84E991E10F945CA863E0CE010BDF59
:1064D00084E991E10F945CA863E0CE0104DF86E9D2
:1064E00090E00F945CA862E0CE01FDDE13C0606214
:1064F000CE017DDF84E991E10F945CA86F85606235
:10650000CE0175DF86E990E00F945CA86F8560622C
:10651000CE016DDF6F856062CE0169DF8CE390E0B4
:106520000F945CA884E0888BCE019BDF8CE390E025
:106530000F945CA8CE015DDF88EB9BE00F945CA814
:1065400082E0898B66E0CE0152DF8CE390E0DF9140
:10655000CF910D945CA86F927F928F92AF92CF9261
:10656000EF920F931F93CF93DF93CDB7DEB73C012C
:10657000162F842F5E854F8538899989F30184838E
:1065800025830683E782C086A18682865387448757
:106590003587968761E00F94E1A9F30185818F3FEC
:1065A00019F061E00F94E1A961E0F30186810F9495
:1065B000E1A9112319F0F301178603C080E1F3016B
:1065C000878720E041E060E1C301DF91CF911F9117
:1065D0000F91EF90CF90AF908F907F906F9048CFBA
:1065E0008F92AF92CF92EF920F93DC0113961C9291
:1065F0001E921297E0E6F4E0ED93FC931F921F9237
:106600001F921F928C2CAE2CC02EE22E042F2FEF47
:10661000462F61E0A0DF0F900F900F900F900F9129
:10662000EF90CF90AF908F900895CF93DF93EC01D0
:10663000423018F08F8588608F874B8B1C8A22230D
:1066400029F0413019F48F8584608F8780E593ECC1
:106650000F945CA860E08C810F941AAA60E08E8190
:106660000F941AAA8D818F3F19F060E00F941AAA37
:106670006F8564FD19C063E0CE0135DE84E991E1E8
:106680000F945CA863E0CE012EDE84E991E10F94C3
:106690005CA863E0CE0127DE86E990E00F945CA859
:1066A00062E0CE0120DE13C06062CE01A0DE84E98C
:1066B00091E10F945CA86F856062CE0198DE86E957
:1066C00090E00F945CA86F856062CE0190DE6F85CC
:1066D0006062CE018CDE8CE390E00F945CA884E0D5
:1066E000888BCE01BEDE8CE390E00F945CA8CE01D7
:1066F00086DE80E496E00F945CA882E0898B66E0F9
:10670000CE0175DE8CE390E00F945CA840E068E079
:10671000CE017BDE66EB79E0CE010F94B5AA41E0B5
:1067200068E0CE0172DE66EB79E0CE010F94B5AA87
:1067300042E066E0CE0169DE64EB79E0CE01DF91F4
:10674000CF910D94B5AACF92DF92EF92FF920F9363
:106750001F93CF93DF931F921F92CDB7DEB78C01AB
:10676000677088E0689FB00111246064C8014983A4
:106770005A833DDE4981C42E5A81D52EE12CF12C5D
:10678000D6016D916D01D801ED91FC910190F081E0
:10679000E02DC8011995BFEFEB1AFB0AE8E0EE16F1
:1067A000F10471F70F900F90DF91CF911F910F912E
:1067B000FF90EF90DF90CF90089541E0F2DD81E00F
:1067C00090E008951F920F920FB60F9211240BB60E
:1067D0000F922F933F934F935F936F938F939F935A
:1067E000EF93FF93CF93DF931F92CDB7DEB78091E6
:1067F000C00084FF04C08091C600898319C06091E5
:10680000C6002091BF0A3091C00AC90101968F7756
:1068100099274091C10A5091C20A8417950741F007
:10682000F901E15CF54F60839093C00A8093BF0A41
:106830000F90DF91CF91FF91EF919F918F916F9189
:106840005F914F913F912F910F900BBE0F900FBE14
:106850000F901F9018951F920F920FB60F92112450
:106860000BB60F922F933F934F935F936F938F933A
:106870009F93EF93FF93CF93DF931F92CDB7DEB734
:106880008091C30A9091C40A019709F58091D000C4
:1068900084FF04C08091D600898319C06091D6001E
:1068A0002091BF0A3091C00AC90101968F779927BC
:1068B0004091C10A5091C20A8417950741F0F9012D
:1068C000E15CF54F60839093C00A8093BF0A0F90FC
:1068D000DF91CF91FF91EF919F918F916F915F9198
:1068E0004F913F912F910F900BBE0F900FBE0F90C5
:1068F0001F901895CF92DF92EF92FF926A017B0171
:10690000411581EE58076105710509F463C082E005
:106910008093C00060E079E08DE390E0A7019601EC
:106920000F94F0B52150310941095109CA01B9014B
:1069300022E030E040E050E00F94F0B591E0309379
:10694000C5002093C4008091C10080618093C10084
:106950008091C10088608093C1008091C1008068EF
:106960008093C100992341F082E08093D00060E0E1
:1069700079E08DE390E006C01092D00060E874E802
:106980008EE190E0A70196010F94F0B521503109F6
:1069900041095109CA01B90122E030E040E050E06C
:1069A0000F94F0B53093D5002093D4008091D1009E
:1069B00080618093D1008091D10088608093D10064
:1069C0008091D10080688093D100FF90EF90DF909C
:1069D000CF9008951092C00090E020E130E0AFCF5A
:1069E0002091C10A3091C20A8091BF0A9091C00AD9
:1069F0008217930771F0F901E15CF54F80812F5FF9
:106A00003F4F2F7733273093C20A2093C10A90E07B
:106A100008958FEF9FEF08958091C10A9091C20A67
:106A20009093C00A8093BF0A08954F925F926F922D
:106A30007F928F929F92AF92BF92CF92DF92EF920E
:106A4000FF920F931F93CF93DF93CDB7DEB7A0973D
:106A50000FB6F894DEBF0FBECDBF5C0141155105E6
:106A600061057105E9F420E030E040E350E060E0CA
:106A700070E0A0960FB6F894DEBF0FBECDBFDF91D9
:106A8000CF911F910F91FF90EF90DF90CF90BF902B
:106A9000AF909F908F907F906F905F904F905BC072
:106AA0008E010F5F1F4FC12CD12C76014801422E61
:106AB000512C612C712C8FEFC81AD80AE80AF80AF9
:106AC000CB01BA01A30192010F94CEB5CA01F8011E
:106AD00061938F01A901BC01411551056105710543
:106AE00051F7F1E0CF1AD108E108F108F401EC0DFB
:106AF000FD1D80818A3010F440E301C047E3480F58
:106B0000552747FD5095652F752F20E030E0C501D2
:106B100022D081E0C81AD108E108F108EFEFCE16C3
:106B2000DE06EE06FE0611F7A0960FB6F894DEBF5D
:106B30000FBECDBFDF91CF911F910F91FF90EF90CE
:106B4000DF90CF90BF90AF909F908F907F906F908D
:106B50005F904F9008952115310539F48091C00060
:106B600085FFFCCF4093C60008952A30310509F413
:106B70003FC05BCF9A01462F552747FD5095652FA3
:106B8000752FE9CFCF93DF93EC0120E030E04DE0AB
:106B900050E060E070E0DFDF20E030E04AE050E00D
:106BA00060E070E0CE01DF91CF91D5CFFB01219164
:106BB000BF01222339F03091C00035FFFCCF209374
:106BC000C600F4CFDFCF9A01AB01662757FD609571
:106BD000762FC1CFCF93DF93EC019A01AB016627EB
:106BE00057FD6095762FB7DFCE01DF91CF91CACFE9
:106BF000CF92DF92EF92FF92CF93DF93EC016A0185
:106C00007B0177FF0FC020E030E04DE250E060E014
:106C100070E0A1DFF094E094D094C094C11CD11C2A
:106C2000E11CF11C2AE0B701A601CE01DF91CF9152
:106C3000FF90EF90DF90CF90F8CE2115310539F419
:106C40008091C00085FFFCCF4093C6000895EDCE33
:106C50009A01462F50E060E070E0EFCFCF93DF93D2
:106C6000EC019A01462F50E060E070E0E6DFCE01D3
:106C7000DF91CF9187CF9A01AB0160E070E0DDCF6B
:106C8000CF93DF93EC019A01AB0160E070E0D5DFB8
:106C9000CE01DF91CF9176CFCF93DF93EC01CDDFA3
:106CA000CE01DF91CF916ECF8F929F92AF92BF9224
:106CB000CF92DF92EF92FF921F93CF93DF93EC017D
:106CC0006A017B01122F20E030E0A901C701B60163
:106CD0000F94DCB087FF0CC020E030E04DE250E0C4
:106CE00060E070E0CE0137DFF7FAF094F7F8F09447
:106CF000B12C60E070E080E09FE3B11641F020E04D
:106D000030E040E251E40F94E3B0B394F6CF9B013E
:106D1000AC01C701B6010F94ECAF6B017C010F947D
:106D200050B14B015C010F947CB19B01AC01C701D8
:106D3000B6010F94EBAF6B017C012AE0B501A40111
:106D4000CE0173DE112361F0E7ECF6E08191882338
:106D500039F09091C00095FFFCCF8093C600F6CF2C
:106D6000112319F120E030E040E251E4C701B601FF
:106D70000F94DDB36B017C010F944BB14B01AA243E
:106D800097FCA094BA2CB501A401CE0131DFC50156
:106D9000B4010F947EB19B01AC01C701B6010F9401
:106DA000EBAF6B017C011150DBCFDF91CF911F91D5
:106DB000FF90EF90DF90CF90BF90AF909F908F901B
:106DC000089572CFCF93DF93EC016EDFCE01DF9198
:106DD000CF91D8CEFC0165917591859194910895DC
:106DE000EF92FF920F931F93CF93DF93EC01CC0FA1
:106DF000DD1FCC0FDD1FCE01875E9F4EEBDF9E01B6
:106E00002B57344F79018E010758144FF801208118
:106E10003181428153810F94ECAFF701608371831C
:106E200082839383CE018F5C9F4ED4DF9E01235DCE
:106E30003D4F7901F80120813181428153810F94C6
:106E4000ECAFF7016083718382839383CE018B5D06
:106E50009F4EC0DFCF5DDD4FF8012081318142813F
:106E600053810F94ECAF688379838A839B83DF918E
:106E7000CF911F910F91FF90EF900895CF93C82F5E
:106E800040910C0250910D0260910E0270910F0220
:106E900040933C0B50933D0B60933E0B70933F0B24
:106EA00020914702309148023093FB0B2093FA0B5C
:106EB00024E630E030934802209347020F94F6A76F
:106EC0006093370B7093380B8093390B90933A0B88
:106ED0008C2FCF910D94D41E80E00F94D41E8091FE
:106EE0003C0B90913D0BA0913E0BB0913F0B8093DA
:106EF0000C0290930D02A0930E02B0930F028091AA
:106F0000FA0B9091FB0B90934802809347020F94E9
:106F1000F6A76093370B7093380B8093390B9093DF
:106F20003A0B0895682F772767FD70958091DD10E3
:106F30009091DE108E519F4E0F94BEB99093D41055
:106F40008093D31021E0892B09F420E0822F08954B
:106F50002091DD103091DE10BC01C9018E519F4E91
:106F60000F94F6B99093D4108093D31021E0892B1D
:106F700009F420E0822F08958091D3109091D410CD
:106F80004AE050E060E070E001960D94CFB70F93B7
:106F90001F93CF93DF930091D3101091D41065E429
:106FA00070E0C8010F94BEB9EC01009751F460E0A5
:106FB00070E0C8010196DF91CF911F910F910D9460
:106FC00067B618828091D3109091D41060E070E081
:106FD00001960F9467B625E42883DF91CF911F9126
:106FE0000F9108958091D3109091D41060E070E0DB
:106FF00001960D9467B62F923F924F925F926F92D7
:107000007F928F929F92AF92BF92CF92DF92EF9238
:10701000FF920F931F93CF93DF93CDB7DEB76097A7
:107020000FB6F894DEBF0FBECDBF1C012A013B0195
:107030004801590120E030E04CE052E4C301B201C4
:107040000F94EBAF25E535E547E052E40F94E3B04C
:107050006B017C010F94B9B10F944BB18B0177FF99
:1070600012C020E030E040E85FE3C701B6010F94B2
:107070000BB318160CF05DC0C12CD12CE0E8EE2E3D
:10708000EFE3FE2E56C066307105DCF02AEA3AE2E4
:107090004CE453E4C301B2010F94EBAF25E535E5B1
:1070A00047E052E40F94E3B06B017C0120E030E054
:1070B000A9010F94DCB087FF3FC0C12CD12C760111
:1070C0003BC0882777FD8095982F0F947EB125E5EA
:1070D00035E547E052E40F94DDB320E030E04CE0CA
:1070E00052E40F94ECAF9B01AC01C301B2010F94C9
:1070F000EBAF25E535E547E052E40F94E3B06B01D3
:107100007C0120E030E0A9010F94DCB087FD17C0BE
:1071100020E030E040E85FE3C701B6010F940BB315
:10712000181684F4C12CD12C70E8E72E7FE3F72EDB
:1071300009C000E010E006C005E010E003C0C12C6B
:10714000D12C760120E030E040EC50E4C501B401E0
:107150000F94EBAF2BEA3AEA42E052E40F94E3B02B
:107160002B013C010F94B9B10F944BB1788B6F8711
:1071700077FF12C020E030E040E85FE3C301B201D6
:107180000F940BB318160CF05FC0412C512C60E823
:10719000662E6FE3762E58C0AF85B8891697E4F057
:1071A00026E535E549E253E4C501B4010F94EBAFA0
:1071B0002BEA3AEA42E052E40F94E3B02B013C019F
:1071C00020E030E0A9010F94DCB087FD40C0E5E08D
:1071D000F0E0F88BEF8746C0882777FD8095982FE1
:1071E0000F947EB12BEA3AEA42E052E40F94DDB309
:1071F00020E030E040EC50E40F94ECAF9B01AC0198
:10720000C501B4010F94EBAF2BEA3AEA42E052E435
:107210000F94E3B02B013C0120E030E0A9010F9472
:10722000DCB087FD1CC020E030E040E85FE3C30134
:10723000B2010F940BB31816ACF4412C512C50E84A
:10724000652E5FE3752E0EC0188A1F860BC0412C79
:10725000512C320125E030E0388B2F8703C0412CC0
:10726000512C3201A701960160E070E080E89FE3B5
:107270000F94EBAF69837A838B839C83C80101965B
:107280009E838D83AF85B8891196BA87A987A3019C
:10729000920160E070E080E89FE30F94EBAF6B87B2
:1072A0007C878D879E8747E02F853889429FF00134
:1072B000439FF00D1124F887EF83E00FF11FEE0FCD
:1072C000FF1FEE0FFF1FE20DF31D2181328143816D
:1072D000548169817A818B819C810F94DDB34B014C
:1072E0005C01EF81F8858D819E81E80FF91FEE0F1B
:1072F000FF1FEE0FFF1FE20DF31D2181328143813D
:107300005481C701B6010F94DDB39B01AC01C501E7
:10731000B4010F94ECAF9B01AC016B857C858D852E
:107320009E850F94DDB34B015C0127E0E985FA856A
:107330002E9FD0012F9FB00D1124B887AF83FD0180
:10734000E00FF11FEE0FFF1FEE0FFF1FE20DF31D09
:10735000218132814381548169817A818B819C8131
:107360000F94DDB369837A838B839C83AF81B88567
:107370008D819E81A80FB91FAA0FBB1FAA0FBB1F2B
:10738000A20DB31D11962D913D914D915C911497D5
:10739000C701B6010F94DDB39B01AC0169817A810D
:1073A0008B819C810F94ECAF9B01AC01C301B201B6
:1073B0000F94DDB39B01AC01C501B4010F94ECAF98
:1073C00060960FB6F894DEBF0FBECDBFDF91CF91B0
:1073D0001F910F91FF90EF90DF90CF90BF90AF90F3
:1073E0009F908F907F906F905F904F903F902F90E5
:1073F00008954F925F926F927F929F92AF92BF9249
:10740000CF92DF92EF92FF920F931F93CF93DF9370
:107410007C015B018A01E90190900F13911014C067
:10742000FC0180819181A281B381FA0180839183E3
:10743000A283B383FB0180819181A281B381888380
:107440009983AA83BB837FC091FE55C0FC01208134
:107450003181428153816091FF12709100138091BC
:107460000113909102130F94DDB32B013C01F50140
:107470002081318142815381609103137091041303
:1074800080910513909106130F94DDB39B01AC011D
:10749000C301B2010F94ECAFF80160837183828362
:1074A0009383F701208131814281538160910713D9
:1074B000709108138091091390910A130F94DDB312
:1074C0006B017C01F5012081318142815381609102
:1074D0000B1370910C1380910D1390910E130F9458
:1074E000DDB39B01AC01C701B6010F94ECAF68831B
:1074F00079838A839B8390FE26C02091E712309186
:10750000E8124091E9125091EA12F801608171810C
:10751000828193810F94ECAFF80160837183828341
:1075200093832091EB123091EC124091ED12509127
:10753000EE12688179818A819B810F94ECAF688318
:1075400079838A839B83DF91CF911F910F91FF9065
:10755000EF90DF90CF90BF90AF909F907F906F9013
:107560005F904F9008952F923F924F925F926F924B
:107570007F928F929F92AF92BF92CF92DF92EF92C3
:10758000FF920F931F93CF93DF93CDB7DEB728976A
:107590000FB6F894DEBF0FBECDBF8C011B019E015C
:1075A0002F5F3F4FAE014B5F5F4F23DF20E030E0A6
:1075B000A9016D817E818F8198850F94DCB087FF52
:1075C00007C01D821E821F821886FF24F39401C00B
:1075D000F12C20E030E040E451EC69817A818B812C
:1075E0009C810F94DCB087FF0AC080E090E0A0E4AB
:1075F000B1EC89839A83AB83BC83FF24F39420E0AE
:1076000030E04FE753E46D817E818F8198850F9440
:107610000BB3181654F480E090E0AFE7B3E48D8329
:107620009E83AF83B887FF24F39420E030E042E5E7
:1076300053E469817A818B819C810F940BB3181676
:107640004CF480E090E0A2E5B3E489839A83AB83B5
:10765000BC8303C0FF2009F483C0C980DA80EB80BB
:10766000FC808D809E80AF80B88470900F13711065
:107670000BC0F80180829182A282B382F101C082A4
:10768000D182E282F3826AC070FE1CC02091E712B0
:107690003091E8124091E9125091EA12C501B4010B
:1076A0000F94EBAF4B015C012091EB123091EC1287
:1076B0004091ED125091EE12C701B6010F94EBAF5D
:1076C0006B017C0171FE4AC02091EF123091F012E3
:1076D0004091F1125091F212C501B4010F94DDB343
:1076E0002B013C012091F3123091F4124091F512DC
:1076F0005091F612C701B6010F94DDB39B01AC01A6
:10770000C301B2010F94ECAFF801608371838283EF
:1077100093832091F7123091F8124091F912509111
:10772000FA12C501B4010F94DDB34B015C01209145
:10773000FB123091FC124091FD125091FE12C701D4
:10774000B6010F94DDB39B01AC01C501B4010F94E8
:10775000ECAFF1016083718382839383FF24F39400
:107760008F2D28960FB6F894DEBF0FBECDBFDF91E8
:10777000CF911F910F91FF90EF90DF90CF90BF902E
:10778000AF909F908F907F906F905F904F903F90C1
:107790002F900895CF93DF931F92CDB7DEB7BE0130
:1077A0006F5F7F4F0F944C5B0F90DF91CF910895E7
:1077B000682F87EF9FE00D947CBC0895FC01249115
:1077C000222341F03091C00035FFFCCF2093C6004A
:1077D0000196F4CF22E030E08EE39AE0F2CAFC0199
:1077E0002491222341F03091C00035FFFCCF20933B
:1077F000C6000196F4CF2AE030E08EE39AE01DCA7D
:10780000CF9364E674E08EE39AE0D0D9C1E0C093F0
:10781000A2026FEF89E69FE00F947CBCC093CF0279
:10782000CF91089564E774E08EE39AE0BFD9109297
:10783000A20260E089E69FE00F947CBC1092CF0228
:107840000895EF92FF920F931F93CF93DF931F92B0
:10785000CDB7DEB789830F940D578981823009F443
:1078600068C0B4F5882309F442C0813009F0F4C03F
:107870009FB7F894809102018460809302019FBFBA
:10788000EFEFF1EE24E0E150F0402040E1F700C0DE
:1078900000009FB7F894809102018B7F80930201D2
:1078A0009FBF40E050E0BA018DEE9FE00F948EBC88
:1078B00040E050E0BA0181EF9FE00F948EBC0F9042
:1078C000DF91CF911F910F91FF90EF900D948C7CE1
:1078D000833009F45CC0843009F0BEC00F90DF91A2
:1078E000CF911F910F91FF90EF900D94FB849FB764
:1078F000F894809102018460809302019FBF2FEF72
:1079000081EE94E0215080409040E1F700C00000FB
:107910009FB7F894809102018B7F809302019FBFF3
:107920000F90DF91CF911F910F91FF90EF900D94E9
:10793000B5570F94B55780EF3BDF10921A1C109289
:10794000191C60911B1C84EC9FE00F947CBC69E1C6
:107950007CE181EC9FE00F9439579FB7F8948091B8
:1079600002018460809302019FBF8FEF91EEE4E0FB
:1079700081509040E040E1F700C000009FB7F894CC
:10798000809102018B7F809302019FBF65C080EFD1
:107990009FE00F94956C4FED5FE062E081E00F9403
:1079A000F2889FB7F894809102018460809302016D
:1079B0009FBFFFEF21EE84E0F15020408040E1F7CF
:1079C00000C000009FB7F894809102018B7F8093E4
:1079D00002019FBF1092230B1092220B48ED5FE033
:1079E00063E083E00F94F2884091220B5091230BC7
:1079F00063E083E00F941857E12CF12C09E210E0CA
:107A00006FEFC7010F949ABCC701B8010F94BBB5C3
:107A1000892BD9F48091220B9091230B019690939E
:107A2000230B8093220B41ED5FE063E083E00F9432
:107A3000F2884091220B5091230B63E083E00F9476
:107A400018578FEC9FE00F94956C9FEFE91AF90A95
:107A5000E114E0E1FE06A1F60F90DF91CF911F91B6
:107A60000F91FF90EF90089580E1E5E8FBE0A0E53D
:107A7000BBE001900D928A95E1F708954F925F92D5
:107A80006F927F928F929F92AF92BF92CF92DF922E
:107A9000EF92FF92CF93DF9300D01F92CDB7DEB766
:107AA0000F9447288BE43EDA882391F070DA6B015B
:107AB0007C0120E030E0A9010F940BB387FD08C0E2
:107AC000C092F813D092F913E092FA13F092FB13DC
:107AD00082E528DA882359F05ADA6B017C0120E02C
:107AE00030E0A9010F94DCB087FF83C006C0C12C31
:107AF000D12C60E8E62E6FEBF62E84E413DA8823AF
:107B000021F045DA4B015C0106C0812C912C50E834
:107B1000A52E5FEBB52E87E505DA882321F037DA4D
:107B20002B013C0106C0412C512C40E8642E4FEB48
:107B3000742E88E4F7D9882331F029DA69837A83AF
:107B40008B839C8308C080E090E0A0E8BFEB898332
:107B50009A83AB83BC8320E030E0A901C501B40166
:107B60000F940BB387FD45C020E030E0A901C301AD
:107B7000B2010F940BB387FD3CC020E030E0A901B7
:107B800069817A818B819C810F940BB387FD31C011
:107B900020E030E0A901C501B4010F94DCB08823D6
:107BA00091F120E030E040E05FE3C501B4010F94C3
:107BB000DDB36B017C0129813A814B815C81C3017A
:107BC000B2010F94DDB34B015C01A7019601C7011F
:107BD000B6010F94DDB32BED3FE049E450E40F9480
:107BE000DDB39B01AC01C501B4010F94E3B06B019F
:107BF0007C0120E030E0A901C701B6010F940BB36E
:107C000087FF04C00BC0C12CD12C7601C092F413A5
:107C1000D092F513E092F613F092F713EDE3F0E152
:107C20008491882341F09091C00095FFFCCF809310
:107C3000C6003196F5CFEEE2FAE08491882341F058
:107C40009091C00095FFFCCF8093C6003196F5CF90
:107C50004091F8135091F9136091FA137091FB134E
:107C600022E030E08EE39AE0ACD88091C00085FF3E
:107C7000FCCF8AE08093C600E8E2FAE08491882392
:107C800041F09091C00095FFFCCF8093C6003196E3
:107C9000F5CFC090F413D090F513E090F613F09068
:107CA000F71320E030E0A901C701B6010F94DCB062
:107CB000882361F022E030E0B701A6018EE39AE06C
:107CC00080D88091C00085FFFCCF11C0E3E2FAE0CC
:107CD0008491882341F09091C00095FFFCCF809360
:107CE000C6003196F5CF8091C00085FFFCCF8AE0B9
:107CF0008093C6000F900F900F900F90DF91CF915F
:107D0000FF90EF90DF90CF90BF90AF909F908F90BB
:107D10007F906F905F904F9008952F923F924F9277
:107D20005F926F927F928F929F92AF92BF92CF920B
:107D3000DF92EF92FF920F931F93CF93DF931F92E7
:107D4000CDB7DEB7E0E0F8E28591949123DD81E0E4
:107D50000F94D41E8983E0E0F0E1E4918E2F9927FF
:107D600081950CF490951C0184E00F94D943ADE803
:107D7000BBE01D921D921D921C921397E9E8FBE057
:107D80002081318142815381A5E8BBE06D917D91D5
:107D90008D919C91E1E9CE2EEBE0DE2EE12CF12CD1
:107DA00087010F945F1B60DE85E190E113D82DEC15
:107DB0003CEC4CE85FE30F94DDB34B015C01B10197
:107DC000882777FD8095982F0F947EB19B01AC0199
:107DD000C501B4010F94DDB3E8E5FBE020813181FA
:107DE000428153810F94ECAF2B013C01A8E5BBE02D
:107DF0006D937D938D939C931397E1E5F2E0608101
:107E000071818281938160930C0270930D02809343
:107E10000E0290930F0220E030E040E752E40F940E
:107E2000E3B04B015C01A4E5BBE02D913D914D9188
:107E30005C91E0E5FBE06081718182819381A1E743
:107E4000BBE0BF93AF93FCE5CF2EFBE0DF2E8301B9
:107E500072010F94B10E82E00F944E410F944728A7
:107E60000F94594480E00F94D41EADE8BBE01D92FE
:107E70001D921D921C921397E9E8FBE0208131814D
:107E800042815381A5E8BBE06D917D918D919C91DC
:107E9000A1E9CA2EABE0DA2EE12CF12C87010F9478
:107EA0005F1BE2DD2AE0229DC001239D900D11247D
:107EB000BC01882777FD8095982F0F947EB1E8E567
:107EC000FBE020813181428153810F94ECAF2B0183
:107ED0003C01A8E5BBE06D937D938D939C93139734
:107EE00020E030E040E05FE3E1E5F2E060817181B5
:107EF000828193810F94DDB360930C0270930D0225
:107F000080930E0290930F0220E030E040E752E4AD
:107F10000F94E3B04B015C01A4E5BBE02D913D91D2
:107F20004D915C91E0E5FBE06081718182819381FC
:107F3000A1E7BBE0BF93AF93BCE5CB2EBBE0DB2E4C
:107F4000830172010F94B10E0F94472889810F9419
:107F5000D41E80E090E0AFE4B3E4EDE8FBE0808382
:107F60009183A283B383A9E8BBE02D913D914D910C
:107F70005C91E5E8FBE0608171818281938111E988
:107F8000C12E1BE0D12EE12CF12C0FE413E40F9451
:107F90005F1B81E00F900F900F900F900F90DF917B
:107FA000CF911F910F91FF90EF90DF90CF90BF90F6
:107FB000AF909F908F907F906F905F904F903F9089
:107FC0002F9008952F923F924F925F926F927F92DF
:107FD0008F929F92AF92BF92CF92DF92EF92FF92D9
:107FE0000F931F93CF93DF93CDB7DEB729970FB6CB
:107FF000F894DEBF0FBECDBF3C0181E00F94D41ECC
:108000008F8382E06816710408F081C2F301E250A8
:10801000F04FE491D301AA0FBB1FAA0FBB1FBA8375
:10802000A983A75BBD4FBE83AD838D919D910D90BC
:10803000BC91A02D80930C0290930D02A0930E0290
:10804000B0930F0281E0062C01C0880F0A94EAF772
:108050000F94D943E981FA81EB57F44FF987E88708
:108060001082118212821382E0908D0BF0908E0BA1
:1080700000918F0B1091900B2091890B30918A0BFE
:1080800040918B0B50918C0B6091850B7091860BFE
:108090008091870B9091880BE1E9CE2EEBE0DE2EEC
:1080A0000F945F1BE981FA81E05BF44F2F0180E0C0
:1080B00090E0A0E4B0E480839183A283B38320E0C6
:1080C00030E040E752E460910C0270910D02809123
:1080D0000E0290910F020F94E3B04B015C01E0900F
:1080E000580BF090590B00915A0B10915B0B20919B
:1080F000540B3091550B4091560B5091570B60919A
:10810000500B7091510B8091520B9091530BF1E7F2
:108110002F2EFBE03F2E3F922F92ACE5CA2EABE014
:10812000DA2E0F94B10E0F9447280F94BC1E80E0F6
:108130000F94D41EA885B9851D921D921D921C9284
:108140001397E0908D0BF0908E0B00918F0B109198
:10815000900B2091890B30918A0B40918B0B5091A1
:108160008C0B6091850B7091860B8091870B9091A1
:10817000880BB1E9CB2EBBE0DB2E0F945F1B80E0B8
:1081800090E0A0E8BFEBF20180839183A283B383E8
:1081900020E030E040E752E460910C0270910D0263
:1081A00080910E0290910F020F94E3B04B015C019D
:1081B000E090580BF090590B00915A0B10915B0B0B
:1081C0002091540B3091550B4091560B5091570B09
:1081D0006091500B7091510B8091520B9091530B09
:1081E0003F922F92ECE5CE2EEBE0DE2E0F94B10EF7
:1081F0000F94472881E00F94D41E89819A81835F70
:108200009F4E0E94EA362DEC3CEC4CE85FEB0F945D
:10821000DDB3D2016D937D938D939C93139720E0F2
:1082200030E040E752E460910C0270910D028091C1
:108230000E0290910F020F94E3B04B015C01E090AD
:10824000580BF090590B00915A0B10915B0B209139
:10825000540B3091550B4091560B5091570B609138
:10826000500B7091510B8091520B9091530B3F9298
:108270002F920F94B10E0F9447280F94BC1E80E0EC
:108280000F94D41EE885F985108211821282138220
:10829000E0908D0BF0908E0B00918F0B1091900B56
:1082A0002091890B30918A0B40918B0B50918C0B54
:1082B0006091850B7091860B8091870B9091880B54
:1082C000F1E9CF2EFBE0DF2E0F945F1B80E090E002
:1082D000A0E2B1E4F20180839183A283B38320E022
:1082E00030E040E752E460910C0270910D02809101
:1082F0000E0290910F020F94E3B04B015C01E090ED
:10830000580BF090590B00915A0B10915B0B209178
:10831000540B3091550B4091560B5091570B609177
:10832000500B7091510B8091520B9091530B3F92D7
:108330002F92ACE5CA2EABE0DA2E0F94B10E0F945B
:1083400047280F94BC1E81E00F94D41E80E090E07B
:10835000A0E7B1ECF20180839183A283B38320E094
:1083600030E040E05FE3AD81BE816D917D918D9104
:108370009C910F94DDB360930C0270930D02809377
:108380000E0290930F0220E030E040E752E40F9499
:10839000E3B04B015C01E090580BF090590B009159
:1083A0005A0B10915B0B2091540B3091550B40915F
:1083B000560B5091570B6091500B7091510B80915F
:1083C000520B9091530B3F922F920F94B10E0F943A
:1083D0004728C3010E94F036F301EA58F44F81E0C8
:1083E00080830F9459440F94BC1E80E00F94D41ED8
:1083F0002AE037ED43E25FE3E885F985608171812A
:10840000828193810F94EBAFA885B9856D937D939D
:108410008D939C931397E0908D0BF0908E0B0091B1
:108420008F0B1091900B2091890B30918A0B40910A
:108430008B0B50918C0B6091850B7091860B80910A
:10844000870B9091880BB1E9CB2EBBE0DB2E0F940C
:108450005F1B2AE037ED43E25FE3E885F985608141
:108460007181828193810F94ECAFA885B9856D935A
:108470007D938D939C931397F20160837183828324
:1084800093832AE939E949E95EE360910C0270912E
:108490000D0280910E0290910F020F94DDB320E047
:1084A00030E040E752E40F94E3B04B015C01E09010
:1084B000580BF090590B00915A0B10915B0B2091C7
:1084C000540B3091550B4091560B5091570B6091C6
:1084D000500B7091510B8091520B9091530B3F9226
:1084E0002F92ECE5CE2EEBE0DE2E0F94B10E0F9422
:1084F000472810920C0210920D0210920E02109258
:108500000F020FB6F894DEBF0FBECDBF62C192E07E
:108510006916710409F05DC1E0E0F0E17490109219
:108520008D0B10928E0B10928F0B1092900B20914E
:10853000890B30918A0B40918B0B50918C0B609181
:10854000850B7091860B8091870B9091880BF1E9D8
:10855000CF2EFBE0DF2EE12CF12C87010F945F1B67
:1085600085E190E10E94EA364B015C01672D772797
:1085700067FD7095872F972F0F947EB12B013C01DB
:1085800020E030E040EC5FE3C501B4010F94DDB3BF
:10859000A30192010F94DDB369837A838B839C835B
:1085A0006093580B7093590B80935A0B90935B0B0D
:1085B0006091510270915202809153029091540245
:1085C00060930C0270930D0280930E0290930F0241
:1085D00020E030E040E752E40F94E3B04B015C014F
:1085E0002091540B3091550B4091560B5091570BE5
:1085F0006091500B7091510B8091520B9091530BE5
:10860000A1E72A2EABE03A2E3F922F92BCE5CB2E6B
:10861000BBE0DB2EE980FA800B811C810F94B10E48
:108620000F94472810928D0B10928E0B10928F0B87
:108630001092900B2091890B30918A0B40918B0BFB
:1086400050918C0B6091850B7091860B8091870BFC
:108650009091880B11E9C12E1BE0D12EE12CF12C59
:1086600087010F945F1B89E090E10E94EA369058E1
:10867000A30192010F94DDB369837A838B839C837A
:108680006093580B7093590B80935A0B90935B0B2C
:1086900020E030E040E752E460910C0270910D025E
:1086A00080910E0290910F020F94E3B04B015C0198
:1086B0002091540B3091550B4091560B5091570B14
:1086C0006091500B7091510B8091520B9091530B14
:1086D0003F922F920CE5C02E0BE0D02EE980FA805D
:1086E0000B811C810F94B10E0F94472889E090E113
:1086F0000E94EA369B01AC010F94ECAFA3019201FA
:108700000F94DDB32B013C016093580B7093590B10
:1087100080935A0B90935B0B20E030E040E05FE3E6
:1087200060915102709152028091530290915402D3
:108730000F94DDB360930C0270930D0280930E02D0
:1087400090930F0220E030E040E752E40F94E3B052
:108750004B015C012091540B3091550B4091560B0D
:108760005091570B6091500B7091510B8091520BAF
:108770009091530B3F922F92830172010F94B10E8F
:108780000F94472882E090E00E94F03680918D0B94
:1087900090918E0BA0918F0BB091900B8093580B02
:1087A0009093590BA0935A0BB0935B0B10920C0251
:1087B00010920D0210920E0210920F020F94BC1E26
:1087C00081E08093780B0F900F900F900F900F9097
:1087D0000F908F8129960FB6F894DEBF0FBECDBFE4
:1087E000DF91CF911F910F91FF90EF90DF90CF908D
:1087F000BF90AF909F908F907F906F905F904F90C1
:108800003F902F900D94D41ECF92DF92EF92FF9263
:108810000F931F9329D980E090E0D4DB81E090E0B2
:10882000D1DBE0908D0BF0908E0B00918F0B1091AF
:10883000900B2091890B30918A0B40918B0B5091BA
:108840008C0B6091850B7091860B8091870B9091BA
:10885000880BF1E9CF2EFBE0DF2E0F945F1B1F91F9
:108860000F91FF90EF90DF90CF900D94BC1E0F946E
:10887000F6A76093370B7093380B8093390B909366
:108880003A0B089520E030E0A90168EB71E084E53F
:108890000F9444AC69E170E080E090E00F9425A86B
:1088A00084E50F946AAF64E170E080E090E00D949D
:1088B00025A87F928F929F92AF92BF92CF92DF9224
:1088C000EF92FF920F931F93CF93DF9300D01F92ED
:1088D000CDB7DEB71092111B1092101B10920F1B18
:1088E00010920E1B0F940D5786ED9EE00F94956C21
:1088F0008E010F5F1F4F7E0125E0E20EF11C8EE31B
:108900009AE00E94F0348F3FEFEF9E07C1F3F80129
:1089100081938F01EE15FF0591F789809A80AB80D6
:10892000BC808091C00085FFFCCF8BE28093C600A5
:10893000C12CD12C7601ABE27A2E8091C10B882319
:1089400009F450C001EE1AE0C814D904EA04FB048B
:10895000A1F08EE39AE00E94F0348F3FFFEF9F0773
:10896000C1F32FEFC21AD20AE20AF20AF801819388
:108970008F01FBE001321F0739F761EE7AE084E0F6
:108980009CE00E942FAC8091C00085FFFCCF7092CC
:10899000C6000F94DD39C814D904EA04FB0469F653
:1089A00071DF60E084E09CE00E9462AD1092C10B38
:1089B000ECEBF7E285919491FC012491222341F0A4
:1089C0003091C00035FFFCCF2093C6000196F4CF54
:1089D0008091C00085FFFCCF8AE08093C60080E0D4
:1089E00090E000C00F900F900F900F90DF91CF910B
:1089F0001F910F91FF90EF90DF90CF90BF90AF90BD
:108A00009F908F907F9008950F94F6A76093370BF7
:108A10007093380B8093390B90933A0BE091DD10F3
:108A2000F091DE10E152FF4E80818130B9F4E0E533
:108A3000F7E285919491FC012491222341F0309139
:108A4000C00035FFFCCF2093C6000196F4CF809183
:108A5000C00085FFFCCF8AE08093C60008958EE3B6
:108A60009AE00E940C35E6E2F7E285919491FC01D0
:108A70002491222341F03091C00035FFFCCF209398
:108A8000C6000196F4CF4091C3105091C41060917C
:108A9000C5107091C6104F5F5F4F6F4F7F4F2AE038
:108AA00030E08EE39AE00E94AB358091C00085FFF4
:108AB000FCCF8AE08093C600A7CF8F929F92AF929F
:108AC000BF92CF92DF92EF92FF920F931F93CF93BB
:108AD000DF93B3E7EB2EB6E0FB2E05E81BE0C0E525
:108AE000DBE08CEFC82E8BE0D82EF70181917F015F
:108AF0000E949237882319F10E94F2374B015C01E2
:108B0000F6018081811103C060913B0B01C061E0DF
:108B100070E080E090E00F947EB1F8012081318117
:108B2000428153810F94DDB39B01AC01C501B401B7
:108B30000F94ECAF688379838A839B8309C0F80123
:108B400080819181A281B38188839983AA83BB8329
:108B50000C5F1F4F2496FFEFCF1ADF0A87E7E81656
:108B600086E0F80611F686E40E9492378823D9F051
:108B70000E94F2376B017C016093400B7093410BB4
:108B80008093420B9093430B20E030E0A9010F94B7
:108B90000BB3181644F4C0920C02D0920D02E0926E
:108BA0000E02F0920F02DF91CF911F910F91FF9073
:108BB000EF90DF90CF90BF90AF909F908F900895EF
:108BC0007CDF89E40E949237882359F00E94F237B3
:108BD0006093440B7093450B8093460B9093470B27
:108BE00008C01092440B1092450B1092460B109245
:108BF000470B8AE40E949237882359F00E94F2378B
:108C00006093480B7093490B80934A0B90934B0BE6
:108C100008951092480B1092490B10924A0B109233
:108C20004B0B0895CF92DF92EF92FF92CF93DF9399
:108C3000EC01BC016C5F7F4F0E94B33A20E030E052
:108C4000A9016091350270913602809137029091AE
:108C500038020F94ECAF6B017C019B01AC0168857D
:108C600079858A859B850F94DCB087FF04C0C88610
:108C7000D986EA86FB86C0902902D0902A02E0902D
:108C80002B02F0902C02A7019601688579858A85D0
:108C90009B850F940BB3181624F4C886D986EA86F0
:108CA000FB86DF91CF91FF90EF90DF90CF900895FA
:108CB0002F923F924F925F926F927F928F929F92EC
:108CC000AF92BF92CF92DF92EF92FF920F931F93DA
:108CD000CF93DF93CDB7DEB7AB970FB6F894DEBF77
:108CE0000FBECDBF9F878E87798B688B5B8B4A8B3E
:108CF0003D8B2C8B1F8B0E8BED82DC018D909D901C
:108D0000AD90BC904090850B5090860B6090870B87
:108D10007090880BDB018D919D910D90BC91A02DE1
:108D200088879987AA87BB87C090890BD0908A0BC8
:108D3000E0908B0BF0908C0B20918D0B30918E0B73
:108D400040918F0B5091900BEA89FB896081718172
:108D5000828193810F94EBAF688F798F8A8F9B8F7D
:108D600080911013811173C0AE89BF898D909D9041
:108D7000AD90BC90EA89FB89E080F180028113818B
:108D8000A889B9892D913D914D915C91EE85FF8522
:108D90006081718182819381FE013596FF93EF930B
:108DA000CC88DD880F94B10EEE85FF85808191819E
:108DB000A281B3818093850B9093860BA093870B40
:108DC000B093880BE889F98980819181A281B38170
:108DD0008093890B90938A0BA0938B0BB0938C0B91
:108DE000EA89FB8980819181A281B38180938D0B77
:108DF00090938E0BA0938F0BB093900BEC89FD8911
:108E000080819181A281B3818093910B9093920B89
:108E1000A093930BB093940B0F900F90AB960FB65B
:108E2000F894DEBF0FBECDBFDF91CF911F910F91A0
:108E3000FF90EF90DF90CF90BF90AF909F908F907A
:108E40007F906F905F904F903F902F900895A30177
:108E50009201C501B4010F94EBAF2B013C0120E05E
:108E600030E0A9010F940BB353014201181624F00E
:108E7000B7FAB094B7F8B094A701960168857985E0
:108E80008A859B850F94EBAF688779878A879B8754
:108E900020E030E0A9010F940BB3288539854A857D
:108EA0005B8518160CF05058C501B4010F94ECAF57
:108EB0006B017C0120E030E0A9010F940BB3181680
:108EC0000CF052CF20E030E040EF51E4C701B60192
:108ED0000F94E3B00F94C9B00F944BB17D876C87AA
:108EE000623071050CF440CF2091910B3091920BC0
:108EF0004091930B5091940BAC89BD896D917D91FC
:108F00008D919C910F94EBAF6C8F7D8F8E8F9F8F87
:108F100022242394312C8C859D85AA2797FDA0952A
:108F2000BA2F88A799A7AAA7BBA7DE011596BF836A
:108F3000AE83B101882777FD8095982F0F947EB17D
:108F40006B017C0168A579A58AA59BA50F947EB1CC
:108F50009B01AC01C701B6010F94E3B06B017C012A
:108F6000EE89FF8980809180A280B3802C8D3D8D19
:108F70004E8D5F8D0F94DDB39B01AC016091910B21
:108F80007091920B8091930B9091940B0F94ECAF96
:108F900069837A838B839C83288D398D4A8D5B8D81
:108FA000C701B6010F94DDB320918D0B30918E0B6C
:108FB00040918F0B5091900B0F94ECAF68A379A365
:108FC0008AA39BA3288539854A855B85C701B6019D
:108FD0000F94DDB32091890B30918A0B40918B0B5C
:108FE00050918C0B0F94ECAF6CA37DA38EA39FA329
:108FF000A3019201C701B6010F94DDB32091850B47
:109000003091860B4091870B5091880B0F94ECAFF9
:10901000FF81FF932E812F93DE0111966D01E8A051
:10902000F9A00AA11BA12CA13DA14EA15FA10F9403
:10903000B10EBFEF2B1A3B0A0F900F90EC85FD8508
:109040002E163F0609F075CF8FCE4F925F926F922A
:109050007F928F929F92AF92BF92CF92DF92EF92C8
:10906000FF920F931F93CF93DF93CDB7DEB728976F
:109070000FB6F894DEBF0FBECDBF80E59BE0D2DD1A
:109080000F94F6A76093370B7093380B8093390BCE
:1090900090933A0B8091500B9091510BA091520BF1
:1090A000B091530B8D839E83AF83B8879C01AD0134
:1090B0006091850B7091860B8091870B9091880B46
:1090C0000F94DCB0811197C04090540B5090550B19
:1090D0006090560B7090570BA30192016091890B21
:1090E00070918A0B80918B0B90918C0B0F94DCB05C
:1090F000811181C020E030E040E752E460910C0231
:1091000070910D0280910E0290910F020F94E3B0C6
:109110004B015C01E090580BF090590B00915A0BF9
:1091200010915B0B81E79BE09F938F932CE5C22E00
:109130002BE0D22EA30192016D817E818F819885D3
:109140000F94B10E0F900F908091500B9091510B96
:10915000A091520BB091530B8093850B9093860B8B
:10916000A093870BB093880B8091540B9091550B73
:10917000A091560BB091570B8093890B90938A0B5B
:10918000A0938B0BB0938C0B8091580B9091590B43
:10919000A0915A0BB0915B0B80938D0B90938E0B2B
:1091A000A0938F0BB093900B80915C0B90915D0B13
:1091B000A0915E0BB0915F0B8093910B9093920BFB
:1091C000A093930BB093940B28960FB6F894DEBF40
:1091D0000FBECDBFDF91CF911F910F91FF90EF9008
:1091E000DF90CF90BF90AF909F908F907F906F90C7
:1091F0005F904F900895E090710B609147027091DD
:109200004802882777FD8095982F0F947EB1209192
:109210000C0230910D0240910E0250910F020F94FA
:10922000DDB32EE333EC4EE259E30F94DDB36983F3
:109230007A838B839C838E010F5F1F4F2CE53BE06D
:1092400048E55BE064E57BE080E59BE031DD7CCFD9
:109250004F925F926F927F928F929F92AF92BF9246
:10926000CF92DF92EF92FF920F931F93CF93C62F6F
:10927000E091710BF0E0882309F4D9C0DF01A35914
:10928000B44F8C918111AFC18091850B9091860B69
:10929000A091870BB091880B8093500B9093510B4A
:1092A000A093520BB093530B8091890B90918A0B32
:1092B000A0918B0BB0918C0B8093540B9093550B1A
:1092C000A093560BB093570B80918D0B90918E0B02
:1092D000A0918F0BB091900B8093580B9093590BEA
:1092E000A0935A0BB0935B0BC090910BD090920B54
:1092F000E090930BF090940BC0925C0BD0925D0BBE
:10930000E0925E0BF0925F0BEE0FFF1FEE0FFF1F60
:10931000E75CFD4F2081318142815381662349F012
:109320006091190270911A0280911B0290911C02A7
:1093300008C060911D0270911E0280911F029091E1
:1093400020020F94E3B09B01AC01C701B6010F945A
:10935000ECAF6093910B7093920B8093930B90936F
:10936000940B81E99BE00F94FE1C80900C0290907E
:109370000D02A0900E02B0900F0220E030E040E716
:1093800052E460911502709116028091170290913B
:1093900018020F94DDB360930C0270930D0280935A
:1093A0000E0290930F02E091710BF0E0E359F44F3D
:1093B00081E080834ADE2091690B30916A0B4091F5
:1093C0006B0B50916C0B60918D0B70918E0B80919B
:1093D0008F0B9091900B0F94EBAF7B018C016093FE
:1093E0008D0B70938E0B80938F0B9093900B20912D
:1093F000890B30918A0B40918B0B50918C0B6091B3
:10940000850B7091860B8091870B9091880BE1E919
:10941000CE2EEBE0DE2E0F945F1B17DE80920C0247
:1094200090920D02A0920E02B0920F02DCC0E3599E
:10943000F44F8081882309F4D6C08090850B9090EA
:10944000860BA090870BB090880B8092500B909267
:10945000510BA092520BB092530B4090890B50903D
:109460008A0B60908B0B70908C0B4092540B509237
:10947000550B6092560B7092570B60918D0B70914B
:109480008E0B80918F0B9091900B6093580B709383
:10949000590B80935A0B90935B0B0091910B109199
:1094A000920B2091930B3091940B00935C0B1093D3
:1094B0005D0B20935E0B30935F0B2091690B309115
:1094C0006A0B40916B0B50916C0B0F94ECAF7B01CE
:1094D0008C0160938D0B70938E0B80938F0B909308
:1094E000900B31E9C32E3BE0D32EA3019201C501BD
:1094F000B4010F945F1B1091710BCC2389F0209164
:10950000610B3091620B4091630B5091640B609141
:10951000190270911A0280911B0290911C0210C0D6
:109520002091650B3091660B4091670B5091680B51
:1095300060911D0270911E0280911F029091200285
:109540000F94ECAF24E0129FF0011124E75CFD4F73
:1095500020813181428153810F94E3B09B01AC01A2
:109560006091910B7091920B8091930B9091940B61
:109570000F94EBAF6093910B7093920B8093930BCE
:109580009093940B81E99BE00F94FE1CC0900C0219
:10959000D0900D02E0900E02F0900F0220E030E03B
:1095A00040E752E46091110270911202809113021F
:1095B000909114020F94DDB360930C0270930D022E
:1095C00080930E0290930F02E091710BF0E0E3594B
:1095D000F44F10823ADDC0920C02D0920D02E0925C
:1095E0000E02F0920F02CF911F910F91FF90EF901A
:1095F000DF90CF90BF90AF909F908F907F906F90B3
:109600005F904F900895AF92BF92CF92DF92EF920A
:10961000FF920F931F93CF93DF93D82F2091480B86
:109620003091490B40914A0B50914B0B6091440B88
:109630007091450B8091460B9091470B0F9418B396
:10964000C62F172F082FF92E6091470270914802FC
:10965000882777FD8095982F0F947EB120910C027A
:1096600030910D0240910E0250910F020F94DDB324
:1096700020E030E040E752E40F94E3B020E030E037
:1096800048EC52E40F94E3B02091710B2F93DF93D9
:10969000FF920F931F93CF935B016C01B2E0EB2E0F
:1096A00001E020E044E45BE060E57BE085E89BE0EE
:1096B0000F9431058091500B9091510BA091520B5A
:1096C000B091530B8093850B9093860BA093870BDF
:1096D000B093880B8091540B9091550BA091560B31
:1096E000B091570B8093890B90938A0BA0938B0BAF
:1096F000B0938C0B8091580B9091590BA0915A0B01
:10970000B0915B0B80938D0B90938E0BA0938F0B7E
:10971000B093900B80915C0B90915D0BA0915E0BD0
:10972000B0915F0B8093910B9093920BA093930B4E
:10973000B093940B0F94F6A76093370B7093380B8C
:109740008093390B90933A0B0F900F900F900F90DE
:109750000F900F90DF91CF911F910F91FF90EF909D
:10976000DF90CF90BF90AF900895EC01ECE1FAE06C
:109770008491882341F09091C00095FFFCCF8093A5
:10978000C6003196F5CF70E04AE050E08EE39AE0F3
:109790000E94EA35F8940F947732179A1092760B5C
:1097A000169A1092770B149AE3E4F0E184918823DF
:1097B00041F09091C00095FFFCCF8093C600319698
:1097C000F5CFE6EDF7E285919491FC0124912223F7
:1097D00041F03091C00035FFFCCF2093C6000196C8
:1097E000F4CF8091C00085FFFCCF8AE08093C60053
:1097F0002097C9F0FE018491FE01882349F09091E1
:10980000C00095FFFCCF8093C60031968491F5CFC0
:109810008091C00085FFFCCF8AE08093C600CE0116
:109820000E94CA3B06C0E2E9F7E2859194910F9449
:109830004A587894C6E0D0E0219751F068EC70E087
:1098400080E090E00F9425A880E00F94A359F4CF16
:10985000F894FFCFCF92DF92EF92FF920F931F9376
:10986000CF93C82F8091D9109091DA10039714F4F8
:109870000E94B3B50F94F6A70091330B1091340BEF
:109880002091350B3091360BC090370BD090380BB0
:10989000E090390BF0903A0B6C197D098E099F0905
:1098A000061717072807390740F4012B022B032B53
:1098B00021F064E083EF98E058DF40910802509176
:1098C000090260910A0270910B02452B462B472B2F
:1098D00019F10F94F6A70091370B1091380B2091D6
:1098E000390B30913A0B601B710B820B930B00917B
:1098F00008021091090220910A0230910B0206170A
:1099000017072807390740F49091FD138091FC1345
:10991000981302C0CC2349F0CF911F910F91FF9073
:10992000EF90DF90CF900D94DF0C179A1092760B8A
:10993000169A1092770B149AEFCF0F94773280918A
:10994000250B81113DC081E08093250B8091C310D0
:109950009091C410A091C510B091C6108093BF1013
:109960009093C010A093C110B093C210E3E4F0E153
:109970008491882341F09091C00095FFFCCF8093A3
:10998000C6003196F5CFECECF7E285919491FC019D
:109990002491222341F03091C00035FFFCCF209369
:1099A000C6000196F4CF8091C00085FFFCCF8AE00D
:1099B0008093C600E2EBF6E2859194910D942458D1
:1099C00008958091250B0895CF93DF93EC0180914A
:1099D000710B8093260B84E50E949237811102C09F
:1099E00080E084C00E94F2370F9450B16093260B40
:1099F0006623B1F3EDE3F0E18491882341F0909187
:109A0000C00095FFFCCF8093C6003196F5CFCD36D0
:109A1000D10509F435C064F4C836D105B1F0C936B2
:109A2000D10509F052C0E4E8F7E2A591B49124C051
:109A3000CA3DD10509F432C0CD3DD10509F045C07C
:109A4000E8E7F7E2A591B4913DC0E6E8F7E2859139
:109A50009491FC012491222309F437C03091C00075
:109A600035FFFCCF2093C6000196F3CF9091C00044
:109A700095FFFCCF8093C6008D918111F7CF25C053
:109A8000E2E8F7E2A591B4918D918823F1F09091ED
:109A9000C00095FFFCCF8093C600F6CFEAE7F7E25F
:109AA000A591B4918D91882381F09091C00095FF8C
:109AB000FCCF8093C600F6CF9091C00095FFFCCFFD
:109AC0008093C6008D918111F7CF6091260B70E0D5
:109AD0004AE050E08EE39AE00E94E3358091C000B6
:109AE00085FFFCCF8AE08093C60081E0DF91CF91B3
:109AF00008954F925F926F927F928F929F92AF9252
:109B0000BF92CF92DF92EF92FF92CF93DF9300D07C
:109B10001F92CDB7DEB72B013C0129833A834B83DB
:109B20005C838DEE9FE00F946ABC8F3F01F58EEE53
:109B30009FE00F946ABC8F3FD1F48FEE9FE00F94AB
:109B40006ABC8F3FA1F480EF9FE00F946ABC8F3F07
:109B500071F440E050E0BA018DEE9FE00F948EBCAE
:109B600040E050E0BA0181EF9FE00F948EBC81EF9E
:109B70009FE00F9472BC4B015C018DEE9FE00F944F
:109B800072BC6B017C0169817A818B819C812CE3A1
:109B900030E040E050E00F94CEB5C20ED31EE41E7C
:109BA000F51EB701A6018DEE9FE00F948EBCC30198
:109BB000B20128EE33E040E050E00F94CEB5BA0198
:109BC000A901480D591D6A1D7B1D81EF9FE00F946F
:109BD0008EBC1092BB0B1092BC0B1092BD0B10925E
:109BE000BE0B0F900F900F900F90DF91CF91FF90D1
:109BF000EF90DF90CF90BF90AF909F908F907F902D
:109C00006F905F904F900895CF92DF92EF92FF9206
:109C10002091950B2223F1F020E030E040E05FE35B
:109C20000F94DDB36B017C0120E030E0A9010F94BB
:109C3000DCB0882379F0A7019601C701B6010F9423
:109C4000DDB32BED3FE049E450E40F94DDB39B011D
:109C5000AC0104C020E030E040E85FE360E070E089
:109C600080E89FE30F94E3B0FF90EF90DF90CF90F8
:109C7000089560913D0270913E0280913F02909163
:109C80004002C2DF6093390270933A0280933B0234
:109C900090933C020895CF93DF93EC010F94DD394C
:109CA00081E0D8DD80E00F94A359209799F0C2336A
:109CB000D10540F062E370E080E090E00F9425A8C9
:109CC000E297ECCFBE0180E090E00F9425A8C0E0C1
:109CD000D0E0E4CFDF91CF9108952F923F924F9241
:109CE0005F926F927F928F929F92AF92BF92CF922C
:109CF000DF92EF92FF921F93CF93DF934B015C01B2
:109D0000CC24CA94DC2C760151E1252E5AE0352E64
:109D100068EE462E63E0562E612C712C1AE080917D
:109D2000600B811126C12FEFC216D206E206F206A1
:109D300051F0F7FC1EC10F94F6A76C197D09683B22
:109D40007B4008F016C10F94F6A7681979098A09B3
:109D50009B09693E73408105910508F47FC080919D
:109D60001B1C811177C0E9E1FAE08491882341F05E
:109D70009091C00095FFFCCF8093C6003196F5CF3F
:109D8000E091260B24E0E29FF0011124E85FF44EFD
:109D9000408151816281738121E030E08EE39AE05D
:109DA0000E94E136E5E1FAE08491882341F0909148
:109DB000C00095FFFCCF8093C6003196F5CF60912F
:109DC000260B70E04AE050E08EE39AE00E94E33513
:109DD000F1018491E1E1FAE0882349F09091C0001B
:109DE00095FFFCCF8093C60031968491F5CFF7FEA6
:109DF00003C0E4ECF9E025C00F94F6A74B015C0129
:109E0000C701B6016854744F8F4F9F4F6819790985
:109E10008A099B09A30192010F94CEB5BA01A90149
:109E20002AE030E08EE39AE00E94AB358091C000DA
:109E300085FFFCCF0DC09091C00095FFFCCF8093B3
:109E4000C60081918111F7CF8091C00085FFFCCFC2
:109E50001093C6000F94F6A74B015C010F94DD39F7
:109E600080E0F8DC80E00F94A359FFEFCF16DF0607
:109E7000EF06FF0609F046C08091240BE091260B07
:109E8000F0E0EF01CC0FDD1FCC0FDD1FC85FD44E1B
:109E9000EE0FFF1FE05FF44E8823D1F080819181A7
:109EA000BC01882777FD8095982F0F947EB120E024
:109EB00030E040E85FE30F94EBAF9B01AC016881B9
:109EC00079818A819B810F940BB387FF4DC027CF87
:109ED00080819181BC01882777FD8095982F0F9410
:109EE0007EB120E030E040E85FE30F94ECAF9B01EF
:109EF000AC01688179818A819B810F94DCB018164E
:109F00009CF50DCFF7FC0BCFE091260BF0E0EF01B5
:109F1000CC0FDD1FCC0FDD1FC85FD44EEE0FFF1F2F
:109F2000E05FF44E80819181BC01882777FD8095A8
:109F3000982F0F947EB19B01AC01688179818A8151
:109F40009B810F94EBAF0F944BB197FF07C0909597
:109F50008095709561957F4F8F4F9F4F663071054B
:109F6000810591050CF4DBCE0F94F6A76B017C0103
:109F7000D6CEDF91CF911F91FF90EF90DF90CF90E1
:109F8000BF90AF909F908F907F906F905F904F9019
:109F90003F902F900895CF93DF931F921F92CDB7DC
:109FA000DEB7BE016F5F7F4F88EF9FE00F944A5787
:109FB00089819A818156904F803A9F4020F11A8280
:109FC0001982E8EEF9E08491882341F09091C00075
:109FD00095FFFCCF8093C6003196F5CF8091C000ED
:109FE00085FFFCCF8AE08093C600BE016F5F7F4F84
:109FF00088EF9FE00F9439578BEA99E00F94185D32
:10A0000081E00F94105B0F900F90DF91CF91089536
:10A010002F923F924F925F926F927F928F929F9278
:10A02000AF92BF92CF92DF92EF92FF920F931F9366
:10A03000CF93DF93CDB7DEB7CA58D2400FB6F894AE
:10A04000DEBF0FBECDBFC958DD4F688379838A83D9
:10A050009B83C757D240FE01E75FFD4F88E2DF01D7
:10A060001D928A95E9F7E850F24080E991E0DF011E
:10A070009C011D9221503040E1F7C75ADD4F1982F3
:10A080001882C955D240CE01875A9D4F5C014E01BE
:10A090009FE6891A9EEF990ADE01AF51BE4F3D013E
:10A0A00090EBC92E9FE0D92E23E2E22EF12C00E0A6
:10A0B00010E0C359DD4F8882CD56D240CD58DD4FD8
:10A0C0009882C357D240B701882777FD8095982F93
:10A0D0000F947EB1D3016D937D938D939D933D013C
:10A0E000F501619171915F01882777FD8095982F27
:10A0F0000F947EB1D4016D937D938D939D934D010B
:10A100000F5F1F4F0630110559F0B501C6010F94BE
:10A110004A57B5E0EB0EF11CE2E0CE0ED11CD3CFD6
:10A12000CF51DE4F288139814A815B81C15ED140A8
:10A13000C958DD4F688179818A819B81C757D24098
:10A140000F94DCB087FD2BC3FE01EF51FE4F7F0162
:10A150006E01FFE2CF1AFEEFDF0A3E012BEB621A1F
:10A160002DEF720AC359DD4F0881CD56D240CD582C
:10A17000DD4F1881C357D24085E090E0CF58DD4FC6
:10A1800099838883C157D240CF58DD4FA881B981C8
:10A19000C157D2401197CF58DD4FB983A883C1571B
:10A1A000D240F701208931894289538964897589B0
:10A1B000868997890F94EBAF4B015C01D8015096CB
:10A1C0002D913D914D915C91539754966D917D9158
:10A1D0008D919C9157970F94EBAFA50194010F942B
:10A1E000E3B0F60192938293729362936F01D3016D
:10A1F000BE92AE929E928E923D0104501109B4E03F
:10A20000EB1AF108CF58DD4FE881F981C157D240F0
:10A21000EF2B09F0B9CF6E01FFECCF1AFDEFDF0A8B
:10A220003E0127E4621A2EEF720A2E013DE3430E2F
:10A23000511CCE0101967C0101E010E0D6018D9009
:10A240009D90AD90BC90139714962D913D914D919A
:10A250005C911797C501B4010F94ECAF9B01AC0161
:10A260000F94ECAFF70164A775A786A797A70130F5
:10A27000110541F080A691A6A2A6B3A6848295827C
:10A28000A682B7820F5F1F4FD30114962D913D9187
:10A290004D915C91179718966D917D918D919C9140
:10A2A0001B970F94EBAF20E030E040EC50E40F94AC
:10A2B000DDB3F2016083718382839383F4E0CF0E78
:10A2C000D11C2CE2E20EF11C34E0630E711C88E21A
:10A2D000480E511C0530110509F0B0CF8E010B5A04
:10A2E0001F4F6E0191E5C90ED11C22242394312CFD
:10A2F0002C0E3D1EA8ED2A0E311CF801B8972081C6
:10A30000318142815381F801608171818281938121
:10A310000F94E3B04B015C01E12CF12C3601F8E223
:10A320006F1A710826014E0C5F1CF301EE0DFF1D24
:10A330002481358146815781C501B4010F94DDB375
:10A340009B01AC01D20114966D917D918D919C91F0
:10A3500017970F94EBAFF20164837583868397831D
:10A36000F4E0EF0EF11C24E1E216F104D9F6045DED
:10A370001F4F38E2C30ED11C0215130509F0BDCFE3
:10A380001E0185EB280E311C6E0191EBC90ED11C0C
:10A390003E01A7EE6A1AADEF7A0A14E0E12EF12C25
:10A3A000270100E010E0812C912CA12CB12CF601AA
:10A3B000E00FF11FD301A00FB11F2D913D914D91E1
:10A3C0005C9160817181828193810F94DDB39B01E7
:10A3D000AC01B401C5010F94ECAF4B015C01BFEFC0
:10A3E0004B1A5B0A0C5F1F4FE5E04E165104F9F65D
:10A3F0009B01AC01D1016D917D918D919C910F9448
:10A40000EBAFF60120813181428153810F94E3B09B
:10A41000D3016D937D938D939C931397B1E0EB1AC9
:10A42000F108E8E22E1A3108FCE2CF1AD10824E044
:10A43000621A7108E114F10409F0B2CFCB50DE4F7B
:10A4400088819981AA81BB81C55FD140C957DD4F01
:10A4500088839983AA83BB83C758D2408E01075F44
:10A460001D4FDE01AF5CBD4FC558DD4FB983A883DA
:10A47000CB57D240C359DD4F2880CD56D240CD585E
:10A48000DD4F3880C357D240FE01EF51FE4FC35815
:10A49000DD4FF983E883CD57D240C358DD4FA88103
:10A4A000B981CD57D240CD90DD90ED90FD90C3584D
:10A4B000DD4FB983A883CD57D240C958DD4F2881DD
:10A4C00039814A815B81C757D240C701B6010F94D9
:10A4D000DCB01816B4F0C358DD4FE881F981CD57D0
:10A4E000D2402081318142815381C958DD4F68813A
:10A4F00079818A819B81C757D2400F94DCB01816AE
:10A50000FCF4CF58DD4F28813981C157D240243027
:10A51000310509F01FC1C957DD4F288139814A81B2
:10A520005B81C758D240C958DD4F688179818A81E3
:10A530009B81C757D2400F940BB318160CF00AC179
:10A54000D80114968D919D910D90BC91A02DC1586C
:10A55000DD4F88839983AA83BB83CF57D240F8010C
:10A560004080518062807380C558DD4FA881B981D9
:10A57000CB57D2408D919D910D90BC91A02DC35988
:10A58000DD4F88839983AA83BB83CD56D240D10106
:10A590008D919D910D90BC91A02DCD57DD4F88835D
:10A5A0009983AA83BB83C358D240A7019601C95897
:10A5B000DD4F688179818A819B81C757D2400F9492
:10A5C000EBAFCD58DD4F688379838A839B83C35774
:10A5D000D24020E030E040E450E40F9440B46B01FE
:10A5E0007C01A3019201C158DD4F688179818A8184
:10A5F0009B81CF57D2400F94EBAF4B015C0120E021
:10A6000030E040EC50E4C359DD4F688179818A81A4
:10A610009B81CD56D2400F94DDB39B01AC01C501A7
:10A62000B4010F94E3B0A70196010F94DDB36B0161
:10A630007C0120E030E040E05FE3C301B2010F9411
:10A64000DDB34B015C01CD58DD4F288139814A8152
:10A650005B81C357D240CA01B9010F94DDB39B019E
:10A66000AC01C501B4010F94DDB39B01AC01C7017E
:10A67000B6010F94ECAF6B017C01CD57DD4F288103
:10A6800039814A815B81C358D240F101648175816F
:10A69000868197810F94EBAFC359DD4F28813981B3
:10A6A0004A815B81CD56D2400F94E3B04B015C01EF
:10A6B000C359DD4F288139814A815B81CD56D24013
:10A6C000CA01B9010F94ECAFA30192010F94DDB35D
:10A6D0002B013C01C359DD4F288139814A815B81BF
:10A6E000CD56D240C158DD4F688179818A819B81E6
:10A6F000CF57D2400F94DDB39B01AC01C301B2012F
:10A700000F94ECAF20E030E040EC50E40F94E3B065
:10A710009B01AC01C501B4010F94EBAFCD58DD4FE7
:10A72000288139814A815B81C357D2400F94DDB3C0
:10A730009B01AC01C701B6010F94ECAFCD57DD4FC3
:10A74000288139814A815B81C358D2400F94ECAF94
:10A750004B015C01CF58DD4F28813981C157D24070
:10A760002F5F3F4FCF58DD4F39832883C157D240E9
:10A770000C5F1F4FC558DD4F88819981CB57D24060
:10A780000496C558DD4F99838883CB57D24094E017
:10A79000290E311C2530310509F07FCE04C0812CF3
:10A7A000912CA12CB12CB401C501C657DD4F0FB6B9
:10A7B000F894DEBF0FBECDBFDF91CF911F910F91F7
:10A7C000FF90EF90DF90CF90BF90AF909F908F90D1
:10A7D0007F906F905F904F903F902F900895809161
:10A7E000EF0B8823C9F086EA9FE00F946ABC8823A8
:10A7F00099F06091021B7091031B8091041B909152
:10A80000051B06DC2091E1193091E2194091E31912
:10A810005091E4190D94E3B060E070E0CB0108952D
:10A820004F925F926F927F928F929F92AF92BF9260
:10A83000CF92DF92EF92FF920F931F93CF93DF930C
:10A84000CDB7DEB728970FB6F894DEBF0FBECDBFE9
:10A850000F94472880914702909148029093FB0BF8
:10A860008093FA0BE091710BF0E0EE0FFF1FE05FB9
:10A87000F44E60817181882777FD8095982F0F9421
:10A880007EB16093E30B7093E40B8093E50B9093A0
:10A89000E60B80916F0B9091700B9093E20B80937D
:10A8A000E10B0F94F6A76093C90B7093CA0B8093CA
:10A8B000CB0B9093CC0B8091850B9091860BA09144
:10A8C000870BB091880B89839A83AB83BC83809379
:10A8D000D10B9093D20BA093D30BB093D40B409099
:10A8E000890B50908A0B60908B0B70908C0B409270
:10A8F000D50B5092D60B6092D70B7092D80B8091EB
:10A900008D0B90918E0BA0918F0BB091900B8D833E
:10A910009E83AF83B8878093D90B9093DA0BA09373
:10A92000DB0BB093DC0B6091910B7091920B8091DB
:10A93000930B9091940B6093DD0B7093DE0B8093DF
:10A94000DF0B9093E00B20E030E040E85FE30F94F2
:10A95000EBAF6093910B7093920B8093930B90935A
:10A96000940B81E79BE09F938F93812C912CB8EC03
:10A97000AB2EB3E4BB2E11E9C12E1BE0D12EED802E
:10A98000FE800F811885A301920169817A818B81F4
:10A990009C810F94B10E20E030E040EA51E46091D8
:10A9A0008D0B70918E0B80918F0B9091900B0F946B
:10A9B000ECAF2B013C010F900F9020E030E042E51E
:10A9C00053E40F940BB318164CF040928D0B509239
:10A9D0008E0B60928F0B7092900B0CC080E090E019
:10A9E000A2E5B3E480938D0B90938E0BA0938F0B15
:10A9F000B093900BE0908D0BF0908E0B00918F0B2D
:10AA00001091900B2091890B30918A0B40918B0B08
:10AA100050918C0B6091850B7091860B8091870B08
:10AA20009091880BA1E76A2EABE07A2E7F926F920D
:10AA3000812C912CB0E7AB2EB1E4BB2EE1E9CE2EF8
:10AA4000EBE0DE2E0F94B10E1092111B1092101B32
:10AA50001092131B1092121B1092151B1092141BB4
:10AA600080E090E0A8E4B2E48093850B9093860B9D
:10AA7000A093870BB093880B80E090E0AEE3B3E443
:10AA80008093890B90938A0BA0938B0BB0938C0BC4
:10AA9000E0908D0BF0908E0B00918F0B1091900B2E
:10AAA0007F926F92812C912CF8E4AF2EF2E4BF2EAE
:10AAB0009C01AD01C501B4010F94B10E1092700B51
:10AAC00010926F0B0F900F900F900F9028960FB66B
:10AAD000F894DEBF0FBECDBFDF91CF911F910F91D4
:10AAE000FF90EF90DF90CF90BF90AF909F908F90AE
:10AAF0007F906F905F904F900D944728E091710B7D
:10AB000084E0E89FF0011124E85FF44E4081518118
:10AB100062817381E8EAF9E08491882341F09091A1
:10AB2000C00095FFFCCF8093C6003196F5CF22E0A0
:10AB300030E08EE39AE00E94E136E4EAF9E08491A5
:10AB4000882341F09091C00095FFFCCF8093C60010
:10AB50003196F5CF6091710B70E04AE050E08EE3E2
:10AB60009AE00E94E335E0EAF9E08491882341F01D
:10AB70009091C00095FFFCCF8093C6003196F5CF31
:10AB80004091F61A5091F71A6091F81A7091F91ADB
:10AB900021E030E08EE39AE00E94E1368091C0002F
:10ABA00085FFFCCF8AE08093C6000895CF93DF93A2
:10ABB00000D000D0CDB7DEB7179A1092760B169A58
:10ABC0001092770BEBE9F9E08491882341F09091A2
:10ABD000C00095FFFCCF8093C6003196F5CF8091E1
:10ABE000C00085FFFCCF8AE08093C60083E40F9409
:10ABF000F5473C012090BB103090BC104090BD1038
:10AC00005090BE100F948C1D281A390A4108510823
:10AC10000E94F0BA281A390A4108510857FE03C0A9
:10AC2000212C312C21019091FD138091FC13981758
:10AC300099F0E091FC1327E5E29FF0011124E25026
:10AC4000FC4E20E030E040E752E462A173A184A111
:10AC500095A10F94DDB308C060910C0270910D02B4
:10AC600080910E0290910F020F944BB17E836D8301
:10AC70000F94360D0E949AB31092060C789420E03F
:10AC800030E040E85FE36091910B7091920B80910E
:10AC9000930B9091940B0F94EBAF69837A838B8322
:10ACA0009C83E0908D0BF0908E0B00918F0B109198
:10ACB000900B2091890B30918A0B40918B0B509116
:10ACC0008C0B6091850B7091860B8091870B909116
:10ACD000880BA1E7BBE0BF93AF93812C912CE8ECEC
:10ACE000AE2EE3E4BE2EDE0111966D010F94B10E7F
:10ACF00020E030E040E85FE36091910B7091920BAF
:10AD00008091930B9091940B0F94EBAF69837A83AE
:10AD10008B839C832FE832EC45EF5FE360918D0BD2
:10AD200070918E0B80918F0B9091900B0F94ECAFE4
:10AD30006B017C0167E074E066197709F4E07695B1
:10AD40006795FA95E1F780E090E00F947CB120914F
:10AD5000E1193091E2194091E3195091E4190F94EF
:10AD6000E3B09B01AC01C701B6010F94ECAF7B01CE
:10AD70008C012091890B30918A0B40918B0B509163
:10AD80008C0B6091850B7091860B8091870B909155
:10AD9000880BA1E7BBE0BF93AF93812C912CA0E27D
:10ADA000AA2EA2E4BA2EDE0111966D010F94B10E07
:10ADB000B201A10181E99FE00F948EBC0F900F902A
:10ADC0000F900F9005E71FE0F12CB3E0EB2E809180
:10ADD0001013882341F18F2D6E2D0F949AB5B5E194
:10ADE0008B02F001112423E09202E00DF11D1124E9
:10ADF000EE0FFF1FEE0FFF1FE05FFC4E20E030E084
:10AE00004AE754E461817281838194810F94DDB3B8
:10AE100020E030E040E05FE30F94ECAF0F94B9B175
:10AE20000F944BB102C060E070E0C8010F9496BC73
:10AE3000F3940E5F1F4F89E0F812C9CFB30183E787
:10AE40009FE00F9496BC4091850B5091860B6091CA
:10AE5000870B7091880B8DE99FE00F948EBC409119
:10AE6000890B50918A0B60918B0B70918C0B81EA4E
:10AE70009FE00F948EBC40918D0B50918E0B609192
:10AE80008F0B7091900B8DE89FE00F948EBCBE01EC
:10AE90006B5F7F4F89E89FE00F943957E091710B0A
:10AEA000F0E0EE0FFF1FE05FF44E60818CE89FE062
:10AEB0000F947CBC60910E1B8BE89FE00F947CBCD0
:10AEC00060916F0B88E89FE00F947CBC61E085EA9D
:10AED0009FE00F947CBC0F944728E6E9F9E0849149
:10AEE000882341F09091C00095FFFCCF8093C6006D
:10AEF0003196F5CF83E40F94F5474AE050E0BC016A
:10AF00008EE39AE00E94403684E69FE00F946ABC8C
:10AF100061E0680F84E69FE00F947CBCEBE8F9E009
:10AF20008491882341F09091C00095FFFCCF8093DD
:10AF3000C6003196F5CF8091C00085FFFCCF8AE036
:10AF40008093C600F894FFCF6C987498EAE6F0E01E
:10AF500080818160808380818D7F8083EC9A0895D9
:10AF60001F920F920FB60F9211240BB60F922F93D0
:10AF70003F934F935F936F937F938F939F93AF9381
:10AF8000BF93EF93FF93EC98E6E8F9E08491882370
:10AF900041F09091C00095FFFCCF8093C6003196A0
:10AFA000F5CF8091C00085FFFCCF8AE08093C6007A
:10AFB0008091060C8111FADDFF91EF91BF91AF9165
:10AFC0009F918F917F916F915F914F913F912F91C1
:10AFD0000F900BBE0F900FBE0F901F901895BF9251
:10AFE000CF92DF92EF92FF920F931F93CF93DF9355
:10AFF000CDB7DEB7E1970FB6F894DEBF0FBECDBF79
:10B0000088E89FE00F946ABCB82EBE01605D7F4F58
:10B0100089E89FE00F944A57EFE2F8E08491882393
:10B0200041F09091C00095FFFCCF8093C60031960F
:10B03000F5CF68A979A94AE050E08EE39AE00E9432
:10B04000EA358E01015E1F4F85E9E82E8FE0F82E6C
:10B05000D02EC12EC7010F946ABCF80181938F01D5
:10B06000FFEFEF1AFF0A8DE9E8168FE0F80691F777
:10B070001FA2ED2DFC2D8191882339F09091C00005
:10B0800095FFFCCF8093C600F6CF6AE278E08D2D65
:10B090009C2D0F9419B9CF92DF9283E298E09F9391
:10B0A0008F938E010F5F1F4F1F930F930F943EBA24
:10B0B0000F900F900F900F900F900F907E0195E0E2
:10B0C000E90EF11CF7018081882349F0992787FD5B
:10B0D00090950F9408B9F70181937F01F3CF60E059
:10B0E000C8010E9410B481E99FE00F9472BCF62E53
:10B0F000E72ED82EC92EE8E0F8E08491882341F0AD
:10B100009091C00095FFFCCF8093C6003196F5CF9B
:10B110002AE030E04F2D5E2D6D2D7C2D8EE39AE0E0
:10B120000E944C3661E084E098E00E9410B46FEF1A
:10B1300077E0C8010F9424B98DE99FE00F9472BCA9
:10B140006CA77DA78EA79FA7CE018C960F94995FC1
:10B15000BC01C8010F94B3B96CEF77E0C8010F943C
:10B1600019B981EA9FE00F9472BC6CA77DA78EA7E6
:10B170009FA7CE018C960F94995FBC01C8010F94D4
:10B18000B3B965EF77E0C8010F9419B960E0C80161
:10B190000E9410B460EF77E0C8010F9424B98DE8E5
:10B1A0009FE00F9472BC6CA77DA78EA79FA7CE01CE
:10B1B0008C960F94995FBC01C8010F94B3B960E0FD
:10B1C000C8010E9410B461E085EE97E00E9410B4BF
:10B1D00089A98F9388A98F938EED97E09F938F9382
:10B1E0001F930F930F943EBA60E0C8010E9410B401
:10B1F00067ED77E0C8010F9424B98B2D90E09DA7EF
:10B200008CA7CE018C960F94FB61BC01C8010F94F2
:10B21000B3B960E0C8010E9410B4CF92DF92EF9200
:10B22000FF928EEC97E09F938F931F930F930F9451
:10B230003EBA60E0C8010E9410B461E08AEC97E079
:10B240000E9410B40FB6F894DEBF0FBECDBFE196DA
:10B250000FB6F894DEBF0FBECDBFDF91CF911F9127
:10B260000F91FF90EF90DF90CF90BF9008954F9295
:10B270005F926F927F92AF92BF92CF92DF92EF92E6
:10B28000FF920F931F93CF93DF93CDB7DEB7E09775
:10B290000FB6F894DEBF0FBECDBF2B013C01690194
:10B2A0007A018091E00A8111E5C0F8940F946C1D39
:10B2B0008091BB109091BC10A091BD10B091BE10B8
:10B2C0008093DC0A9093DD0AA093DE0AB093DF0A34
:10B2D0000F948C1D4091DC0A5091DD0A6091DE0ACA
:10B2E0007091DF0A481B590B610971094093DC0A10
:10B2F0005093DD0A6093DE0A7093DF0A0E94F0BA71
:10B300004091DC0A5091DD0A6091DE0A7091DF0AFB
:10B31000481B590B610971094093DC0A5093DD0AFF
:10B320006093DE0A7093DF0A9091FD138091FC1305
:10B33000981799F0E091FC1387E5E89FF00111243C
:10B34000E250FC4E20E030E040E752E462A173A1FD
:10B3500084A195A10F94DDB308C060910C02709197
:10B360000D0280910E0290910F026093C80A7093B3
:10B37000C90A8093CA0A9093CB0A0F94360D80E1D4
:10B38000E5E8FBE0ACECBAE001900D928A95E1F7BC
:10B390008091710B8093C70A809107028093C60A3F
:10B3A0000E949AB31092060C81E08093E00A789490
:10B3B00020E030E0A901C301B2010F94DCB081119B
:10B3C0000AC020E030E0A901C701B6010F94DCB04B
:10B3D000882309F44FC065EC77E0FE0131965F01E8
:10B3E000CF010F9424B9F50101900020E9F78F01F6
:10B3F000015011092091D40A3091D50A4091D60A02
:10B400005091D70AC301B2010F94ECAF23E048E09A
:10B410000F9447B662EC77E0C5010F9419B9F501B6
:10B4200001900020E9F78F010150110923E046E067
:10B43000C701B6010F9447B66FEB77E0C5010F94D3
:10B4400019B9F50101900020E9F78F0101501109A8
:10B450006091510270915202809153029091540276
:10B4600023E048E00F9447B660E0C5010E9410B4A5
:10B470000E94A6B5E0960FB6F894DEBF0FBECDBF12
:10B48000DF91CF911F910F91FF90EF90DF90CF90C0
:10B49000BF90AF907F906F905F904F90089520E0A5
:10B4A00030E0A90160E070E080E291E4E0CE8F92AC
:10B4B0009F92AF92BF92CF92DF92EF92FF920F9343
:10B4C0001F93CF93DF9300D01F92CDB7DEB79B01C0
:10B4D000AC018091E00A882309F497C08091C70AE3
:10B4E0008093710B8091C80A9091C90AA091CA0AF1
:10B4F000B091CB0A80930C0290930D02A0930E02A0
:10B50000B0930F026091D80A7091D90A8091DA0A3B
:10B510009091DB0A0F94EBAF69837A838B839C83D2
:10B52000CE0101960F94FE1C20E030E040E551E48E
:10B530006091510270915202809153029091540295
:10B540000F94E3B04B015C01E090D40AF090D50A6F
:10B550000091D60A1091D70A2091D00A3091D10AD1
:10B560004091D20A5091D30A6091CC0A7091CD0AD1
:10B570008091CE0A9091CF0AE1E7FBE0FF93EF9331
:10B58000E8EDCE2EEAE0DE2E0F94B10E0F944728A0
:10B5900080E1ECECFAE0A5E8BBE001900D928A9521
:10B5A000E1F780E1E5E8FBE0A0E5BBE001900D926A
:10B5B0008A95E1F74091DC0A5091DD0A6091DE0A3C
:10B5C0007091DF0A4093A20E5093A30E6093A40ED5
:10B5D0007093A50E8DEE9DE00E94849B8091DC0A05
:10B5E0009091DD0AA091DE0AB091DF0A8093BB1032
:10B5F0009093BC10A093BD10B093BE1081E08093D7
:10B60000060C1092E00A0F900F900F900F900F9081
:10B610000F90DF91CF911F910F91FF90EF90DF90EE
:10B62000CF90BF90AF909F908F90089560E070E0B2
:10B63000CB013DCFEAEAF7E08491882341F0909175
:10B64000C00095FFFCCF8093C6003196F5CF4091A6
:10B65000850B5091860B6091870B7091880B23E0CE
:10B6600030E08EE39AE00E94E136E7EAF7E0849169
:10B67000882341F09091C00095FFFCCF8093C600D5
:10B680003196F5CF4091890B50918A0B60918B0BCD
:10B6900070918C0B23E030E08EE39AE00E94E1365B
:10B6A000E4EAF7E08491882341F09091C00095FF8F
:10B6B000FCCF8093C6003196F5CF40918D0B509111
:10B6C0008E0B60918F0B7091900B23E030E08EE336
:10B6D0009AE00E94E136E2EAF7E08491882341F0A3
:10B6E0009091C00095FFFCCF8093C6003196F5CFB6
:10B6F0008091C00085FFFCCF8AE08093C60008954A
:10B70000EAE8F7E08491882341F09091C00095FF2A
:10B71000FCCF8093C6003196F5CF0F94B628AB01CD
:10B72000BC0123E030E08EE39AE00E94E136E7E8D6
:10B73000F7E08491882341F09091C00095FFFCCF01
:10B740008093C6003196F5CF81E00F94B628AB0107
:10B75000BC0123E030E08EE39AE00E94E136E4E8A9
:10B76000F7E08491882341F09091C00095FFFCCFD1
:10B770008093C6003196F5CF82E00F94B628AB01D6
:10B78000BC0123E030E08EE39AE00E94E136E2E87B
:10B79000F7E08491882341F09091C00095FFFCCFA1
:10B7A0008093C6003196F5CF8091C00085FFFCCF15
:10B7B0008AE08093C6000895EF92FF920F931F9343
:10B7C000CF93DF93EEE6F7E08491882341F09091E8
:10B7D000C00095FFFCCF8093C6003196F5CF00E105
:10B7E00013E1FCE6EF2EF7E0FF2EC0E0D0E0F80119
:10B7F000EC0FFD1F418152816381748123E030E0B1
:10B800008EE39AE00E94E136F7018491ECE6F7E0DE
:10B81000882349F09091C00095FFFCCF8093C6002B
:10B8200031968491F5CF2496CC31D10501F7045E91
:10B830001F4FF3E1043D1F07C1F6EBE6F7E08491EB
:10B84000882341F09091C00095FFFCCF8093C60003
:10B850003196F5CF8091C00085FFFCCF8AE08093C0
:10B86000C600DF91CF911F910F91FF90EF90089547
:10B870002F923F924F925F926F927F928F929F9200
:10B88000AF92BF92CF92DF92EF92FF920F931F93EE
:10B89000CF93DF93CDB7DEB7C955D1090FB6F89472
:10B8A000DEBF0FBECDBF85E894E00E94A837882395
:10B8B000B1F08091D3109091D4106AE270E00596B7
:10B8C0000F94BEB9009711F0DC011C928091D31047
:10B8D0009091D41005960F9417580C94D98B8AE840
:10B8E00094E00E94A837882309F481C180E994E09C
:10B8F0000E94A837882391F080911B1C882311F4A3
:10B900000C94D98B0F94F6A76093000C7093010CE4
:10B910008093020C9093030C0C94D98B85E994E0EE
:10B920000E94A837882361F06091BF0B7091C00B13
:10B930004AE050E08EE39AE00E9440360C94D98BA6
:10B9400089E994E00E94A8378823C1F080911B1CEC
:10B95000882361F06091191C70911A1C4AE050E034
:10B960008EE39AE00E94EA350C94D98B6CE974E07E
:10B970008EE39AE00E94D6350C94D98B8EEA94E03F
:10B980000E94A837882379F16091D3107091D41068
:10B990006D5F7F4F21E041E084E09CE00E94D2ADEA
:10B9A0008091F50D9091F60DA091F70DB091F80DE5
:10B9B0008093A20E9093A30EA093A40EB093A50E15
:10B9C0008DEE9DE00E94BB9A2091C00025FFFCCF28
:10B9D0008093C6000A9721F760E084E09CE00E9413
:10B9E00062AD0C94D98B81EB94E00E94A837882338
:10B9F00099F00E94424481E08093C10B6091D31082
:10BA00007091D4106C5F7F4F21E040E084E09CE0B7
:10BA10000E94D2AD0C94D98B85EB94E00E94A8379C
:10BA2000882309F44FC080911B1C882309F49ECF02
:10BA30001092C40A1092C30AE8EBF4E081918823C3
:10BA400039F09091C00095FFFCCF8093C600F6CFEF
:10BA500000E010E0EE24E394F12C8091BF0A909175
:10BA6000C00A2091C10A3091C20A821B930B8F77C2
:10BA70009927892BA9F08EE39AE00E94F034F09286
:10BA8000C40AE092C30A9091C00095FFFCCF809356
:10BA9000C6000F5F1F4F1092C40A1092C30ADDCF79
:10BAA00003311105D4F281E090E09093C40A8093B1
:10BAB000C30A8091C00085FFFCCF8AE08093C60056
:10BAC0000C94D98B8BEB94E00E94A8378823A9F0C3
:10BAD000EFEBF4E08191882339F09091C00095FF5D
:10BAE000FCCF8093C600F6CF8091C00085FFFCCFCD
:10BAF0008AE08093C6000C94D98B8AEC94E00E9473
:10BB0000A8378823A9F0EEECF4E08191882339F07E
:10BB10009091C00095FFFCCF8093C600F6CF809136
:10BB2000C00085FFFCCF8AE08093C6000C94D98BBF
:10BB30008CEE94E00E94A837882321F00F94B5572B
:10BB40000C94D98B81EF94E00E94A837882341F0B0
:10BB500060E070E088EF9FE00F9439570C94D98B28
:10BB600084EF94E00E94A837882359F064EF74E0D2
:10BB70008EE39AE00E94D63540E052EC61E070E03E
:10BB800010C08FEF94E00E94A837882381F06FEFF8
:10BB900074E08EE39AE00E94D63540E054E961E11A
:10BBA00070E08EE39AE00E947A340C944E8D8BE024
:10BBB00095E00E94A837882361F00F94F6A7609360
:10BBC000EB0B7093EC0B8093ED0B9093EE0B0C94BE
:10BBD000D98B80E195E00E94A837882311F40C945A
:10BBE000D98B61E080E00E94213C0C94D98B8EE5DA
:10BBF0000E94923781110C94D98B87E40E9492376E
:10BC0000882311F40C945D6F0E94F2370F944BB1AE
:10BC10006C34710509F434C47CF56430710509F4A1
:10BC200009C154F46230710509F4ECC00CF0F6C09F
:10BC300077FF78C00C94D98B6C31710509F451C130
:10BC40007CF46A30710509F446C16B30710511F05E
:10BC50000C94D98B60E080E00E9428490C94D98B29
:10BC60006E31710509F451C36B34710511F00C94F8
:10BC7000D98B08E210E0FAC36735710511F40C9412
:10BC8000DD6E14F56035710511F40C9414676CF4D5
:10BC90006F34710511F00C94D98B0FEF10E0A1E90E
:10BCA000CA2EADE0DA2E0C9403676135710511F4EC
:10BCB0000C94246E6635710511F00C94D98B86EEC8
:10BCC0000E94D83B0C94D98B6C35710511F40C94FF
:10BCD000E66E7CF46A35710511F40C94E26E6B35F6
:10BCE000710511F00C94D98B81E080933B0B0C947F
:10BCF000D98B6236710511F40C94486F6336710567
:10BD000011F00C94D98B10921B1C0F94BA576091B0
:10BD10001B1C84EC9FE00F947CBC82E00F94A35921
:10BD20000C94D98B8091250B81110C94D98B0E9496
:10BD30005D456091BB0B7091BC0B8091BD0B9091E8
:10BD4000BE0B0F947CB14B015C01C090910BD09065
:10BD5000920BE090930BF090940B40905C0B509002
:10BD60005D0B60905E0B70905F0BA3019201C701A9
:10BD7000B6010F94EBAF20E030E048EC52E40F94B2
:10BD8000DDB39B01AC01C501B4010F940BB31816D0
:10BD9000E4F4A7019601C301B2010F94EBAF20E0D8
:10BDA00030E048EC52E40F94DDB39B01AC01C501D7
:10BDB000B4010F94ECAF0F9450B16093BB0B709330
:10BDC000BC0B8093BD0B9093BE0B80916E0B8823B0
:10BDD000A9F088E50E949237811110C089E50E9480
:10BDE000923781110BC08AE50E949237811106C0FB
:10BDF00085E40E94923781110C94DC8B0E942548C7
:10BE00000C94D98B8091250B81110C94D98B0E94B5
:10BE1000E04581E00E94034B0C94D98B8091250B67
:10BE200081110C94D98B0E94E04580E00E94034B65
:10BE30000C94D98B80E50E949237882339F00E94B8
:10BE4000F2370F9450B14B015C0103C0812C912C4F
:10BE5000540183E50E949237882361F00E94F237F3
:10BE600020E030E04AE754E40F94DDB30F9450B182
:10BE70004B015C0181149104A104B10431F0E6EEA0
:10BE8000F7E2859194910F9424580F9447280F94CA
:10BE9000F6A72B013C01480C591C6A1C7B1C0F9413
:10BEA000F6A76093370B7093380B8093390B909300
:10BEB0003A0B0F94F6A7641575058605970510F0E3
:10BEC0000C94D98B0F94DD3980E00E942A4C80E0DD
:10BED0000F94A359EECF60E081E00E9428490C94B2
:10BEE000D98B0F944728EFEBFEE08491882341F033
:10BEF0009091C00095FFFCCF8093C6003196F5CF9E
:10BF000099DBE1EBFEE08491882341F09091C00041
:10BF100095FFFCCF8093C6003196F5CFF1DB81E031
:10BF20008093F00B88E50E949237182F89E50E94D4
:10BF30009237082F8AE50E949237782E101308C096
:10BF4000181305C07724739401E011E001C0012F9C
:10BF50000E949DD9609010131092101382E00F94EC
:10BF6000B62860938D0B70938E0B80938F0B9093FC
:10BF7000900B71100F947F0240910C0250910D02B2
:10BF800060910E0270910F0240933C0B50933D0B59
:10BF900060933E0B70933F0B809147029091480253
:10BFA0009093FB0B8093FA0B84E690E09093480209
:10BFB000809347020F94F6A76093370B7093380B6A
:10BFC0008093390B90933A0B81E00F94D41E80E15B
:10BFD000E5E8FBE0A0E5BBE001900D928A95E1F772
:10BFE00010920C0210920D0210920E0210920F028B
:10BFF000112321F080E090E00E94E23F002321F035
:10C0000081E090E00E94E23F88E50E949237882319
:10C0100041F00E94BC37672B682B692B11F00C9400
:10C020000B8C89E50E949237882341F00E94BC372F
:10C03000672B682B692B11F00C94218C772009F465
:10C04000F1C08091760B882321F08091770B8111CC
:10C0500008C080E090E00E94E23F81E090E00E9412
:10C06000E23F0E94F2D9EFE3F3E385919591A59128
:10C07000B49189839A83AB83BC83EBE3F3E385912B
:10C080009591A591B4918F8F98A3A9A3BAA324E504
:10C090003BE040E55BE0BE016F5F7F4FCE014F9616
:10C0A0000E94F9390E9464D920E030E040E451EC6C
:10C0B0006091540B7091550B8091560B9091570BDA
:10C0C0000F94DCB087FF0CC080E090E0A0E4B1ECFE
:10C0D0008093540B9093550BA093560BB093570B32
:10C0E00080E090E0A0EAB0E48093580B9093590B65
:10C0F000A0935A0BB0935B0B20E030E040E251E498
:10C1000060915102709152028091530290915402B9
:10C110000F94E3B060930C0270930D0280930E02B3
:10C1200090930F0210928D0B10928E0B10928F0B2A
:10C130001092900B80E00F94D41EE0908D0BF09045
:10C140008E0B00918F0B1091900B2091890B3091E9
:10C150008A0B40918B0B50918C0B6091850B7091E9
:10C16000860B8091870B9091880BF1E9CF2EFBE035
:10C17000DF2E0F945F1B80900C0290900D02A09018
:10C180000E02B0900F02E090580BF090590B009106
:10C190005A0B10915B0B2091540B3091550B409131
:10C1A000560B5091570B6091500B7091510B809131
:10C1B000520B9091530BE1E7FBE0FF93EF93ACE55B
:10C1C000CA2EABE0DA2E0F94B10E0F94472880915F
:10C1D000500B9091510BA091520BB091530B809347
:10C1E000850B9093860BA093870BB093880B80915F
:10C1F000540B9091550BA091560BB091570B809317
:10C20000890B90938A0BA0938B0BB0938C0B81E0DE
:10C210000F94D41E0F94BC1E82E090E00E94E23F77
:10C220000F900F908AE50E949237882341F00E9478
:10C23000BC37672B682B692B11F00C94378CE0907E
:10C240008D0BF0908E0B00918F0B1091900B209125
:10C25000890B30918A0B40918B0B50918C0B609124
:10C26000850B7091860B8091870B9091880BE1E98B
:10C27000CE2EEBE0DE2E0F945F1B80E00F94D41ED9
:10C2800080913C0B90913D0BA0913E0BB0913F0BE8
:10C2900080930C0290930D02A0930E02B0930F02B4
:10C2A0008091FA0B9091FB0B909348028093470288
:10C2B0000F94F6A76093370B7093380B8093390B6C
:10C2C00090933A0B0F94BC1E0E94F2D90E940EDC90
:10C2D00088E50E94923781110C944D8C89E50E946B
:10C2E000923781110C944D8C87E50E949237811111
:10C2F0000C944D8C8AE50E94923781110C944D8CE0
:10C300000F9447281092F00B8FC50F94472881E0B7
:10C310000E943E378091510290915202A0915302A7
:10C32000B091540280930C0290930D02A0930E02E0
:10C33000B0930F0220E030E043E060E070E080E284
:10C3400091EC0E949DDCE4E3F8E285919491FC017C
:10C350002491222341F03091C00035FFFCCF20937F
:10C36000C6000196F4CFE8E8FEE08491882341F00E
:10C370009091C00095FFFCCF8093C6003196F5CF19
:10C380004091850B5091860B6091870B7091880BC3
:10C3900025E030E08EE39AE00E94E136E3E8FEE03B
:10C3A0008491882341F09091C00095FFFCCF809349
:10C3B000C6003196F5CF4091890B50918A0B609160
:10C3C0008B0B70918C0B25E030E08EE39AE00E949D
:10C3D000E136EEE7FEE08491882341F09091C000C1
:10C3E00095FFFCCF8093C6003196F5CF40918D0B21
:10C3F00050918E0B60918F0B7091900B25E030E087
:10C400008EE39AE00E94E136ECE7FEE08491882317
:10C4100041F09091C00095FFFCCF8093C60031960B
:10C42000F5CF0E946C370C94D98B9091C00095FF8A
:10C43000FCCF8093C60081918111F7CFB801882786
:10C4400077FD8095982F0F947EB10E940850AB0124
:10C45000BC0122E030E08EE39AE00E94E2360F5FFA
:10C460001F4F0F36110511F40C94D98B4AE050E0A0
:10C47000B8018EE39AE00E94E335E8EBF9E0DBCF08
:10C480008091760B882341F08091770B882321F0EF
:10C490008091780B811109C00E94A6B561E085E703
:10C4A0009EE00E94EEB40C94D98BE7E5FEE0849107
:10C4B000882341F09091C00095FFFCCF8093C60087
:10C4C0003196F5CF8091C00085FFFCCF8AE0809344
:10C4D000C6001A8219828090021B9090031BA090C4
:10C4E000041BB090051B20E030E040EA50E4C50199
:10C4F000B4010F94E3B00F944BB145E0469F900117
:10C50000479F300D1124B901882777FD8095982F1A
:10C510000F947EB12B013C0120E030E04CE052E46E
:10C520000F94DCB087FF06C0412C512C9CE0692E93
:10C5300092E4792EA5019401C301B2010F94DCB0FD
:10C5400087FF0AC020E030E040EA50E4C301B201B6
:10C550000F94ECAF2B013C01E3E4FEE084918823CF
:10C5600041F09091C00095FFFCCF8093C6003196BA
:10C57000F5CF22E030E0B301A2018EE39AE00E9401
:10C58000E23620E030E040EF51E4C301B2010F9405
:10C59000EBAF20E030E040E251E40F94DDB320E067
:10C5A00030E040EA50E40F94E3B020E030E048E4AB
:10C5B00052E40F94ECAF0F944BB170930F1B609348
:10C5C0000E1B84E090E09093B40B8093B30B81E05A
:10C5D00090E09093B20B8093B10BEAEAF6E285917A
:10C5E000949121E0892B09F420E02093B60B80E0A0
:10C5F00090E0ACE8B2E48093850B9093860BA09317
:10C60000870BB093880B80E090E0A0E4B0EC8093BF
:10C61000890B90938A0BA0938B0BB0938C0B80E0CB
:10C6200090E0A0E8BFE380938D0B90938E0BA093D6
:10C630008F0BB093900B81E79BE09F938F93812C9E
:10C64000912C18E4A12E12E4B12E01E9C02E0BE0CA
:10C65000D02EE12CF12C00E81FE320E030E040E494
:10C6600050EC60E070E08CE892E40F94B10E0F940F
:10C6700047280F900F90A30192016091021B7091C7
:10C68000031B8091041B9091051B0F94DCB087FF66
:10C6900007C088EE93E00E944B4E0E947E55EBCF80
:10C6A00060E086EA9FE00F947CBC80E090E0A0EA26
:10C6B000B0E480938D0B90938E0BA0938F0BB0936F
:10C6C000900B2091890B30918A0B40918B0B5091EC
:10C6D0008C0B6091850B7091860B8091870B9091EC
:10C6E000880BE1E7FBE0FF93EF93812C912CE8E4CA
:10C6F000AE2EE2E4BE2EF1E9CF2EFBE0DF2EE12CE0
:10C70000F12C00EA10E40F94B10EEBE3F3E3859112
:10C710009591A591B4918093850B9093860BA093EE
:10C72000870BB093880BEFE3F3E3259135914591A7
:10C7300054912093890B30938A0B40938B0B509329
:10C740008C0BE0908D0BF0908E0B00918F0B109165
:10C75000900B6091850B7091860B8091870B909167
:10C76000880BE1E7FBE0FF93EF93812C912CB8E479
:10C77000AB2EB2E4BB2E0F94B10E0F94472820E0ED
:10C7800030E043E060E070E080E89FEB0E949DDCD9
:10C7900080918D0B90918E0BA0918F0BB091900B8F
:10C7A00024968CAF9DAFAEAFBFAF2497E2E4FEE01E
:10C7B00084910F900F900F900F9040918D0B50919E
:10C7C0008E0B60918F0B7091900B882349F09091A4
:10C7D000C00095FFFCCF8093C60031968491F5CFC1
:10C7E0008091C00085FFFCCF8AE08093C600EBE318
:10C7F000FEE08491882341F09091C00095FFFCCF2A
:10C800008093C6003196F5CF22E030E08EE39AE0C7
:10C810000E94E136EAE3FEE08491882341F09091A2
:10C82000C00095FFFCCF8093C6003196F5CF809174
:10C83000C00085FFFCCF8AE08093C6002EEAA22EBE
:10C840002FE0B22E33E2E32EF12C0FEF1FEF4AE080
:10C85000D42E53E0252E5EE0352E62E0862E6EE06B
:10C86000962EB701882777FD8095982F0F947EB17B
:10C8700068AF79AF8AAF9BAFE3E3FEE08491882392
:10C8800041F09091C00095FFFCCF8093C600319697
:10C89000F5CF4AE050E0B8016E5F7F4F8EE39AE03B
:10C8A0000E94E335E6E2FEE08491882341F0909116
:10C8B000C00095FFFCCF8093C6003196F5CF8091E4
:10C8C000C00085FFFCCFD092C600E2E1FEE084917B
:10C8D000882341F09091C00095FFFCCF8093C60063
:10C8E0003196F5CF4AE050E0B7018EE39AE00E941E
:10C8F000E335F1018491E3E0FEE0882349F0909173
:10C90000C00095FFFCCF8093C60031968491F5CF8F
:10C910004AE050E060E070E08EE39AE00E94E33588
:10C92000F4018491E2E0FEE0882349F09091C00098
:10C9300095FFFCCF8093C60031968491F5CF80910E
:10C94000C00085FFFCCFD092C6000F3FFFEF1F074E
:10C9500031F0BE016F5F7F4FC5010F94395728AD8D
:10C9600039AD4AAD5BADC301B2010F94DCB018160E
:10C9700064F40F5F1F4F25E0E20EF11C32E0A30EBE
:10C98000B11C0530110509F06CCF280187E2481A67
:10C9900088EF580A440C551C380193E0690E711C4D
:10C9A00085E0809F1001819F300C112419AE18AED4
:10C9B000ADE22A0E311CC301029705970CF0C7C1E6
:10C9C00068AD79AD620D731D882777FD8095982F2E
:10C9D0000F947EB16CAF7DAF8EAF9FAFEBEFFDE0FC
:10C9E0008491882341F09091C00095FFFCCF809303
:10C9F000C6003196F5CF4AE050E0B3018EE39AE0ED
:10CA00000E94E335E8EFFDE08491882341F09091A6
:10CA1000C00095FFFCCF8093C6003196F5CF809182
:10CA2000C00085FFFCCFFAE0F093C6007092B20B15
:10CA30006092B10B20E030E040EF51E46CAD7DAD91
:10CA40008EAD9FAD0F94EBAF20E030E040E251E4BB
:10CA50000F94DDB320E030E040EA50E40F94E3B0FF
:10CA600020E030E048E452E40F94ECAF0F944BB177
:10CA700070930F1B60930E1B80E090E0ACE8B2E473
:10CA80008093850B9093860BA093870BB093880BB4
:10CA900080E090E0A0E4B0EC8093890B90938A0B47
:10CAA000A0938B0BB0938C0B80E090E0A0E8BFE3E9
:10CAB00080938D0B90938E0BA0938F0BB093900B64
:10CAC000A1E7BBE0BF93AF93812C912CA8E4AA2EE1
:10CAD000A2E4BA2EB1E9CB2EBBE0DB2EE12CF12C87
:10CAE00000E81FE320E030E040E450EC60E070E05C
:10CAF0008CE892E40F94B10E0F9447280F900F909A
:10CB00002CAD3DAD4EAD5FAD6091021B7091031B2E
:10CB10008091041B9091051B0F94DCB087FF07C028
:10CB200088EE93E00E944B4E0E947E55E9CF80E054
:10CB300090E0A0EAB0E480938D0B90938E0BA093CD
:10CB40008F0BB093900B2091890B30918A0B409101
:10CB50008B0B50918C0B6091850B7091860B8091A3
:10CB6000870B9091880BA1E7BBE0BF93AF93812C1B
:10CB7000912CB8E4AB2EB2E4BB2E11E9C12E1BE020
:10CB8000D12EE12CF12C00EA10E40F94B10EEBE36E
:10CB9000F3E385919591A591B4918093850B909342
:10CBA000860BA093870BB093880BEFE3F3E32591FB
:10CBB0003591459154912093890B30938A0B409382
:10CBC0008B0B50938C0BE0908D0BF0908E0B0091A3
:10CBD0008F0B1091900B6091850B7091860B80915B
:10CBE000870B9091880BA1E7BBE0BF93AF93812C9B
:10CBF000912CF8E4AF2EF2E4BF2E0F94B10E0F94F7
:10CC0000472820E030E043E060E070E080E89FEB00
:10CC10000E949DDC24962CAD3DAD4EAD5FAD2497BA
:10CC200060918D0B70918E0B80918F0B9091900B7A
:10CC30000F94EBAF2091E1193091E2194091E31983
:10CC40005091E4190F94DDB30F944BB17A8369834B
:10CC5000E7EFFDE084910F900F900F900F908823E5
:10CC600049F09091C00095FFFCCF8093C6003196AB
:10CC70008491F5CF8091C00085FFFCCFFAE0F0935E
:10CC8000C600E3EEFDE08491882341F09091C0005E
:10CC900095FFFCCF8093C6003196F5CF4091021BE3
:10CCA0005091031B6091041B7091051B22E030E042
:10CCB0008EE39AE00E94E136E4EDFDE08491882362
:10CCC00041F09091C00095FFFCCF8093C600319653
:10CCD000F5CF24962CAD3DAD4EAD5FAD2497609160
:10CCE0008D0B70918E0B80918F0B9091900B0F9408
:10CCF000EBAFAB01BC0122E030E08EE39AE00E9492
:10CD0000E136E3EDFDE08491882341F09091C0008D
:10CD100095FFFCCF8093C6003196F5CF8091C0007F
:10CD200085FFFCCFFAE0F093C600BE016F5F7F4F36
:10CD3000C2010F94395722E0420E511C3FEF631A93
:10CD4000730A88AD99AD059699AF88AF34CE10922D
:10CD5000B40B1092B30B1092B60B61E086EA9FE021
:10CD60000F947CBCE4E9FDE08491882341F090912C
:10CD7000C00095FFFCCF8093C6003196F5CF80911F
:10CD8000C00085FFFCCF8AE08093C600179A1092FE
:10CD9000760B169A1092770B149AE8EAF6E28591D0
:10CDA00094910F94185D81E00F94105B82E00F94D2
:10CDB000A35910920F1B10920E1B0C94D98B84E672
:10CDC00090E00E944B4E91E0E91AF108C1F74AE069
:10CDD00050E0B8018EE39AE00E94E335F601249119
:10CDE000E1E9FDE0211117C06091980B7091990B5A
:10CDF0004AE050E08EE39AE00E94EA3505501109BE
:10CE000011F40C94D98B1093700B00936F0BF4E614
:10CE1000EF2EF12CD4CF3091C00035FFFCCF209302
:10CE2000C60031962491DECF81E08093C40B86E565
:10CE30000E9492378823A1F08091D3109091D41052
:10CE4000DC0111962C91293069F02F7D71F04AE0B8
:10CE500050E060E070E001960F94CFB768AF07C074
:10CE600018AE05C0B1E0B8AF02C0E1E0E8AF209174
:10CE7000760B80911F1C9091201C222341F0209161
:10CE8000770B222321F02091780B21110FC00297FC
:10CE900049F00E94A6B561E08AE89DE00E94EEB4E8
:10CEA0000C94D98B1092C40B0C94D98B1092C50A98
:10CEB000029721F41092C40B0C94D98BF091B60B0D
:10CEC0002E96FFAF2E972091B30B3091B40B609646
:10CED0003FAF2EAF60978091B10B9091B20B6296ED
:10CEE0009FAF8EAF629781E08093B60B81E090E0B8
:10CEF0009093B40B8093B30B83E190E09093B20BCB
:10CF00008093B10B81E00F94A35980E193E10F94DA
:10CF10004C030F947F0280E090E0A0EAB0E480939D
:10CF20008D0B90938E0BA0938F0BB093900B20E002
:10CF300030E040E752E460915102709152028091DA
:10CF40005302909154020F94E3B04B015C01209185
:10CF5000890B30918A0B40918B0B50918C0B609117
:10CF6000850B7091860B8091870B9091880BE1E780
:10CF7000FBE0FF93EF9311E9C12E1BE0D12EE12CD2
:10CF8000F12C00EA10E40F94B10EEBE3F3E385918A
:10CF90009591A591B4918093850B9093860BA09366
:10CFA000870BB093880BEFE3F3E385919591A591FF
:10CFB000B4918093890B90938A0BA0938B0BB093C1
:10CFC0008C0B69E87BE085E89BE00E94B33A2996E8
:10CFD0008FAF29970F900F9098AD19160CF45FC082
:10CFE00020E030E040EF51E46091490270914A0244
:10CFF00080914B0290914C020F94E3B04B015C0185
:10D00000E0908D0BF0908E0B00918F0B1091900B98
:10D010002091890B30918A0B40918B0B50918C0B96
:10D020006091850B7091860B8091870B9091880B96
:10D03000E1E7FBE0FF93EF93B1E9CB2EBBE0DB2E02
:10D040000F94B10E0F94472820E030E040EA51E4FD
:10D050006091490270914A0280914B0290914C027A
:10D060000F94E3B00F944BB18B0120E030E040E22D
:10D0700052E460915102709152028091530290915A
:10D0800054020F94E3B00F944BB17B010E9450D92E
:10D090008CAF0F900F90A8AD1A1614F129C02996E5
:10D0A000BFAD2997BB2371F0E8E6FDE084918823AA
:10D0B00009F496CF9091C00095FFFCCF8093C600F5
:10D0C0003196F4CFEEE3FDE08491882309F488CF14
:10D0D0009091C00095FFFCCF8093C6003196F4CFAD
:10D0E0009CAD992379F1ECE1FDE08491811122C09E
:10D0F00080E00E943E37EBE3F3E32696FFAFEEAF0E
:10D100002697212C312CC701AA2797FDA095BA2F6D
:10D1100066968CAF9DAFAEAFBFAF6697C801AA272A
:10D1200097FDA095BA2F6A968CAF9DAFAEAFBFAFFB
:10D130006A9715C09091C00095FFFCCF8093C60000
:10D140003196D3CFE6EFFCE08491882389F2909169
:10D15000C00095FFFCCF8093C6003196F5CFA8ADF7
:10D160001A16A4F4E5EFFCE08491882341F0909135
:10D17000C00095FFFCCF8093C6003196F5CF80911B
:10D18000C00085FFFCCF8AE08093C600C10163E048
:10D1900070E00F94BBB528967FAF6EAF28972296AC
:10D1A0009FAF8EAF22972796FFAD2797F0FF08C05D
:10D1B00022E030E0281B390B22963FAF2EAF22979A
:10D1C0003CAD332309F477C02114310409F473C052
:10D1D00028968EAD9FAD2897880F991F2896AEADE3
:10D1E000BFAD28978A0F9B1F2296EEADFFAD229709
:10D1F0008E0F9F1F880F991F8D53904F0F9477BCF0
:10D20000BC01882777FD8095982F0F947EB12AE086
:10D2100037ED43E25CE30F94DDB3209111133091BD
:10D22000121340911313509114130F94ECAF2B0170
:10D230003C01F8AD1F160CF041C0EFEDFCE084910D
:10D24000882341F09091C00095FFFCCF8093C600E9
:10D250003196F5CF4AE050E0B1018EE39AE00E94AA
:10D26000E335EDECFCE08491882341F09091C0001F
:10D2700095FFFCCF8093C6003196F5CF25E030E0D6
:10D28000B301A2018EE39AE00E94E136ECECFCE0EF
:10D290008491882341F09091C00095FFFCCF80934A
:10D2A000C6003196F5CF8091C00085FFFCCF8AE0A3
:10D2B0008093C60003C0412C512C320180E090E0E5
:10D2C000A0EAB0E480938D0B90938E0BA0938F0B0C
:10D2D000B093900B66966CAD7DAD8EAD9FAD6697AD
:10D2E0000F947EB12D966CAF7DAF8EAF9FAF2D9713
:10D2F0002091890B30918A0B40918B0B50918C0BB4
:10D300006091850B7091860B8091870B9091880BB3
:10D31000A1E7BBE0BF93AF932D968CAC9DACAEACB8
:10D32000BFAC2D97B1E9CB2EBBE0DB2EE12CF12C6D
:10D3300000EA10E40F94B10E0F9447282696EEAD44
:10D34000FFAD269785919591A591B4918093850B1A
:10D350009093860BA093870BB093880B2696EEAD27
:10D36000FFAD2697349685919591A591B4918093C0
:10D37000890B90938A0BA0938B0BB0938C0B69E86D
:10D380007BE085E89BE00E94B33A0F900F90F8ADE8
:10D390001F16A4F16A966CAD7DAD8EAD9FAD6A97F8
:10D3A0000F947EB14B015C01E0908D0BF0908E0BE1
:10D3B00000918F0B1091900B2091890B30918A0B6B
:10D3C00040918B0B50918C0B6091850B7091860B6B
:10D3D0008091870B9091880BA1E7BBE0BF93AF933F
:10D3E000A1E9CA2EABE0DA2E0F94B10E0F944728B4
:10D3F0000F900F90FCADF11129C034C04AE050E00D
:10D40000B1018EE39AE00E94E33529962FAD29976A
:10D41000222371F0EDEBFCE08491882309F4BACF6C
:10D420009091C00095FFFCCF8093C6003196F4CF59
:10D43000EBEAFCE08491882309F4ACCF9091C00022
:10D4400095FFFCCF8093C6003196F4CF21143104B0
:10D4500049F020E030E040E85FE3C301B2010F94FF
:10D46000EBAF04C060E070E080E291EC20E030E0DF
:10D4700043E00E949DDC811103C0E0E2F8E21AC0A3
:10D4800080908D0B90908E0BA0908F0BB090900B96
:10D49000A501940160E070E080EA90E40F94EBAFA6
:10D4A0002DEC3CEC4CEC5DE30F94DCB087FF05C049
:10D4B000EEE1F8E26590749004C1FCADFF2391F0B9
:10D4C000A5019401C301B2010F94EBAF9F7720E057
:10D4D00030E040E85FE30F940BB318161CF4E2E26F
:10D4E000F8E2E8CF28AD2A305CF40E94EF534B01FC
:10D4F0005C0138AD13160CF09CC0ECE8FCE05FC09A
:10D50000E7EAFCE08491882341F09091C00095FF08
:10D51000FCCF8093C6003196F5CF4091850B50919A
:10D52000860B6091870B7091880B25E030E08EE3CD
:10D530009AE00E94E136E6EAFCE08491882341F01B
:10D540009091C00095FFFCCF8093C6003196F5CF37
:10D550008091C00085FFFCCF8AE08093C600E2EA9C
:10D56000FCE08491882341F09091C00095FFFCCFAE
:10D570008093C6003196F5CF4091890B50918A0B6C
:10D5800060918B0B70918C0B25E030E08EE39AE07C
:10D590000E94E136E0EAFCE08491882309F4A5CFFB
:10D5A0009091C00095FFFCCF8093C6003196F4CFD8
:10D5B0009091C00095FFFCCF8093C6003196849176
:10D5C0008111F6CF40918D0B50918E0B60918F0B96
:10D5D0007091900B25E030E08EE39AE00E94E136F6
:10D5E000E2E8FCE08491882341F09091C00095FF2F
:10D5F000FCCF8093C6003196F5CF25E030E0B50131
:10D60000A4018EE39AE00E94E136E1E8FCE0849117
:10D61000882341F09091C00095FFFCCF8093C60015
:10D620003196F5CF8091C00085FFFCCF8AE08093D2
:10D63000C60087E02896AEADBFAD28978A9F8001CF
:10D640008B9F100D11242296EEADFFAD22970E0F89
:10D650001F1F000F111F000F111F005F1C4EA5019F
:10D66000940160918D0B70918E0B80918F0B909136
:10D67000900B0F94EBAFD80111966D937D938D9322
:10D680009C9314978091B10B9091B20B019790935A
:10D69000B20B8093B10BBFEF2B1A3B0A81E00F94C2
:10D6A000A3592696EEADFFAD269738962696FFAF86
:10D6B000EEAF2697F9E02F16310409F050CD612C1A
:10D6C000712C28AD2431A4F0EAE5FCE08491882394
:10D6D00041F09091C00095FFFCCF8093C600319639
:10D6E000F5CF8091C00085FFFCCF8AE08093C60013
:10D6F00080E090E0A0EAB0E480938D0B90938E0BD5
:10D70000A0938F0BB093900B38AD343114F1E5E456
:10D71000FCE08491882341F09091C00095FFFCCFFC
:10D720008093C6003196F5CF8091C00085FFFCCF75
:10D730008AE08093C60040918D0B50918E0B6091D2
:10D740008F0B7091900B25E030E08EE39AE00E9401
:10D75000E136E0908D0BF0908E0B00918F0B1091C5
:10D76000900B2091890B30918A0B40918B0B50913B
:10D770008C0B6091850B7091860B8091870B90913B
:10D78000880BE1E7FBE0FF93EF932D968CAC9DAC0B
:10D79000AEACBFAC2D97E1E9CE2EEBE0DE2E0F94C0
:10D7A000B10E0F9447280F900F9089E0281631048E
:10D7B00021F060E0C3010C9462760E946C37E2E3D2
:10D7C000FCE08491882341F09091C00095FFFCCF4C
:10D7D0008093C6003196F5CF8091C00085FFFCCFC5
:10D7E0008AE08093C6000F946702E1E2FCE0849136
:10D7F000882341F09091C00095FFFCCF8093C60034
:10D800003196F5CF8091C00085FFFCCF8AE08093F0
:10D81000C60080EC9FE00F946ABCEE24E394813054
:10D8200009F0E12C98AD19164CF0DE0111966D014E
:10D83000F12C2CE4622E36E4732E1CC0EE2069F02D
:10D84000E6E0FCE08491882381F39091C00095FF8D
:10D85000FCCF8093C6003196F5CFE7EEFBE08491D4
:10D86000882319F39091C00095FFFCCF8093C600E8
:10D870003196F5CF6982B2E5BA837B8282E48C83EC
:10D88000F60181916F010E949237882319F00E945E
:10D89000BC371EC0EE2009F436C1F1E0FF1528F0B8
:10D8A000F11009C08FEB9FE00BC022E0F21206C01E
:10D8B0008DEB9FE005C08EEB9FE002C08CEB9FE0FC
:10D8C0000F946ABC682F772767FD7095872F972F75
:10D8D000611571058105910509F415C10F947EB19B
:10D8E0002FE632E143E85AE30F94DDB34B015C01CC
:10D8F0009F7727E139ED4EEC5DE30F940BB31816DB
:10D900000CF037C0E3E4F0E18491882341F090917A
:10D91000C00095FFFCCF8093C6003196F5CFE3ECB5
:10D92000FBE08491882341F09091C00095FFFCCFEB
:10D930008093C6003196F5CF22E030E0B501A40116
:10D940008EE39AE00E94E136EAEBFBE084918823C3
:10D9500041F09091C00095FFFCCF8093C6003196B6
:10D96000F5CF8091C00085FFFCCF8AE08093C60090
:10D97000CAC0F2E0FF1609F469C023E0F21609F408
:10D9800094C031E0F31689F120E030E040E05FE33D
:10D99000C501B4010F94DDB31B012C0101E113E1BA
:10D9A000A2019101D80114966D917D918D919C9168
:10D9B00017970F94ECAFF801648375838683978380
:10D9C000A501940160817181828193810F94ECAFF4
:10D9D000D8016D937D938D939C931397045E1F4F95
:10D9E000B3E105361B07E1F68EC020E030E040E0F1
:10D9F0005FE3C501B4010F94DDB31B012C0105E108
:10DA000013E1A2019101F80160817181828193810A
:10DA10000F94ECAFD8016D937D938D939C931397E6
:10DA2000A501940114966D917D918D919C9117970C
:10DA30000F94ECAFF8016483758386839783045E4B
:10DA40001F4FF3E109361F07E1F65DC020E030E02B
:10DA500040E05FE3C501B4010F94DDB31B012C016D
:10DA600001E113E1A2019101D8015C966D917D91D4
:10DA70008D919C915F970F94ECAFF801648F758F37
:10DA8000868F978FA5019401608171818281938136
:10DA90000F94ECAFD8016D937D938D939D938D0181
:10DAA000B3E10D311B07F1F62EC020E030E040E07D
:10DAB0005FE3C501B4010F94DDB31B012C010DE23E
:10DAC00013E1A2019101F80160817181828193814A
:10DAD0000F94ECAFD8016D937D938D939D938D0141
:10DAE000A501940158966D917D918D919C915B97C4
:10DAF0000F94ECAFF801608F718F828F938FF3E1F9
:10DB000009331F07F1F6F39424E0F212B3CEE9E9EA
:10DB1000FBE08491882341F09091C00095FFFCCFF9
:10DB20008093C6003196F5CF8091C00085FFFCCF71
:10DB30008AE08093C60080E193E10F946703E7E8F1
:10DB4000FBE08491882341F09091C00095FFFCCFC9
:10DB50008093C6003196F5CF8091C00085FFFCCF41
:10DB60008AE08093C60081E080931013EBE6FBE02F
:10DB70008491882341F09091C00095FFFCCF809361
:10DB8000C6003196F5CF8091C00085FFFCCF8AE0BA
:10DB90008093C6000E9454F8EAE5FBE08491882354
:10DBA00041F09091C00095FFFCCF8093C600319664
:10DBB000F5CF8091C00085FFFCCF8AE08093C6003E
:10DBC000E091710B34E0E39FF0011124E85FF44E23
:10DBD00020E030E042E053E46081718182819381F2
:10DBE0000F940BB3181694F48091EF0B882371F007
:10DBF00086EA9FE00F946ABC882341F080910E1B57
:10DC000090910F1BC29714F00C94AF8C2E968FAD91
:10DC10002E978093B60B6096AEADBFAD6097B09374
:10DC2000B40BA093B30B6296EEADFFAD6297F09389
:10DC3000B20BE093B10B1092C40B1092C30B82E0B5
:10DC40000F94A3590C94D98B80911013882309F455
:10DC50009EC0E0E5FBE08491882341F09091C000F4
:10DC600095FFFCCF8093C6003196F5CF4AE050E097
:10DC700067E070E08EE39AE00E94E335EEE4FBE0BB
:10DC80008491882341F09091C00095FFFCCF809350
:10DC9000C6003196F5CF4AE050E067E070E08EE3D1
:10DCA0009AE00E94E335EBE3FBE08491882341F0A6
:10DCB0009091C00095FFFCCF8093C6003196F5CFC0
:10DCC0004AE050E065E070E08EE39AE00E94E335C0
:10DCD000E9E2FBE08491882341F09091C00095FF38
:10DCE000FCCF8093C6003196F5CF8091C00085FFB0
:10DCF000FCCF8AE08093C60000E010E086E2A82E08
:10DD00008BE0B82E94E2892E9BE0992EE12CF12C29
:10DD1000980128543C4E6901F5018491E6E2FBE04C
:10DD2000882349F09091C00095FFFCCF8093C600F6
:10DD300031968491F5CFF601EE0DFF1D41815281A0
:10DD40006381748125E030E08EE39AE00E94E13641
:10DD5000F4E0EF0EF11C2CE1E216F104E9F6F40117
:10DD60008491E4E2FBE0882349F09091C00095FFA4
:10DD7000FCCF8093C60031968491F5CF0C511109E8
:10DD80000C33FFEF1F0709F0C1CF0C94D98BE6E0ED
:10DD9000FBE08491882341F09091C00095FFFCCF77
:10DDA0008093C6003196F5CF8091C00085FFFCCFEF
:10DDB0008AE08093C6000C94D98B81E00E94D83B06
:10DDC0000C94D98B10923B0B0C94D98B85E40E9458
:10DDD0009237811102C00F944728B3E76B2EB6E04B
:10DDE0007B2E19E7812E1BE0912E05E8A02E0BE07B
:10DDF000B02E512CD3018D913D010E949237882382
:10DE0000D9F1B3E05B120CC00E94F237F5016083D8
:10DE100071838283938381E99BE00F94FE1C2CC065
:10DE20000E94F237D4012D913D914D915C910F9458
:10DE3000ECAFF5016083718382839383E0908D0B57
:10DE4000F0908E0B00918F0B1091900B2091890B0D
:10DE500030918A0B40918B0B50918C0B6091850B0C
:10DE60007091860B8091870B9091880BA1E9CA2E47
:10DE7000ABE0DA2E0F945F1B5394F4E08F0E911CED
:10DE800024E0A20EB11C34E05312B4CF0C94D98B11
:10DE900081E080931B1C0F94F6A76093000C709395
:10DEA000010C8093020C9093030C60911B1C84EC7A
:10DEB0009FE00F947CBC0C94D98B8DE40E94923728
:10DEC000882311F40C94BB89E091D310F091D41005
:10DED000319681918032E9F38930D9F380538A30C9
:10DEE000B0F0E7EFFAE08491882341F09091C00010
:10DEF00095FFFCCF8093C6003196F5CF8091C0008E
:10DF000085FFFCCF8AE08093C6000C94D98B0E94D9
:10DF1000F2370F944BB16B3C710511F40C94D87D22
:10DF20000CF021C16F32710509F4AAC60CF06AC069
:10DF30006931710509F451C3B4F56431710509F40F
:10DF4000F1C294F46131710509F4E0C234F4623035
:10DF5000710508F434C20C94A6896231710511F47C
:10DF60000C94AF790C94A6896631710509F414C339
:10DF70000CF40CC36731710509F414C368317105E1
:10DF800011F00C94A68984E09CE00E942AA90F94C9
:10DF9000F6A760932F0B7093300B8093310B909307
:10DFA000320B0C94D98B6E31710509F45FC38CF47C
:10DFB0006B31710509F425C30CF415C36C3171057F
:10DFC00009F425C36D31710511F40C94D98B0C94AF
:10DFD000A6896A32710509F477C454F46F3171056A
:10DFE00009F412C46032710509F478C30C94A6894F
:10DFF0006C32710509F4AFC46D32710509F4BAC40D
:10E000000C94A6896D36710509F4B2C70CF064C092
:10E010006535710511F40C94E8790CF03DC062355A
:10E02000710511F40C94A6795CF56135710511F058
:10E030000C94A6890F9477320F944728149A0F9462
:10E04000C9281092700B10926F0B68EE73E080E09D
:10E0500090E00F9425A810921002E2E5F7E24591B6
:10E06000549122EB3AE060EB7AE083E195E00E9484
:10E0700095BD0F94245880E00F94A3590C94D98B2C
:10E080006335710511F40C94AA796435710511F4A6
:10E090000C94AF790C94A6896936710509F425C6EC
:10E0A0005CF46C35710511F40C94037A68367105D3
:10E0B00009F4EAC50C94A6896A36710511F40C942A
:10E0C00076796B36710511F00C94A6891092700B5D
:10E0D00010926F0B0C94D98B6837710511F40C9466
:10E0E000CE7BFCF46237710511F40C94C67A4CF4C3
:10E0F0006037710511F00C94A68963E083EF98E016
:10E10000E1C56337710511F40C94867A67377105A0
:10E1100011F00C94A689EEE7F7E2859194910C94A6
:10E12000DF7B6E3B710509F4B9C75CF46937710593
:10E1300011F40C94D37B6C38710509F4C5C50C94AB
:10E14000A689683C710511F40C94467D693C710503
:10E1500011F00C94A68903E716E069ECE62E69E15C
:10E16000F62E0C94BD7D673F81E0780711F40C9486
:10E1700003820CF07EC06C32A1E07A0711F40C949B
:10E180000880C4F5603D710511F40C94E27EA4F49E
:10E190006D3C710511F40C94177E14F40C94F57D0C
:10E1A0006E3C710511F40C948E7E6F3C710511F478
:10E1B0000C94AB7E0C94A6896D3D710511F40C9402
:10E1C0007C7F64F4613D710511F40C940A7F6C3D11
:10E1D000710511F40C946B7F0C94A689623E710555
:10E1E00011F40C94A67F603F710511F40C94D98B47
:10E1F0000C94A6896036E1E07E07E4F46E35F1E028
:10E200007F0714F00C94D98B6E3221E0720711F461
:10E210000C94AD8114F40C9440806F3281E0780747
:10E2200011F40C94BC816033714011F40C940B8197
:10E230000C94A689643FA1E07A0711F40C94F5814F
:10E240004CF46039714011F00C94A6890F94472862
:10E250000C94D98B653FF1E07F0711F40C94FC819D
:10E26000663F714011F00C94A6890E94982A0C9484
:10E27000D98B6E3833E0730711F40C94E7860CF0F9
:10E2800047C06D3B92E0790711F40C943888FCF498
:10E290006835B2E07B0711F40C9417835CF46D3F92
:10E2A000714011F00C94A6890F94B557EDE3F0E19D
:10E2B0000C940F82693522E0720711F40C94A28647
:10E2C0006A35724011F40C94B0860C94A6896438B7
:10E2D00083E0780711F40C94BE866CF46E3BA2E0E8
:10E2E0007A0711F40C9448896335734011F40C9447
:10E2F00021820C94A6896B38E3E07E0711F40C941C
:10E30000C1866C38734011F40C94D98B0C94A68997
:10E31000633923E0720711F40C945187D4F4603907
:10E3200083E0780711F40C941C8714F40C94EA86AB
:10E330006139A3E07A0711F40C944E876239734077
:10E3400011F00C94A68910927B1B0F945A450C94E3
:10E35000D98B6639E3E07E0711F40C9406886CF4DF
:10E36000643923E0720711F40C94578765397340C0
:10E3700011F40C94D4870C94A689603A83E0780752
:10E3800009F415C2673E734011F00C94A6891092EF
:10E39000250B0F9450588091BF109091C010A09100
:10E3A000C110B091C2108093C3109093C410A09379
:10E3B000C510B093C6100E942F450C94D98B0091C4
:10E3C000D3101091D4100E5F1F4F80E50E9492373A
:10E3D000882379F00E94F2370F9450B14B015C0111
:10E3E000FF24F394611571058105910531F4F12C39
:10E3F00004C0F12C812C912C540183E50E949237AA
:10E40000882399F00E94F23720E030E04AE754E494
:10E410000F94DDB30F9450B14B015C01EE24E394F3
:10E42000611571058105910509F4E12C6AE270E03E
:10E43000C8010F94BEB9009711F0DC011C92F801DD
:10E44000CF0121912032E1F3F11007C0E11005C0A6
:10E45000222319F00F94175806C0E4E9F6E28591DB
:10E4600094910F94245881E00F94F7570F94472804
:10E470000F94F6A76093370B7093380B8093390B8A
:10E4800090933A0B81149104A104B104A9F00F9464
:10E49000F6A72B013C01480C591C6A1C7B1C0F94ED
:10E4A000F6A76415750586059705C8F40F942B5CCF
:10E4B000811115C00C94F18C0F94295C882311F400
:10E4C0000C94D98B0F942B5C81110CC00F94DD3907
:10E4D00081E00E942A4C80E00F94A359F3CF80E0A2
:10E4E0000F94F7578091060C882341F0E2E2F7E29F
:10E4F000859194910F9424580C94D98BECE7F6E213
:10E50000859194910F9424580C94D98BE4E5F7E20B
:10E51000859194910F9424581798169815981498EB
:10E520000C94D98BEAE0F8E285919491FC01249156
:10E53000222341F03091C00035FFFCCF2093C6006C
:10E540000196F4CF8091C00085FFFCCF8AE08093D4
:10E55000C60084E09CE00E94FBA7EEEDF7E2859107
:10E560009491FC012491222341F03091C00035FFA9
:10E57000FCCF2093C6000196F4CF8091C00085FFA8
:10E58000FCCF8AE08093C6000C94D98B84E09CE099
:10E590000E9451A80C94D98B84E09CE00E9426A98B
:10E5A0000C94D98B8091D3109091D4106AE270E0D2
:10E5B00004960F94BEB9009711F0DC011C92609193
:10E5C000D3107091D4106C5F7F4F21E041E084E064
:10E5D0009CE00E94D2AD0C94D98B84E09CE00E9418
:10E5E00031A90C94D98B8091070C882311F40C94D9
:10E5F000D98B83E50E94923781110C94FB8C0C948B
:10E60000D98B84E09CE00E94D6AA0C94D98B80918F
:10E61000D3109091D4106AE270E004960F94BEB9C2
:10E620008C010097A9F08091DD109091DE106EE4CE
:10E6300070E08E519F4E0F94BEB960E270E00F946F
:10E64000BEB901969093D4108093D310F801108234
:10E650006091D3107091D4106C5F7F4F21E040E047
:10E6600084E09CE00E94D2AD0C94D98B8091070C81
:10E67000882311F40C94D98B60E084E09CE00E9424
:10E6800062AD8091D3109091D4106AE270E004964C
:10E690000F94BEB98C010097A9F08091DD10909184
:10E6A000DE106EE470E08E519F4E0F94BEB960E2B2
:10E6B00070E00F94BEB901969093D4108093D3105C
:10E6C000D8011C926091D3107091D4106C5F7F4F71
:10E6D00084E09CE00E9495A90C94D98B8091060C53
:10E6E00081110F9447280091D3101091D4100C5F22
:10E6F0001F4F6AE270E0C8010F94BEB97C0161E26D
:10E7000070E0C8010F94BEB9009719F08C010F5F3B
:10E710001F4FE114F10411F0F701108280E50E940F
:10E720009237F82E2091D3103091D410021713078E
:10E7300008F4F12C8091070C882311F40C94D98BE8
:10E7400021E02F2541E0B80184E09CE00E94D2AD99
:10E7500083E50E9492378823B9F02091D31030913D
:10E76000D4102017310780F40E94BC37AB01BC01E4
:10E770004093A20E5093A30E6093A40E7093A50E27
:10E780008DEE9DE00E94849B84E09CE00E942AA97B
:10E79000F1100C94D98B0F94F6A760932F0B709304
:10E7A000300B8093310B9093320B0C94D98B80916A
:10E7B000D3109091D4106AE270E005960F94BEB920
:10E7C0008C010097A9F08091DD109091DE106EE42D
:10E7D00070E08E519F4E0F94BEB960E270E00F94CE
:10E7E000BEB901969093D4108093D310D8011C9297
:10E7F0006091D3107091D4106B5F7F4F84E09CE0E8
:10E800000E9410B10C94D98B0F94F6A760932B0B38
:10E8100070932C0B80932D0B90932E0B00912F0B4C
:10E820001091300B2091310B3091320B601B710B2A
:10E83000820B930B28EE33E040E050E00F94CEB50E
:10E84000CA01B9012CE330E040E050E00F94CEB5AE
:10E850007F936F933F932F9388EE9AE09F938F93CC
:10E86000CE0101969F938F930F943EBAEDE3F0E1B2
:10E8700084910FB6F894DEBF0FBECDBFEDE3F0E19B
:10E88000882349F09091C00095FFFCCF8093C6008B
:10E8900031968491F5CFFE0131968191882339F02C
:10E8A0009091C00095FFFCCF8093C600F6CF809179
:10E8B000C00085FFFCCF8AE08093C600CE010196A0
:10E8C0000F9417580C94D98B83E50E9492378823B4
:10E8D00011F40C94D98B0E94F2370F944BB1F62EA1
:10E8E000E72E862F9E2D8C0180E50E94923788238B
:10E8F00031F00F3F110509F010F40C940C8D0DE070
:10E9000010E0EBE3F6E0819191918017910711F40B
:10E910000C94D98B26E0E337F207A9F706301105EE
:10E9200039F48F2D9E2D9093700B80936F0B04C044
:10E9300017FF02C00C94D98B61E0802F0F94E1A9DE
:10E940006F2D802F0F941AAA6F2D7E2D802F0F947C
:10E95000C9A80C94D98B8FEF0E94D83B60E070E07F
:10E9600088EF9FE00F9496BC0E940AD90E949DD91F
:10E970000C94D98B8AE50E949237382E811112C0EF
:10E9800010920F1B10920E1B1092111B1092101B55
:10E990001092131B1092121B1092151B1092141B35
:10E9A0000F94605780E00F94105B80E193E10F9427
:10E9B0004C030E949DD90F949A021092760B1092EC
:10E9C000770B1092780B81E00E943E37ECE3F8E27F
:10E9D000859194910E94CA3B0E9404440E948D3EFE
:10E9E000882309F448C10E94374420E030E048E41D
:10E9F00052E46091081B7091091B80910A1B909151
:10EA00000B1B0F940BB3181684F020E030E048E4A1
:10EA100052E46091F61A7091F71A8091F81A909169
:10EA2000F91A0F940BB3181624F4332011F40C9434
:10EA3000138D80E090E0A0EAB0E480938D0B90937A
:10EA40008E0BA0938F0BB093900B20E030E040E250
:10EA500052E4609151027091520280915302909160
:10EA600054020F94E3B04B015C012091890B30916B
:10EA70008A0B40918B0B50918C0B6091850B7091A0
:10EA8000860B8091870B9091880BE1E7FBE0FF9369
:10EA9000EF93E1E9CE2EEBE0DE2EE12CF12C00EA43
:10EAA00010E40F94B10E0F94472886E50E94923728
:10EAB0000F900F908823A1F08091D3109091D410E3
:10EAC000DC0111962C91293069F02F7D71F04AE01C
:10EAD00050E060E070E001960F94CFB768AF07C0D8
:10EAE00018AE05C0B1E0B8AF02C0E1E0E8AF332036
:10EAF000B1F00E946C370E94F2D90E940EDC0E9495
:10EB0000BAF8882309F4B5C087EF9FE00F946ABC78
:10EB1000803F09F0AEC081E00E94D83BAAC08FEFD1
:10EB20000E94D83B60E070E088EF9FE00F9496BCB5
:10EB30001982BE016F5F7F4F88AD0E9411F13C01C9
:10EB40000E946C37212C312C10EA412E10E4512EFA
:10EB500020928D0B30928E0B40928F0B5092900B27
:10EB600020E030E040E252E46091510270915202A4
:10EB700080915302909154020F94E3B04B015C01D9
:10EB80002091890B30918A0B40918B0B50918C0B0B
:10EB90006091850B7091860B8091870B9091880B0B
:10EBA000A1E7BBE0BF93AF9301E9C02E0BE0D02EED
:10EBB000820171010F94B10E0F9447280F900F90AE
:10EBC00077FC48C0198280E193E10F944C030E94C6
:10EBD00064D981E00E943E370E940444AE014F5F39
:10EBE0005F4F68AD81E00E94D2FA3C010E946C3711
:10EBF00020928D0B30928E0B40928F0B5092900B87
:10EC000020E030E040E252E4609151027091520203
:10EC100080915302909154020F94E3B04B015C0138
:10EC20002091890B30918A0B40918B0B50918C0B6A
:10EC30006091850B7091860B8091870B9091880B6A
:10EC4000A1E7BBE0BF93AF930F94B10E0F94472899
:10EC50000F900F906981C3010F94515D77FC09C03B
:10EC600086EE0E94D83BE6E3F8E2859194910F94FA
:10EC7000185D0F94594481E00F94105B0C94D98B6C
:10EC80000F94D9700C94D98B88E690E00E94E44CE4
:10EC900081110C94D98B83E50E949237882371F0FF
:10ECA0000091260B0E94F23710E0000F111F005F49
:10ECB000144E0F944BB1D8016D937C930F94763220
:10ECC0000C94D98B0E94B54B83E50E949237882320
:10ECD00011F40C94D98B0E94F2370F944BB17093BE
:10ECE0000F1B60930E1B0C94D98B89E690E00E9459
:10ECF000E44C81110C94D98BE2EEFAE084918823E4
:10ED000041F09091C00095FFFCCF8093C6003196F2
:10ED1000F5CFE091260BB4E0EB9FF0011124E85F02
:10ED2000F44E408151816281738121E030E08EE3B5
:10ED30009AE00E94E136EFEDFAE08491882341F0F9
:10ED40009091C00095FFFCCF8093C6003196F5CF1F
:10ED5000E091260BF0E0EE0FFF1FE05FF44E6081C4
:10ED60007181882777FD8095982F0F947EB1AB0134
:10ED7000BC0121E030E08EE39AE00E94E136EBED49
:10ED8000FAE08491882341F09091C00095FFFCCF78
:10ED90008093C6003196F5CF4091F61A5091F71A3C
:10EDA0006091F81A7091F91A21E030E08EE39AE050
:10EDB0000E94E136E8EDFAE08491882341F09091D9
:10EDC000C00095FFFCCF8093C6003196F5CF6091CF
:10EDD0000E1B70910F1B882777FD8095982F0F943D
:10EDE0007EB1AB01BC0121E030E08EE39AE00E94ED
:10EDF000E136E5EDFAE08491882341F09091C0007E
:10EE000095FFFCCF8093C6003196F5CF4AE050E0E5
:10EE100060E070E08EE39AE00E94E335E3EDFAE013
:10EE20008491882341F09091C00095FFFCCF80939E
:10EE3000C6003196F5CF4091081B5091091B609197
:10EE40000A1B70910B1B21E030E08EE39AE00E94D8
:10EE5000E136E0EDFAE08491882341F09091C00022
:10EE600095FFFCCF8093C6003196F5CF6091101BC3
:10EE70007091111B882777FD8095982F0F947EB194
:10EE8000AB01BC0121E030E08EE39AE00E94E13664
:10EE9000ECECFAE08491882341F09091C00095FF5A
:10EEA000FCCF8093C6003196F5CF8091260B90E081
:10EEB0000F94F72F4AE050E0BC018EE39AE00E94E5
:10EEC000E335E7ECFAE08491882341F09091C000AB
:10EED00095FFFCCF8093C6003196F5CF8FEF9FEF63
:10EEE0000F94F72F4AE050E0BC018EE39AE00E94B5
:10EEF000E335E3ECFAE08491882341F09091C0007F
:10EF000095FFFCCF8093C6003196F5CF4091021B50
:10EF10005091031B6091041B7091051B21E030E0B0
:10EF20008EE39AE00E94E136EFEBFAE084918823C9
:10EF300041F09091C00095FFFCCF8093C6003196C0
:10EF4000F5CF4091FC1A5091FD1A6091FE1A709114
:10EF5000FF1A21E030E08EE39AE00E94E1368091D2
:10EF6000C00085FFFCCF8AE08093C6000C944E8DD4
:10EF70008DE690E00E94E44C81110C94D98BEAEA72
:10EF8000F7E2859194910F94245881E090E090935A
:10EF9000BA0B8093B90B80911B1C882321F081E070
:10EFA00090E00F94925783E50E949237882391F066
:10EFB0000091260B0E94F23710E0000F111F005F36
:10EFC000144E0F944BB1F8017183608381E08093FC
:10EFD000060215C082E50E949237882381F00091D5
:10EFE000260B0E94F23710E0000F111F005F144E35
:10EFF0000F944BB1D8016D937C93109206020F943D
:10F0000076320F94F6A76B017C010091260B10E07D
:10F01000F801EE0FFF1FE05FF44E608171818827D9
:10F0200077FD8095982F0F947EB1F801EE0FFF1FAA
:10F03000EE0FFF1FE85FF44E11E020813181428125
:10F0400053810F940BB318160CF010E01093240B9F
:10F050001092600BC701B6010E946D4EE8EAF7E21C
:10F06000859194910F94245882E090E09093BA0B8C
:10F070008093B90B80911B1C882321F082E090E0E3
:10F080000F9492570F94F6A76093370B7093380B39
:10F090008093390B90933A0B0C94D98BE4E2F8E20D
:10F0A000859194910F94245883E090E09093BA0B4B
:10F0B0008093B90B80911B1C882321F081E090E0A4
:10F0C0000F94925783E50E949237882361F00E9443
:10F0D000F2370F944BB170930F1B60930E1B81E0BE
:10F0E000809306020FC082E50E949237882351F078
:10F0F0000E94F2370F944BB170930F1B60930E1B5D
:10F10000109206020F94F6A72B013C011092600B9F
:10F1100060910E1B70910F1B882777FD8095982FAB
:10F120000F947EB111E02091F61A3091F71A4091B8
:10F13000F81A5091F91A0F940BB318160CF010E04E
:10F140001093240B0CEB1AE098EBE92E9AE0F92EC1
:10F1500024EBA22E2AE0B22E3AE0D32E8091240B8B
:10F1600060910E1B70910F1B882309F490C0809151
:10F17000600B81118CC0882777FD8095982F0F94A4
:10F180007EB12091F61A3091F71A4091F81A5091F9
:10F19000F91A0F940BB318160CF090C00F94F6A741
:10F1A0006419750986099709693E734081059105BF
:10F1B00008F464C080911B1C81115CC0E091710B4C
:10F1C00024E0E29FF0011124E85FF44E4081518178
:10F1D00062817381F8018491ECEBFAE0882349F0B5
:10F1E0009091C00095FFFCCF8093C600319684912A
:10F1F000F5CF22E030E08EE39AE00E94E136F7019D
:10F200008491E8EBFAE0882349F09091C00095FFE3
:10F21000FCCF8093C60031968491F5CF6091710B3D
:10F2200070E04AE050E08EE39AE00E94E335F50199
:10F230008491E4EBFAE0882349F09091C00095FFB7
:10F24000FCCF8093C60031968491F5CF4091F61A99
:10F250005091F71A6091F81A7091F91A21E030E094
:10F260008EE39AE00E94E1368091C00085FFFCCFDA
:10F27000D092C6000F94F6A72B013C010F94DD3904
:10F2800080E00E942A4C80E00F94A35967CF882722
:10F2900077FD8095982F0F947EB12091F61A3091CA
:10F2A000F71A4091F81A5091F91A0F94DCB087FFC1
:10F2B00005C080910602882309F470CFE6E2F8E2E7
:10F2C000859194910F94245884E090E09093BA0B28
:10F2D0008093B90B0F94F6A76093370B7093380B9C
:10F2E0008093390B90933A0B0C94D98B83E50E9451
:10F2F0009237882319F10E94F23720E030E0A9010B
:10F300000F94DCB087FD0FC00E94F23720E030E0A0
:10F310004FE753E40F940BB3181644F00E94F237F2
:10F320000F944BB105C060E070E002C06FEF70E079
:10F330007093700B60936F0B0C94D98B8FEF90E0F0
:10F340009093700B80936F0B0C94D98B1092FF0BE2
:10F350000C94D98B81E08093FF0B0C94D98B83E5BF
:10F360000E949237882399F00E94F23720E030E023
:10F370004AE754E40F94DDB30F9450B16093080250
:10F380007093090280930A0290930B021DC088E5D6
:10F390000E94923781110C942F8D89E50E9492373B
:10F3A00081110C942F8D8AE50E94923781110C9463
:10F3B0002F8D85E40E94923781110C942F8D0F942C
:10F3C0004728149A0F94C9281092B00B0C94D98B2B
:10F3D00083E50E949237882311F40C94D98B0E9404
:10F3E000F23720E030E04AE754E40F94DDB30F94A5
:10F3F00050B16093330B7093340B8093350B909323
:10F40000360B0C94D98B23E736E039AF28AF09EDE2
:10F4100019E1B9EEEB2EB9E1FB2E89E9282E89E13D
:10F42000382ED12CA8ADB9AD8D91B9AFA8AF0E943F
:10F430009237882309F45CC0B3E0DB1252C00E940B
:10F44000F2372B013C0120E030E040EA51E40F9418
:10F45000DCB087FF3FC0A3019201F8016081718198
:10F46000828193810F94E3B04B015C019B01AC015D
:10F470006091B9197091BA198091BB199091BC191A
:10F480000F94DDB36093B9197093BA198093BB19C7
:10F490009093BC19A5019401D7016D917D918D9137
:10F4A0009C910F94DDB3F701608371838283938312
:10F4B000D1016D917D918D919C910F947CB1A501AD
:10F4C00094010F94DDB30F9450B1F1016083718307
:10F4D00082839383D8014D925D926D927C921397B3
:10F4E00007C00E94F237F80160837183828393839F
:10F4F000D3940C5F1F4FF4E0EF0EF11C24E0220EBA
:10F50000311C34E0D3128ECF0C94D98B86E50E9447
:10F5100092378823B9F00F9443A4FC01249122234D
:10F5200041F03091C00035FFFCCF2093C60001961A
:10F53000F4CF8091C00085FFFCCF8AE08093C600A5
:10F540000C94D98B85E50E949237882369F08091CD
:10F55000D3109091D41001969093D4108093D3102F
:10F560000F94B4A60C94D98BE0E8F7E285919491BE
:10F57000FC012491222311F40C94D98B3091C0000A
:10F5800035FFFCCF2093C6000196F2CFEDEAFAE0FA
:10F590008491882341F09091C00095FFFCCF809327
:10F5A000C6003196F5CF4091850B5091860B609146
:10F5B000870B7091880B22E030E08EE39AE00E9486
:10F5C000E136E9EAFAE08491882341F09091C000A5
:10F5D00095FFFCCF8093C6003196F5CF4091890B03
:10F5E00050918A0B60918B0B70918C0B22E030E074
:10F5F0008EE39AE00E94E136E5EAFAE084918823FE
:10F6000041F09091C00095FFFCCF8093C6003196E9
:10F61000F5CF40918D0B50918E0B60918F0B7091B7
:10F62000900B22E030E08EE39AE00E94E136E1EABE
:10F63000FAE08491882341F09091C00095FFFCCFBF
:10F640008093C6003196F5CF4091910B5091920B6B
:10F650006091930B7091940B22E030E08EE39AE07E
:10F660000E94E136E0EFF7E285919491FC0124914C
:10F67000222341F03091C00035FFFCCF2093C6001B
:10F680000196F4CF80E00F94A8280F947EB12091CA
:10F69000D9193091DA194091DB195091DC190F9486
:10F6A000E3B0AB01BC0122E030E08EE39AE00E94BF
:10F6B000E136EDE9FAE08491882341F09091C000B1
:10F6C00095FFFCCF8093C6003196F5CF81E00F9473
:10F6D000A8280F947EB12091DD193091DE19409158
:10F6E000DF195091E0190F94E3B0AB01BC0122E0A7
:10F6F00030E08EE39AE00E94E136E9E9FAE0849195
:10F70000882341F09091C00095FFFCCF8093C60004
:10F710003196F5CF82E00F94A8280F947EB1209106
:10F72000E1193091E2194091E3195091E4190F94D5
:10F73000E3B0AB01BC0122E030E08EE39AE00E942E
:10F74000E136E5E9FAE08491882341F09091C00028
:10F7500095FFFCCF8093C6003196F5CF83E00F94E0
:10F76000A8280F947EB12091E5193091E6194091B7
:10F77000E7195091E8190F94E3B0AB01BC0122E006
:10F7800030E08EE39AE00E94E1368091C00085FF70
:10F79000FCCF8AE08093C6000C94D98B80E00F9454
:10F7A000D41E0C94D98B81E00F94D41E0C94D98B69
:10F7B0003091C00035FFFCCF2093C6000196FC01BC
:10F7C00024912111F5CF8091C00085FFFCCF8AE004
:10F7D0008093C600EAE8F6E285919491FC012491B9
:10F7E000222341F03091C00035FFFCCF2093C600AA
:10F7F0000196F4CF1E9B10C0E2EEF7E28591949142
:10F80000FC0124912223C1F03091C00035FFFCCFD0
:10F810002093C6000196F4CFE0EEF7E28591949133
:10F82000FC012491222341F03091C00035FFFCCF30
:10F830002093C6000196F4CF8091C00085FFFCCFD5
:10F840008AE08093C600ECE8F6E285919491FC0191
:10F850002491222341F03091C00035FFFCCF20934A
:10F86000C6000196F4CF8091060182FF10C0E2EE3F
:10F87000F7E285919491FC0124912223C1F030910B
:10F88000C00035FFFCCF2093C6000196F4CFE0EE18
:10F89000F7E285919491FC012491222341F030916B
:10F8A000C00035FFFCCF2093C6000196F4CF8091B5
:10F8B000C00085FFFCCF8AE08093C600E4E8F6E252
:10F8C00085919491FC012491222341F03091C00054
:10F8D00035FFFCCF2093C6000196F4CF1D9B10C0CE
:10F8E000E2EEF7E285919491FC0124912223C1F08C
:10F8F0003091C00035FFFCCF2093C6000196F4CFB5
:10F90000E0EEF7E285919491FC012491222341F0ED
:10F910003091C00035FFFCCF2093C6000196F4CF94
:10F920008091C00085FFFCCF8AE08093C600E6E8A6
:10F93000F6E285919491FC012491222341F03091CB
:10F94000C00035FFFCCF2093C6000196F4CF809114
:10F95000060187FF10C0E2EEF7E285919491FC0169
:10F9600024912223C1F03091C00035FFFCCF2093B9
:10F97000C6000196F4CFE0EEF7E285919491FC0188
:10F980002491222341F03091C00035FFFCCF209319
:10F99000C6000196F4CF8091C00085FFFCCF8AE0BD
:10F9A0008093C600EEE7F6E285919491FC012491E4
:10F9B000222341F03091C00035FFFCCF2093C600D8
:10F9C0000196F4CF1C9B10C0E2EEF7E28591949172
:10F9D000FC0124912223C1F03091C00035FFFCCFFF
:10F9E0002093C6000196F4CFE0EEF7E28591949162
:10F9F000FC012491222341F03091C00035FFFCCF5F
:10FA00002093C6000196F4CF8091C00085FFFCCF03
:10FA10008AE08093C600E0E8F6E285919491FC01CB
:10FA20002491222341F03091C00035FFFCCF209378
:10FA3000C6000196F4CF019910C0E2EEF7E285917D
:10FA40009491FC0124912223C1F03091C00035FF34
:10FA5000FCCF2093C6000196F4CFE0EEF7E285914B
:10FA60009491FC012491222341F03091C00035FF94
:10FA7000FCCF2093C6000196F4CF8091C00085FF93
:10FA8000FCCF8AE08093C6000C94D98B8091710BD7
:10FA90008093260B84E50E949237882329F10E94E7
:10FAA000F2370F9450B16093260B6623E9F0EDE333
:10FAB000F0E18491882341F09091C00095FFFCCF44
:10FAC0008093C6003196F5CFECE7F7E2A591B491AB
:10FAD0008D91882311F40C94D98B9091C00095FFDF
:10FAE000FCCF8093C600F4CF84E40E949237882331
:10FAF00011F40C94D98B0E94F23720E030E0A90178
:10FB00000F94DCB0811103C01092950B32C00091AC
:10FB1000260B10E00E94F237F801EE0FFF1FEE0FE8
:10FB2000FF1FE35CFD4F6083718382839383E090CA
:10FB30003D02F0903E0200913F021091400220E011
:10FB400030E0A901B701C8010F94DCB0811104C0F5
:10FB5000E12CF12C00E410E4C701D80180933D02B0
:10FB600090933E02A0933F02B093400281E08093C5
:10FB7000950B0E94394E0C94D98BD8018D918D0133
:10FB80000E949237882349F00E94F2370F9450B1B7
:10FB9000F7016083718382839383F4E0EF0EF11C9D
:10FBA00026E00737120749F70F94241D0C94D98BD0
:10FBB00003E716E059EEE52E59E1F52ED8018D91B7
:10FBC0008D010E949237882339F00E94F237F701A5
:10FBD0006083718382839383F4E0EF0EF11C26E04F
:10FBE0000737120759F70C94D98B83E50E94923797
:10FBF000882351F00E94F2376093C1197093C219A3
:10FC00008093C3199093C41984E50E949237882386
:10FC100011F40C94D98B0E94F2376093BD19709344
:10FC2000BE198093BF199093C0190C94D98B83E5AA
:10FC30000E949237882351F00E94F2376093C519D1
:10FC40007093C6198093C7199093C81984E50E94D0
:10FC50009237882351F00E94F2376093A91970936C
:10FC6000AA198093AB199093AC1982E40E94923741
:10FC7000882361F00E94F2370F9450B16093F91914
:10FC80007093FA198093FB199093FC1988E50E94F0
:10FC90009237882391F00E94F2376093B1197093E4
:10FCA000B2198093B3199093B4196093AD197093FE
:10FCB000AE198093AF199093B01989E50E949237DD
:10FCC000882351F00E94F2376093B1197093B219F2
:10FCD0008093B3199093B4198AE50E9492378823D0
:10FCE00051F00E94F2376093B5197093B619809362
:10FCF000B7199093B81985E40E949237882311F4BC
:10FD00000C94D98B0E94F2376093B9197093BA1989
:10FD10008093BB199093BC190C94D98B03E716E020
:10FD200049E7E42E4BE0F42ED8018D918D010E941D
:10FD30009237882339F00E94F237F701608371838C
:10FD400082839383F4E0EF0EF11C26E0063712075E
:10FD500059F70C94D98B83E50E949237882351F090
:10FD60000E94F23760931D0270931E0280931F025F
:10FD70009093200286E40E949237882381F00E94AB
:10FD8000F23720E030E040E752E40F94E3B06093B4
:10FD900015027093160280931702909318028AE559
:10FDA0000E949237882311F40C94D98B0E94F23769
:10FDB0006093690B70936A0B80936B0B90936C0B41
:10FDC0000C94D98B83E50E949237882351F00E94CE
:10FDD000F2376093650B7093660B8093670B90937B
:10FDE000680B86E40E949237882311F40C94D98B17
:10FDF0000E94F23720E030E040E752E40F94E3B095
:10FE00006093110270931202809313029093140274
:10FE10000C94D98B83E50E949237882311F40C94BB
:10FE2000D98B0E94F2370F944BB16115710551F0D7
:10FE30006130710569F481E080936E0B10926D0B57
:10FE40000C94D98B10926E0B10926D0B0C94D98B75
:10FE5000EDE3F0E18491882341F09091C00095FF9B
:10FE6000FCCF8093C6003196F5CFECE9F6E28591A0
:10FE70009491FC012491222341F03091C00035FF80
:10FE8000FCCF2093C6000196F4CFE091DD10F091F5
:10FE9000DE10EE51FF4E8191882339F09091C00021
:10FEA00095FFFCCF8093C600F6CFE0E9FAE084919D
:10FEB000882341F09091C00095FFFCCF8093C6004D
:10FEC0003196F5CF8091C00085FFFCCF8AE080930A
:10FED000C6000C94D98B83E50E949237882311F4D5
:10FEE0000C94D98B0E94F2370F944BB17093480257
:10FEF000609347020C94D98B83E50E949237882344
:10FF000011F40C94D98B0E94F2370F944BB16B0112
:10FF10007C0184E50E949237882391F08DED90E07A
:10FF20000E94E44C81110C94D98BE091260BF0E0F7
:10FF3000EE0FFF1FED5BFD4FD182C0820C94D98B79
:10FF4000D0924602C09245020C94D98B80E50E9463
:10FF50009237882311F40C94D98B0E94F2370F94B6
:10FF60004BB1D62E062F172F83E50E949237882398
:10FF700031F00E94F2370F944BB17B0103C0EE24A5
:10FF8000EA94FE2CC7010196039710F00C94D98BCC
:10FF9000EBE3F6E0819191918017910711F40C94B5
:10FFA000D98B26E0E337F207A9F717FF02C00C94BC
:10FFB000D98B0F944728CD2C60E08D2D0F94E1A9AB
:10FFC0003FEFE316F30631F0EA94EF2871F000E01A
:10FFD00010E00DC08D2D0F944FAA31E020E0892B49
:10FFE00009F030E0032F122F02C001E010E08C2D49
:10FFF0000F944FAA8017910711F40C94D98B0F948A
:020000021000EC
:10000000DD3980E00E942A4C80E00F94A359EFCFA5
:1000100083E50E949237882331F00E94F2370F94D3
:100020004BB18B0102C00EE610E080E50E949237D2
:10003000882331F00E94F2370F944BB1CB0102C0FC
:1000400088EE93E06C01EE24D7FCE094FE2C1016B1
:10005000110684F420E030E0A901B80184E50F9492
:1000600044ACC701B6010F9425A884E50F946AAF8C
:100070000C94D98BC701B6010F9425A80C94D98B89
:1000800080E50E949237882351F00E94F2376093F6
:100090009E0270939F028093A0029093A10289E434
:1000A0000E949237882361F00E94F2370F949940A2
:1000B00060939A0270939B0280939C0290939D029E
:1000C00084E40E949237882361F00E94F2370F94F3
:1000D000A540609396027093970280939802909344
:1000E000990283E40E949237882351F00E94F237EC
:1000F000609392027093930280939402909395027E
:100100000F94CA2FE0E5F7E285919491FC012491C8
:10011000222341F03091C00035FFFCCF2093C60070
:100120000196F4CFE0E2F5E08191882339F09091D7
:10013000C00095FFFCCF8093C600F6CF40919E0291
:1001400050919F026091A0027091A10222E030E0E4
:100150008EE39AE00E94E136E4E2F5E081918823A3
:1001600039F09091C00095FFFCCF8093C600F6CF88
:1001700060919A0270919B0280919C0290919D02E5
:100180000F949F40AB01BC0122E030E08EE39AE087
:100190000E94E136E8E2F5E08191882339F0909100
:1001A000C00095FFFCCF8093C600F6CF6091960209
:1001B0007091970280919802909199020F94AB40B0
:1001C000AB01BC0122E030E08EE39AE00E94E13610
:1001D000ECE2F5E08191882339F09091C00095FF21
:1001E000FCCF8093C600F6CF4091920250919302CB
:1001F000609194027091950222E030E08EE39AE0E3
:100200000E94E1368091C00085FFFCCF8AE0809398
:10021000C6000C94D98B80E50E949237882351F058
:100220000E94F23760938E0270938F028093900247
:100230009093910289E40E949237882361F00E9492
:10024000F2370F94994060938A0270938B028093E7
:100250008C0290938D0284E40E949237882361F08F
:100260000E94F2370F94A540609386027093870234
:1002700080938802909389020F94CA2FE0E5F7E2F9
:1002800085919491FC012491222341F03091C0008A
:1002900035FFFCCF2093C6000196F4CFE0E2F5E0F5
:1002A0008191882339F09091C00095FFFCCF809315
:1002B000C600F6CF40918E0250918F02609190025D
:1002C0007091910222E030E08EE39AE00E94E136E4
:1002D000E4E2F5E08191882339F09091C00095FF28
:1002E000FCCF8093C600F6CF60918A0270918B029A
:1002F00080918C0290918D020F949F40AB01BC01C4
:1003000022E030E08EE39AE00E94E136E8E2F5E098
:100310008191882339F09091C00095FFFCCF8093A4
:10032000C600F6CF609186027091870280918802A4
:10033000909189020F94AB40AB01BC0122E030E008
:100340008EE39AE00E94E1368091C00085FFFCCFE9
:100350008AE08093C6000C94D98B83E50E94923783
:10036000882319F00E94F23703C060E070E0CB01EF
:100370000F941B1D0C94D98B85E40E94923788231F
:1003800041F00E94F2370F944BB18B0177FF03C00D
:1003900009C000E010E0812C912C96E1A92E93E495
:1003A000B92E06C0812C912C8CE8A82E82E4B82EA0
:1003B00083E50E949237882321F00E94F2374B0197
:1003C0005C0183E40E949237882331F00E94F23767
:1003D0000F944BB19B0102C025E030E0A801C5019C
:1003E000B4010F948A320C94D98B60E084E190E0E0
:1003F0000E9495240C94D98B60E084E190E00E94E7
:10040000242C0C94D98B80E00E94B5250C94D98BB8
:100410009091C00095FFFCCF8093C60031968491E7
:100420008111F6CFE0E8FAE08491882311F40C946E
:10043000D98B9091C00095FFFCCF8093C600319678
:10044000F3CF8AE50E949237882309F4B0C00E9456
:10045000F2374B015C0120E030E040E751EC0F94B3
:100460000BB387FD4EC020E030E040EA50ECC50100
:10047000B4010F94DCB018160CF443C0B7FAB09472
:10048000B7F8B0948092720B9092730BA092740B99
:10049000B092750BEDE3F0E18491882341F09091E7
:1004A000C00095FFFCCF8093C6003196F5CFE0E504
:1004B000F7E245915491E2E8F6E2859194912FE7B5
:1004C0003AE069EB79E00E9495BDFC01249122237A
:1004D00041F03091C00035FFFCCF2093C60001965B
:1004E000F4CF8091C00085FFFCCF8AE08093C600E6
:1004F0008091C00085FFFCCF8AE08093C6000C94F9
:10050000D98BEDE3F0E18491882341F09091C00014
:1005100095FFFCCF8093C6003196F5CFE2E8F6E276
:1005200085919491FC012491222341F03091C000E7
:1005300035FFFCCF2093C6000196F4CFEEE7F6E23C
:1005400085919491FC012491222341F03091C000C7
:1005500035FFFCCF2093C6000196F4CF4AE050E06F
:1005600061EF7FEF8EE39AE00E94E335E0E8F6E288
:1005700085919491FC012491222341F03091C00097
:1005800035FFFCCF2093C6000196F4CF4AE050E03F
:100590006BEF7FEF8EE39AE00E94E3358091C0001D
:1005A00085FFFCCF8AE08093C6000C94D98BEDE3E5
:1005B000F0E18491882341F09091C00095FFFCCF39
:1005C0008093C6003196F5CFE2E8F6E285919491EA
:1005D0006BE77AE00E9474BDFC012491222341F074
:1005E0003091C00035FFFCCF2093C6000196F4CFB8
:1005F0008091C00085FFFCCF8AE08093C6004091C7
:10060000720B5091730B6091740B7091750B705855
:1006100022E030E08EE39AE00E94E1368091C00053
:1006200085FFFCCF8AE08093C6000C94D98B60E3F1
:1006300075E08EE39AE00E94D6350F9447288091AA
:100640001B1C882321F086E190E00F949257809143
:100650004702909148029093420280934102C090D9
:10066000850BD090860BE090870BF090880BCF8E97
:10067000D8A2E9A2FAA20091890B10918A0B2091CD
:100680008B0B30918C0B0BA31CA32DA33EA340918D
:100690008D0B50918E0B60918F0B7091900B4FA32F
:1006A00058A769A77AA78091910B9091920BA0917E
:1006B000930BB091940B8BA79CA7ADA7BEA7C98243
:1006C000DA82EB82FC820D831E832F833887498771
:1006D0005A876B877C878D879E87AF87B88B85E429
:1006E0000E949237882359F00E94F2379B01AC0197
:1006F0006BA57CA58DA59EA50F94ECAF0AC020E04C
:1007000030E040E050E46BA57CA58DA59EA50F943C
:10071000EBAF6BA77CA78DA79EA7EFA0F8A409A5B8
:100720001AA52BA13CA14DA15EA16F8D78A189A135
:100730009AA1E1E7FBE0FF93EF93812C912CB8ECB9
:10074000AB2EB3E4BB2EDE019B966D010F94B10E70
:100750008AE50E9492370F900F90882349F00E94FB
:10076000F2379B01AC016FA178A589A59AA51EC09F
:1007700020E030E040E050E46FA178A589A59AA57B
:100780000F94ECAF4B015C016FA378A789A79AA7E0
:1007900020E030E040E251E40F94DCB087FF0CC071
:1007A00020E030E040E251E4C501B4010F94ECAF29
:1007B0006FA378A789A79AA7EFA0F8A409A51AA5FF
:1007C0002BA13CA14DA15EA16F8D78A189A19AA119
:1007D000E1E7FBE0FF93EF93812C912CA0E7AA2E99
:1007E000A1E4BA2EFE01BB966F010F94B10E88E50D
:1007F0000E9492370F900F90882379F00E94F23771
:100800009B01AC016F8D78A189A19AA10F94ECAFE7
:100810006F8F78A389A39AA308C080E090E0A3E536
:10082000B3E48F8F98A3A9A3BAA389E50E94923756
:10083000882339F00E94F2376BA37CA38DA39EA37B
:1008400004C01BA21CA21DA21EA2EFA0F8A409A511
:100850001AA52BA13CA14DA15EA16F8D78A189A104
:100860009AA1E1E7FBE0FF93EF93812C912CF8E450
:10087000AF2EF2E4BF2EDE019B966D010F94B10EF8
:100880000F94472881E08093B60BEAE9F6E2859160
:1008900094910F9424588CE40E9492370F900F90FB
:1008A000882359F00E94F2379B01AC016BA57CA50F
:1008B0008DA59EA50F94ECAF0AC020E030E040EA81
:1008C00052E46BA57CA58DA59EA50F94EBAF6BA7FD
:1008D0007CA78DA79EA7EFA0F8A409A51AA52BA118
:1008E0003CA14DA15EA16F8D78A189A19AA1E1E7FC
:1008F000FBE0FF93EF93812C912CE8ECAE2EE3E428
:10090000BE2EFE01BB966F010F94B10E0F944728C7
:10091000149A64E670E080E090E00F9425A80F94AC
:100920003D750F94F6A76093C50B7093C60B80932B
:10093000C70B9093C80B0F900F9000E010E0F12CC4
:100940000F942B5C81112AC0F3940F94DD3981E060
:100950000E942A4CF110F4CF043FF1E01F0711F47C
:1009600000E010E080910101846080930101011595
:10097000110531F49FB7F89480910201846008C09A
:100980000431110541F49FB7F894809102018B7FE7
:10099000809302019FBF0F5F1F4FD2CF9FB7F89484
:1009A000809102018B7F809302019FBF20E030E0A5
:1009B0004CE852E46BA57CA58DA59EA50F94ECAFE9
:1009C0006BA77CA78DA79EA7EFA0F8A409A51AA5E1
:1009D0002BA13CA14DA15EA16F8D78A189A19AA107
:1009E000F1E76F2EFBE07F2E7F926F92812C912C8E
:1009F000A0EAAA2EA1E4BA2EDE019B966D010F9407
:100A0000B10E20E030E048E452E46BA57CA58DA552
:100A10009EA50F94ECAF6BA77CA78DA79EA7EFA018
:100A2000F8A409A51AA52BA13CA14DA15EA16F8D2B
:100A300078A189A19AA17F926F92812C912CA12CEF
:100A4000B0E4BB2E0F94B10E1092E80B1092E70B9E
:100A50000F94A5750F900F900F900F908091E70B5A
:100A60009091E80B019709F48CC01092E80B10925A
:100A7000E70B0F94E5758091E70B9091E80B8230BE
:100A8000910571F1039709F076C020E030E048E469
:100A900052E46BA57CA58DA59EA50F94ECAF6BA72A
:100AA0007CA78DA79EA7EFA0F8A409A51AA52BA146
:100AB0003CA14DA15EA16F8D78A189A19AA17F92E1
:100AC0006F92812C912CA12CA0E4BA2EDE019B9672
:100AD0006D010F94B10E0F9465750F900F90BECFFE
:100AE00020E030E04CE852E46BA57CA58DA59EA5E6
:100AF0000F94ECAF6BA77CA78DA79EA7EFA0F8A4DF
:100B000009A51AA52BA13CA14DA15EA16F8D78A1CD
:100B100089A19AA17F926F92812C912CB0EAAB2E81
:100B2000B1E4BB2EDE019B966D010F94B10E20E067
:100B300030E048E452E46BA57CA58DA59EA50F94FA
:100B4000ECAF6BA77CA78DA79EA7EFA0F8A409A583
:100B50001AA52BA13CA14DA15EA16F8D78A189A101
:100B60009AA17F926F92812C912CA12CE0E4BE2E51
:100B70000F94B10E6DCF0F94577581E00F94105BF9
:100B80006DCF20E030E040EA50E46BA57CA58DA558
:100B90009EA50F94ECAF6BA77CA78DA79EA7EFA097
:100BA000F8A409A51AA52BA13CA14DA15EA16F8DAA
:100BB00078A189A19AA1E1E76E2EEBE07E2E7F92CB
:100BC0006F92812C912CA12CF0E4BF2EFE01BB96DC
:100BD0006F010F94B10EA50194016BA57CA58DA5A5
:100BE0009EA50F94EBAF6BA77CA78DA79EA7EFA048
:100BF000F8A409A51AA52BA13CA14DA15EA16F8D5A
:100C000078A189A19AA17F926F92812C912CA8EC56
:100C1000AA2EA3E4BA2E0F94B10EEFA0F8A409A552
:100C20001AA52D813E814F81588569817A818B81FA
:100C30009C817F926F92812C912CB8E4AB2EB2E410
:100C4000BB2E0F94B10EE984FA840B851C852D818F
:100C50003E814F81588569817A818B819C817F9209
:100C60006F92812C912CE0E7AE2EE1E4BE2E0F9422
:100C7000B10E20E030E040E050E46BA57CA58DA5EE
:100C80009EA50F94ECAF6BA77CA78DA79EA7E984C8
:100C9000FA840B851C852D813E814F8158856981A1
:100CA0007A818B819C817F926F92812C912CF8ECC0
:100CB000AF2EF3E4BF2E0F94B10ECE010D960F941C
:100CC000FE1C8091410290914202809347029093D2
:100CD00048029F938F9382E79AE09F938F938E01B0
:100CE000015D1F4F1F930F930F943EBA60E0C80140
:100CF0000E9410B4ECE7F6E2859194910F94245889
:100D00001092B60B1092B40B1092B30B0FB6F8946E
:100D1000DEBF0FBECDBF8091CF12882309F449C535
:100D20000E943AB30F9447280E94AAB5811105C0CA
:100D30000E94385C0E943AB3F7CF0E9452BB0E94D7
:100D40004DBB37C580911F1C9091201C892B09F049
:100D500030C585E090E09093201C80931F1C29C52E
:100D600080911F1C9091201C892B09F022C586E0E0
:100D700090E09093201C80931F1C1BC50E943E3D59
:100D800018C588E50E949237882339F00E94F2370F
:100D90000F944BB180E00F94BF298AE50E949237EF
:100DA000882339F00E94F2370F944BB181E00F9401
:100DB000BF2985E40E949237882309F4FAC40E946F
:100DC000F2370F944BB182E00F94BF29F2C40F9415
:100DD0005A45EFC488E50E949237882339F00E9473
:100DE000F2370F9450B180E00F94D84489E50E9407
:100DF0009237882339F00E94F2370F9450B181E086
:100E00000F94D8448AE50E949237882339F00E94D3
:100E1000F2370F9450B182E00F94D84485E40E94D9
:100E20009237882309F4C5C40E94F2370F9450B159
:100E300083E00F94D844BDC488E50E94923788238C
:100E400039F00E94F2370F9450B180E00F941945A9
:100E500089E50E949237882339F00E94F2370F9477
:100E600050B181E00F9419458AE50E94923788239A
:100E700039F00E94F2370F9450B182E00F94194577
:100E800085E40E949237882309F493C40E94F237C4
:100E90000F9450B183E00F9419458BC40F946541B2
:100EA00088C481E080937B1B0F945A4582C488E5F7
:100EB0000E949237882331F00E94F2370F9450B18C
:100EC0006093A70289E50E949237882331F00E943F
:100ED000F2370F9450B16093A8028AE50E949237CE
:100EE000882331F00E94F2370F9450B16093A90229
:100EF00085E40E949237882331F00E94F2370F94E4
:100F000050B16093AA02EDE3F5E08191882339F0B6
:100F10009091C00095FFFCCF8093C600F6CF4AE0C9
:100F200050E06091A7028EE39AE00E942E36E0E541
:100F3000F5E08191882339F09091C00095FFFCCFB6
:100F40008093C600F6CF4AE050E06091A8028EE39D
:100F50009AE00E942E36E3E6F5E08191882339F08D
:100F60009091C00095FFFCCF8093C600F6CF4AE079
:100F700050E06091A9028EE39AE00E942E36E6E7E7
:100F8000F5E08191882339F09091C00095FFFCCF66
:100F90008093C600F6CF4AE050E06091AA028EE34B
:100FA0009AE00E942E3605C488E50E949237882375
:100FB00039F00E94F2370F9450B180E00F94D9427B
:100FC00089E50E949237882339F00E94F2370F9406
:100FD00050B181E00F94D9428AE50E94923788236C
:100FE00039F00E94F2370F9450B182E00F94D94249
:100FF00085E40E949237882309F4DBC30E94F2370C
:101000000F9450B183E00F94D942D3C388E50E9476
:101010009237882339F00E94F2370F9450B180E064
:101020000F94304389E50E949237882339F00E945B
:10103000F2370F9450B181E00F9430438AE50E945B
:101040009237882339F00E94F2370F9450B182E032
:101050000F94304385E40E949237882309F4A9C392
:101060000E94F2370F9450B183E00F943043A1C334
:10107000159881E08093B60B82E090E09093B40BDA
:101080008093B30BECE8F7E2859194910F94245888
:1010900020E030E04CE852E46091910B7091920BAB
:1010A0008091930B9091940B0F94ECAF6093910B04
:1010B0007093920B8093930B9093940BE0908D0B15
:1010C000F0908E0B00918F0B1091900B2091890B5B
:1010D00030918A0B40918B0B50918C0B6091850B5A
:1010E0007091860B8091870B9091880BE1E76E2EB3
:1010F000EBE07E2E7F926F92812C912CF0ECAF2E44
:10110000F0E4BF2EA1E9CA2EABE0DA2E0F94B10EA7
:1011100020E030E048EC51E46091910B7091920B2B
:101120008091930B9091940B0F94ECAF6093910B83
:101130007093920B8093930B9093940BE0908D0B94
:10114000F0908E0B00918F0B1091900B2091890BDA
:1011500030918A0B40918B0B50918C0B6091850BD9
:101160007091860B8091870B9091880B7F926F9284
:10117000812C912CB0E8AB2EBFE3BB2E0F94B10EA7
:101180000F9447280F900F900F900F9080911B1C89
:101190008823A9F081E00F94105B82E00F94A3599B
:1011A000ECE7F6E2859194910F9424581092B50BD8
:1011B0001092B60B1092B40B1092B30BFAC280913E
:1011C000B50B882339F300EC602E07E2702EF30193
:1011D0008591949141E060E00F94907F91E08111BE
:1011E00001C090E011E7412E1BE0512E9111D2CFAA
:1011F00081E00F94105B82E00F94A35920E030E06F
:1012000048EC51E46091910B7091920B8091930B9B
:101210009091940B0F94ECAF6093910B7093920BA1
:101220008093930B9093940BE0908D0BF0908E0B2A
:1012300000918F0B1091900B2091890B30918A0BAC
:1012400040918B0B50918C0B6091850B7091860BAC
:101250008091870B9091880B5F924F92812C912CFB
:10126000A0E8AA2EAFE3BA2EB1E9CB2EBBE0DB2E6D
:101270000F94B10E0F944728F3018591949141E0AA
:1012800060E00F94907F0F900F90811183CFB0CFCB
:1012900081E08093B60B82E090E09093B40B809352
:1012A000B30BEAE9F6E2859194910F94245820E07B
:1012B00030E040EA52E46091910B7091920B809182
:1012C000930B9091940B0F94EBAF6093910B7093F1
:1012D000920B8093930B9093940BE0908D0BF09076
:1012E0008E0B00918F0B1091900B2091890B3091F8
:1012F0008A0B40918B0B50918C0B6091850B7091F8
:10130000860B8091870B9091880BE1E7FBE0FF93C0
:10131000EF93812C912CE8EEAE2EE2E4BE2EF1E9A3
:10132000CF2EFBE0DF2E0F94B10E0F944728ECE791
:10133000F6E2859194910F9424581092B60B109276
:10134000B40B1092B30B0F900F9033C2E2E6FAE0A9
:101350008491882341F09091C00095FFFCCF809349
:10136000C6003196F5CF8091C00085FFFCCF8AE0A2
:101370008093C6001EC284E50E949237882309F438
:10138000D1C0E091D310F091D41031968191803288
:10139000E9F38930D9F390ED980F9A30E0F08F336C
:1013A000A9F0E2E5FAE08491882341F09091C00031
:1013B00095FFFCCF8093C6003196F5CF8091C00099
:1013C00085FFFCCF8AE08093C600F3C10F9439A358
:1013D0008093260B06C00E94F2370F9450B16093A1
:1013E000260B2091260B81E090E0022E01C0880F91
:1013F0000A94EAF79091B00B982B9093B00B2223AC
:1014000009F442C0EDE3F0E18491882341F090912A
:10141000C00095FFFCCF8093C6003196F5CFE0E584
:10142000FAE08491882341F09091C00095FFFCCFB1
:101430008093C6003196F5CF6091260B70E04AE0AC
:1014400050E08EE39AE00E94E3358091C00085FF72
:10145000FCCF8AE08093C600E4E9F7E2859194919D
:10146000FC012491222341F03091C00035FFFCCFD4
:101470002093C6000196F4CF8091C00085FFFCCF79
:101480008AE08093C60095C186E40E949237882343
:10149000D9F00E94F2374B015C016093400B7093CE
:1014A000410B8093420B9093430B20E030E0A90165
:1014B0000F940BB3181644F480920C0290920D0214
:1014C000A0920E02B0920F02EDE3F0E18491882326
:1014D00041F09091C00095FFFCCF8093C6003196FB
:1014E000F5CFE2E4F8E285919491FC012491222366
:1014F00041F03091C00035FFFCCF2093C60001962B
:10150000F4CF6091710B70E04AE050E08EE39AE016
:101510000E94E3358091C00085FFFCCF8AE0809374
:10152000C60047C184E40E949237882309F400C1B1
:101530000E94F2370F944BB167307105D9F1BCF4BA
:101540006330710509F43FC054F461307105A9F1AD
:10155000BCF5672B09F02DC10E94D42D2AC165303E
:101560007105A1F10CF0B6C00E948C2F22C1673E1C
:10157000F3E07F0709F467C07CF46A30710509F471
:101580004FC06C30710509F44FC06830710509F027
:1015900010C1E9E8F5E0BEC0693E33E0730709F425
:1015A0008EC00CF486C0653A734209F002C10E94F5
:1015B0000E30FFC0E6E9F5E098C00E94EA2DF9C0C0
:1015C0000E94012EF6C00E94C22EF3C064EA75E0AC
:1015D0008EE39AE00E94D63580E50E9492378823F8
:1015E00041F00E94F2370F944BB17093C40A60939C
:1015F000C30AEEEAF5E08191882339F09091C000AA
:1016000095FFFCCF8093C600F6CF6091C30A70911E
:10161000C40A4AE050E08EE39AE00E94EA35C9C06D
:1016200086EE0E94D83BC5C060E086E69FE00F943E
:101630007CBC60E085E69FE00F947CBC60E084E6C3
:101640009FE00F947CBC64EC75E08EE39AE00E940E
:10165000D6350F94472881E00F94105B0F940D57F7
:1016600082E00F94A35986E69FE00F946ABC61E084
:10167000680F86E69FE00F947CBC81E00F94105BBE
:1016800082E00F94A359ECE7F6E2859194910F94D0
:10169000245861E08AE49AE00E9410B461E084E496
:1016A0009AE00E9410B461E08EE39AE00E9410B4C8
:1016B00080C00E94165B81E08093A2027AC01092E3
:1016C000060C60E084E09CE00E9462AD81E08093C3
:1016D000A2026FC081E090E00E94E23F6AC0909158
:1016E000C00095FFFCCF8093C60081918111F7CF98
:1016F00068EC88EC0F9450094AE050E0BC018EE39E
:101700009AE00E94EA3555C09091C00095FFFCCF49
:101710008093C60081918111F7CF85E70F941F2C2C
:101720004AE050E0BC018EE39AE00E94EA3541C0F5
:10173000EDE3F0E18491882341F09091C00095FFA2
:10174000FCCF8093C6003196F5CFECE9F6E28591A7
:101750009491FC012491222341F03091C00035FF87
:10176000FCCF2093C6000196F4CFE091DD10F091FC
:10177000DE10EE51FF4E8191882339F09091C00028
:1017800095FFFCCF8093C600F6CFE9E3FAE08491A1
:10179000882341F09091C00095FFFCCF8093C60054
:1017A0003196F5CF8091C00085FFFCCF8AE0809311
:1017B000C6000E94044572C180905C0B90905D0B46
:1017C000A0905E0BB0905F0B2091910B3091920B2B
:1017D0004091930B5091940BC501B4010F94EBAF62
:1017E0002DEC3CEC4CEC5DE30F940BB3181614F0AD
:1017F0000C94FE5E8092910B9092920BA092930BB0
:10180000B092940B81E99BE00F94FE1C60E080E0B5
:101810000E94284943C10E94F2372091790B3091F0
:101820007A0B40917B0B50917C0B0F94ECAF609343
:10183000850B7093860B8093870B9093880B0C9489
:1018400011600E94F23720917D0B30917E0B409108
:101850007F0B5091800B0F94ECAF6093890B7093CA
:101860008A0B80938B0B90938C0B0C941E600E94C0
:10187000F2372091810B3091820B4091830B509174
:10188000840B0F94ECAF60938D0B70938E0B809351
:101890008F0B9093900B0C941F61711028C06620E1
:1018A00031F181E0809310130F94B6286B017C0115
:1018B00080E00F94B628AB01BC019701860180E15E
:1018C00093E10E94FB379B01AC0160918D0B7091FD
:1018D0008E0B80918F0B9091900B0F94EBAF6093D8
:1018E0008D0B70938E0B80938F0B9093900B809148
:1018F0001B1C882321F084E190E00F9492571092F2
:10190000F00BE5EAFEE08491882341F09091C0005D
:1019100095FFFCCF8093C6003196F5CF0E941A5BED
:10192000E9E9FEE08491882341F09091C00095FFA1
:10193000FCCF8093C6003196F5CF0E94805BEDE826
:10194000FEE08491882341F09091C00095FFFCCF88
:101950008093C6003196F5CF0E94DC5B2ACF20E051
:1019600030E040E85FE36091910B7091920B8091C1
:10197000930B9091940B0F94ECAF6093910B709339
:10198000920B8093930B9093940BE0908D0BF090BF
:101990008E0B00918F0B1091900B2091890B309141
:1019A0008A0B40918B0B50918C0B6091850B709141
:1019B000860B8091870B9091880BE1E7FBE0FF930A
:1019C000EF93812C912CA8ECAA2EA3E4BA2EB1E9B6
:1019D000CB2EBBE0DB2E0F94B10E0F900F900C942A
:1019E000066E0F94DD3981E00E942A4C80E00F944E
:1019F000A3590C944F720E94BC37AB01BC014093B9
:101A0000A20E5093A30E6093A40E7093A50E8DEEBC
:101A10009DE00E94849BCDCE0E94F2370F944BB183
:101A20008B010C9481740F94326BEEE4F7E2859194
:101A300094910F94185DE8EBF7E2859194910E94E0
:101A4000CA3B41E050E062E080E00F941857E6EBBB
:101A5000F7E2859194910F94956C0C9419750F94FD
:101A6000472888E50E949237882319F0179A109228
:101A7000760B89E50E949237882319F0169A109206
:101A8000770B8AE50E94923785E40E94923788237B
:101A900011F40C94E479149A0C94E479C75ADF4F4A
:101AA0000FB6F894DEBF0FBECDBFDF91CF911F916F
:101AB0000F91FF90EF90DF90CF90BF90AF909F90ED
:101AC0008F907F906F905F904F903F902F900895F0
:101AD0000F931F93CF93DF931F92CDB7DEB7809103
:101AE000E90B9091EA0B892BA1F00F94F6A70091D6
:101AF000270B1091280B2091290B30912A0B601B8A
:101B0000710B820B930B693E73408105910508F0C0
:101B1000B1C08091E90B9091EA0B892B11F41092DE
:101B2000F10B8091C10B882319F00E9459447EC0AB
:101B30000E94B3B560E084E09CE00E946CAC8091B0
:101B4000D9109091DA10892B09F470C01092D81036
:101B50008091040C8823B1F00091DD101091DE100B
:101B60000E511F4E62ED7EE0C8010F9469B9892BBA
:101B700009F5B80184E09CE00E94BBAB8091050CA4
:101B8000882319F00E94385C31C0E0E5F7E28591C6
:101B90009491FC012491222341F03091C00035FF43
:101BA000FCCF2093C6000196F4CF8091C00085FF42
:101BB000FCCF19C060E084E09CE00E9462ADECEBD9
:101BC000F7E285919491FC012491222341F0309118
:101BD000C00035FFFCCF2093C6000196F4CF809162
:101BE000C00085FFFCCF8AE08093C6008091D810AA
:101BF00081111CC08091D9109091DA10892BB1F01D
:101C0000F89410E090E0E091DD10F091DE10E152E8
